:10800000000001209D500200D91D0200D91D020070
:10801000D91D0200D91D0200D91D02000000000078
:10802000000000000000000000000000D91D020058
:10803000D91D020000000000D91D0200F5C3010097
:10804000D91D0200D91D0200D91D0200D91D020050
:10805000D91D0200D91D0200D91D0200D91D020040
:10806000D91D0200D91D0200D91D0200D91D020030
:10807000D91D0200D91D0200D91D0200D91D020020
:10808000D91D0200D91D0200D91D0200D91D020010
:10809000D91D0200D91D0200D91D0200D91D020000
:1080A000D91D0200D91D0200D91D0200D91D0200F0
:1080B000D91D0200D91D0200D91D0200D91D0200E0
:1080C000D91D0200D91D0200D91D0200D91D0200D0
:1080D000D91D0200D91D0200D91D0200D91D0200C0
:1080E000D91D0200D91D0200D91D0200D91D0200B0
:1080F000D91D020019D70100D91D0200D91D0200A7
:10810000D91D0200A9DB0100D91D0200D91D020002
:10811000D91D0200F5D40100D91D0200D91D0200AD
:10812000D91D0200D91D0200D91D0200D91D02006F
:10813000D91D0200D91D0200D91D0200C1F20100A3
:1081400081E80100D91D0200D91D0200D91D0200DD
:10815000D91D0200D91D0200D91D0200D91D02003F
:10816000D91D0200CD300200D91D0200D91D020028
:10817000D91D0200D91D0200D91D0200D91D02001F
:10818000D91D0200D91D0200D91D0200D91D02000F
:10819000D91D0200D91D0200D91D0200D91D0200FF
:1081A000BDE70100D91D0200D91D0200D91D020042
:0C81B000D91D0200D91D0200D91D0200DB
:10840000FFFFFFFFFFFFFFFFFFFFFFFF7EF9FFFF03
:1084200010B5054C237833B9044B13B10448AFF3AE
:1084300000800123237010BD0010FF1F000000000A
:10844000087B0200084B10B51BB108490848AFF380
:1084500000800848036803B910BD074B002BFBD010
:10846000BDE81040184700BF000000000410FF1FC7
:10847000087B0200A80FFF1F0000000010B516F0D7
:108480002FFA064B00221A70054B1B689847054BC4
:108490009B69BDE810405B69184700BF400AFF1F99
:1084A000E000FF1F0C550200431E2DE9F047154662
:1084B000072B00F25182DFE813F008000D000D00D9
:1084C0004E006B00AF000101B401FFF7D7FF47F684
:1084D000A85350E0754B764C02280EBF9946A14632
:1084E0001C46744BDF684FF0FF364FF000084FF02A
:1084F000010A3B68D9F800001B6998473B6820686F
:10850000DB6898473B6820685B6998473B68D9F807
:1085100000001B6A984718B90AFA08F326EA03060E
:108520003B6820689B6998473B68D9F800001B6A44
:10853000984718B10AFA08F326EA030608F1010879
:10854000B8F1110F09F1040904F10404D1D1C6F303
:1085500010062E6062E12960032900F20082DFE844
:1085600001F0020C1014534BDB691B681B8832228C
:108570009BB253431B142B6050E14E4BDB695B688D
:10858000F4E74C4BDB699B68F0E74B4B1B69F2E768
:10859000012929602BD01AD3022940F0E081454BF4
:1085A000DC686068236800F5A270DB689847606843
:1085B000236800F5B270DB6898476068236800F5AF
:1085C000A2705B699847236860685B696AE0394B11
:1085D000DC68606823686430DB68984760682368FB
:1085E0008430DB689847236860685B693DE0314B05
:1085F000DC6860682368C430DB689847606823687B
:10860000A430DB68984760682368C4305B6998478A
:10861000236860685B6943E0012929602CD01AD384
:10862000022940F09C81234BDC686068236800F5D8
:10863000A270DB6898476068236800F5B270DB6859
:1086400098476068236800F5A2705B6998472368C3
:1086500060689B6926E0174BDC686068236884309B
:10866000DB689847236860681B69643098476068D6
:10867000236884305B69D0E00E4BDC686068236857
:10868000C430DB68984760682368A430DB6898478B
:1086900060682368C4305B699847236860689B6999
:1086A000A430BAE000F5B270B7E000BF9C2FFF1F06
:1086B000842EFF1F0C550200400AFF1F296000296D
:1086C00056D0012940F04B817D4BDC6860682368FF
:1086D00000F2C460DB6898476068236800F2C460F9
:1086E0009B6998476068236800F2E460DB689847FC
:1086F0006068236800F2E4609B69984760682368BB
:1087000000F20470DB6898476068236800F2047028
:108710009B6998476068236800F22470DB6898477B
:108720006068236800F224709B699847606823683A
:1087300000F24470DB6898476068236800F2447078
:108740009B6998476068236800F26470DB6898470B
:108750006068236800F264709B69984760682368CA
:1087600000F28470DB689847236860689B6952E078
:10877000534BDD6868682B6800F2C460DB6898477B
:1087800068682B6800F2C4605B69984768682B686A
:1087900000F2E460DB68984768682B6800F2E460E8
:1087A0005B69984768682B6800F20470DB6898473B
:1087B00068682B6800F204705B69984768682B68EA
:1087C00000F22470DB68984768682B6800F2247018
:1087D0005B69984768682B6800F24470DB689847CB
:1087E00068682B6800F244705B69984768682B687A
:1087F00000F26470DB68984768682B6800F2647068
:108800005B69984768682B6800F28470DB6898475A
:108810002B6868685B6900F2847098470020BDE8A7
:10882000F087296000294DD0012940F09880244B21
:10883000DC686068236800F28450DB6898476068F1
:10884000236800F284509B6998476068236800F2AF
:10885000A450DB6898476068236800F2A4509B69C5
:1088600098476068236800F2C450DB6898476068E6
:10887000236800F2C4509B6998476068236800F23F
:10888000E450DB6898476068236800F2E4509B6915
:1088900098476068236800F20460DB689847606866
:1088A000236800F204609B6998476068236800F2BF
:1088B0002460DB689847236860689B6949E000BFD3
:1088C0000C550200274BDD6868682B6800F2845065
:1088D000DB68984768682B6800F284505B699847AA
:1088E00068682B6800F2A450DB68984768682B68BA
:1088F00000F2A4505B69984768682B6800F2C45086
:10890000DB68984768682B6800F2C4505B69984739
:1089100068682B6800F2E450DB68984768682B6849
:1089200000F2E4505B69984768682B6800F20460C5
:10893000DB68984768682B6800F204605B699847B9
:1089400068682B6800F22460DB6898472B686868C9
:108950005B6900F2246060E70420BDE8F087022034
:10896000BDE8F0870C55020038B5064C2368C31AE1
:10897000B3F5FA7F054604D3034B9B699B6998477F
:10898000256038BD1C10FF1F0C550200464B474A9E
:10899000DB68596801F59270443110605160596884
:1089A000843191605968C431D160596801F5827190
:1089B0001161596801F5B2715161596801F5D271BF
:1089C0009161596801F5F271D161596801F5097138
:1089D0001162596801F519715162596801F52971DF
:1089E0009162596801F53971D162596801F549718F
:1089F0001163596801F559715163596801F569713D
:108A00009163596801F57971D163596801F2244184
:108A100011645968264A081D243110605160596854
:108A2000643191605968A431D1605968E4311161B1
:108A3000596801F5A2715161596801F5C2719161DE
:108A4000596801F5E271D161596801F5017111624E
:108A5000596801F511715162596801F521719162EE
:108A6000596801F53171D162596801F5417111639D
:108A7000596801F551715163596801F5617191634C
:108A8000596801F57171D1635B6803F204431364A3
:108A9000084B01221A70084B084A1A65084A9A6561
:108AA000084A5A65704700BF0C550200842EFF1F0C
:108AB0009C2FFF1F400AFF1FC82EFF1FA984000024
:108AC0007D84000069890000704702207047022001
:108AD000704770477047022070470220704702209D
:108AE000704701207047704770474369114A124927
:108AF00010B5C3F80422C3F80822104B8365104B4D
:108B0000836183620363C3610E4B43640E4B8364D2
:108B10000E4B0F4A0F4C416243630F49C36303641A
:108B20000E4B4265C16284630465C164C26503661D
:108B300010BD00BFE38A0000CB8A0000C98A000094
:108B4000CF8A0000D38A0000D58A0000DB8A0000AB
:108B5000E98A0000DF8A0000D78A0000E78A000067
:108B6000704700BF0748084AC2670023137053705C
:108B70004FF0FF3280F8783043670267C366683091
:108B8000FFF7B3BFC82EFF1F2C10FF1F0648074A70
:108B900042610023137053704FF0FF320374C360BF
:108BA00082604360FFF7A1BFC82EFF1F4412FF1F62
:108BB00010B50023064C18461A5D590002F0030256
:108BC00001338A40072B40EA0200F5D110BD00BFF7
:108BD0005C14FF1F044900235A5C02F00302C254D4
:108BE0000133072BF8D170475C14FF1F074B1A782D
:108BF00002705A7842709A788270DA78C2701A7964
:108C000002715A7942719B79837170475C14FF1F1E
:108C1000F8B5094B094F0A4DDE680024E15D336861
:108C20006A6CDB6952F8240001F0030101349847B3
:108C3000072CF3D1F8BD00BF0C5502005C14FF1FD8
:108C40000800FF1F054A002300F003019954013377
:108C5000072B4FEA9000F7D1DAE700BF5C14FF1F43
:108C6000014B586AEEE700BF0800FF1F04490023CC
:108C7000C25C02F003025A540133072BF8D1C7E754
:108C80005C14FF1F074B02781A7042785A70827882
:108C90009A70C278DA7002791A7142795A718279BF
:108CA0009A71B5E75C14FF1F074B1A68821AB2F578
:108CB0007A7F04D39A685A6000229A6018609A6892
:108CC00001329A60704700BF7014FF1F0020704788
:108CD00001207047014B00225A607047C82EFF1FC9
:108CE00010B50C4614F026F8206010BD14F04EB8F4
:108CF000022804BF0B4B93F8D00020B90A4BDB6865
:108D00001B689B690AE001280BD1064B93F8D03011
:108D1000012B06D1044BDB681B685B69034A1068B2
:108D200018477047C82EFF1F0C550200E42FFF1F85
:108D300010B50020FFF7DCFF044B054ADB68106824
:108D40001B68BDE810409B68184700BF0C55020027
:108D5000E42FFF1F4B2938B50446154600F0D78293
:108D600056D83B2900F0C9812ED82E2900F04B811E
:108D700013D82A2900F0DF8009D8282900F0A5801F
:108D800000F2BE80272900F0928000F016BC2C294A
:108D900000F0038140F2E6801AE1332900F0798186
:108DA00009D8302900F05A81C0F04581312900F0FE
:108DB0005E8100F002BC392900F0858100F28D81CE
:108DC000342900F06F81F8E3432900F02A820FD89C
:108DD0003F2900F0DE8105D83D2900F0B48140F242
:108DE0009F81C3E1412900F0F88140F2E48106E26D
:108DF000472900F05F8205D8452900F0368240F20D
:108E0000228244E2492900F0788240F266822EE113
:108E10005B2900F0368323D8532900F0C0820FD895
:108E20004F2900F0948205D84D2900F07A8240F253
:108E3000158181E2512900F09E8240F29282A4E2E3
:108E4000572900F0DE8205D8552900F0BA8240F299
:108E5000AF82C6E2592900F0F48240F2E28200E3D8
:108E6000632900F064830FD85F2900F03C8305D8A4
:108E70005D2900F0268340F214832BE3612900F082
:108E8000448340F2398349E3672900F0748305D8AD
:108E9000652900F05E8340F2538363E3692900F0A3
:108EA0007C83C0F07183FF2900F0808385E338B9AB
:108EB0000146142013F0C9FF00B22860204638BDD7
:108EC000012C14BF0020042038BD38B9112013F044
:108ED00031FFC0F302402860002038BD012840F077
:108EE0006E83112013F026FF2B681B0403F4E0238C
:108EF00020F4E0211943112013F048FF002038BD71
:108F000038B9112013F016FFC0F3C4402860204682
:108F100038BD012840F05583112013F00BFF2B685A
:108F2000DB0403F4780320F478011943112013F0D3
:108F30002DFF002038BD30B9112013F0FBFE80B2A8
:108F40002860204638BD012840F03D83112013F0F1
:108F5000F1FE2988000C00040143112013F016FFD4
:108F6000002038BD38B9112013F0E4FEC0F30260D0
:108F70002860204638BD012840F02783112013F0D7
:108F8000D9FE2B681B0603F0E06320F0E061194373
:108F9000112013F0FBFE002038BD38B9112013F06A
:108FA000C9FEC0F3C2602860002038BD012840F02F
:108FB0000E83112013F0BEFE2B68DB0603F0605316
:108FC00020F060511943112013F0E0FE002038BD5D
:108FD00038B9112013F0AEFEC0F38070286020462F
:108FE00038BD012840F0F582112013F0A3FE2B6854
:108FF0009B0703F0804320F080411943112013F0B8
:10900000C5FE002038BD30B9112013F093FEC00F0B
:109010002860204638BD012840F0DD82112013F081
:1090200089FE296820F0004040EAC171112013F048
:10903000ADFE002038BD38B90146122013F005FFFF
:1090400000B22860204638BD012C40F0C6822A8834
:109050000021122013F02BFF002038BD002C7FF4DC
:109060002FAF152013F066FE2860002038BD34B9FC
:109070000021132013F0E9FE2860002038BD012CE8
:1090800040F0AD822A880021132013F010FF002049
:1090900038BD00287FF414AF014613F0D6FE2860D7
:1090A000204638BD30B90146012013F0CEFE2860BD
:1090B000204638BD012840F094821288002113F028
:1090C000F6FE002038BD00287FF4FAAE0021022011
:1090D00013F0BBFE2860002038BD28B9032013F030
:1090E00029FE2860204638BD012840F07C821168A6
:1090F000032013F04BFE002038BD38B90146042090
:1091000013F0A3FE00B22860204638BD012840F0CD
:109110006C8212880021042013F0C9FE002038BDA3
:1091200038B90146052013F090FE00B228602046B1
:1091300038BD012840F05B8212880021052013F021
:10914000B6FE002038BD38B90021062013F07DFEA0
:1091500000B22860002038BD012840F04A82128801
:109160000021062013F0A3FE002038BD38B90146C7
:10917000072013F06AFE00B22860204638BD01289F
:1091800040F0398212880021072013F090FE002061
:1091900038BD30B90146082013F057FE286020463C
:1091A00038BD012840F0298212880021082013F0E0
:1091B0007EFE002038BD30B90146092013F045FE7F
:1091C0002860204638BD012840F01982128800210D
:1091D000092013F06CFE002038BD30B900210A20B0
:1091E00013F033FE2860002038BD012840F00982CA
:1091F000128800210A2013F05AFE002038BD30B931
:1092000001460B2013F021FE2860204638BD0128BE
:1092100040F0F981128800210B2013F048FE002055
:1092200038BD30B901460C2013F00FFE28602046EF
:1092300038BD012840F0E981128800210C2013F08C
:1092400036FE002038BD30B901460D2013F0FDFD7B
:109250002860204638BD012840F0D98112880021BD
:109260000D2013F024FE002038BD30B900210E205F
:1092700013F0EBFD2860002038BD012840F0C981C3
:10928000128800210E2013F012FE002038BD38B9DC
:1092900001460F2013F0D9FD00B22860204638BDEA
:1092A000012840F0B881128800210F2013F0FFFD43
:1092B000002038BD38B90146102013F0C6FD00B2B9
:1092C0002860204638BD012840F0A781128800217F
:1092D000102013F0ECFD002038BD28B9112013F048
:1092E00029FD2860204638BD012840F0988111688A
:1092F000112013F04BFD002038BD00287FF4A4AEF0
:109300000021122013F0A1FD2860002038BD0028A4
:109310007FF4D6AD0146142013F097FD2860204657
:1093200038BD00287FF4CCAD0021202013F08DFD46
:1093300000B22860002038BD00287FF4C1AD01468E
:10934000212013F082FD00B22860204638BD00289D
:109350007FF4B6AD0146222013F077FD2860204649
:1093600038BD00287FF4ACAD0146232013F06DFD1D
:109370002860204638BD00287FF4A2AD00212420BB
:1093800013F063FD2860002038BD00287FF498ADFD
:109390000146252013F059FD2860204638BD0028DD
:1093A0007FF48EAD262013F0C5FC2860204638BD22
:1093B00000287FF485AD272013F0BCFC28602046F0
:1093C00038BD28B9302013F0B5FC2860002038BD26
:1093D000012840F026811168302013F0D7FC0020CE
:1093E00038BD28B9312013F0A5FC2860204638BDCF
:1093F000012840F018811168312013F0C7FC0020CB
:1094000038BD28B9322013F095FC2860204638BDBD
:10941000012840F00A811168322013F0B7FC0020C7
:1094200038BD28B9332013F085FC2860204638BDAC
:10943000012840F0FC801168332013F0A7FC0020C5
:1094400038BD28B9342013F075FC2860002038BDE1
:10945000012840F0EE801168342013F097FC0020C2
:1094600038BD28B9352013F065FC2860204638BD8A
:10947000012840F0E0801168352013F087FC0020BF
:1094800038BD28B9362013F055FC2860204638BD79
:10949000012840F0D2801168362013F077FC0020BC
:1094A00038BD28B9372013F045FC2860204638BD68
:1094B000012840F0C4801168372013F067FC0020B9
:1094C00038BD00287FF4FCAC382013F033FC286052
:1094D000002038BD00287FF4F3AC392013F02AFCBB
:1094E0002860204638BD00287FF4EAAC3A2013F00B
:1094F00021FC2860204638BD00287FF4E1AC3B20E9
:1095000013F018FC2860204638BD00287FF4D8AC42
:109510003C2013F00FFC2860002038BD00287FF4A9
:10952000CFAC3D2013F006FC2860204638BD002853
:109530007FF4C6AC3E2013F0FDFB2860204638BD0A
:1095400000287FF4BDAC3F2013F0F4FB28602046D8
:1095500038BD00287FF4B4AC762013F0EBFB286014
:10956000002038BD00287FF4ABAC772013F0E2FB7D
:109570002860204638BD00287FF4A2AC7C2013F080
:10958000D9FB2860204638BD00287FF499AC7D20A7
:1095900013F0D0FB2860204638BD00287FF490AC43
:1095A0007E2013F0C7FB2860002038BD00287FF420
:1095B00087AC244B5B68136038BD042038BD0020A5
:1095C00038BD002038BD002038BD002038BD002047
:1095D00038BD002038BD002038BD002038BD002037
:1095E00038BD002038BD002038BD002038BD002027
:1095F00038BD002038BD002038BD002038BD002017
:1096000038BD002038BD002038BD002038BD002006
:1096100038BD002038BD002038BD002038BD0020F6
:1096200038BD002038BD002038BD002038BD0020E6
:1096300038BD002038BD002038BD002038BD0020D6
:1096400038BD00BF7014FF1F0B4619B901461846FC
:10965000FFF780BB082070470120704707B50192D3
:1096600029B9014601AA0120FFF774FB00E0082098
:1096700003B05DF804FB084613F05CBB08461146D6
:1096800013F084BB13F0E1BB13F011BC38B51B4BD6
:109690001B4DDC686068236864302860DB6898478D
:1096A000236828685B699847164B17495A690A600E
:1096B0001649C2F804121649C2F808120120002106
:1096C00051701070134A9A63134A5A63134A9A648A
:1096D000134A5A64134A5A65134A1A65134A1A669A
:1096E000134ADA65134A9A653222DA6018744FF425
:1096F0008C729A60BDE83840FFF7FABA0C55020048
:10970000E42FFF1FC82EFF1FE02FFF1F59960000F8
:10971000D18C0000499600005D960000ED8C0000A1
:10972000E18C0000A98C0000CD8C0000F18C0000C1
:10973000D58C0000318D0000014B0022DA667047A5
:10974000C82EFF1F70B5084E084D336804462A46E0
:109750000146002016F008F933682A462146012008
:10976000BDE8704016F000B9D432FF1FE82FFF1F8C
:10977000014B186816F043B9D432FF1F10B5104CD6
:1097800023681868C8B963681B68BBB90D4B1868B3
:1097900016F02CF9022015F0F3FE0B490B4B0A686A
:1097A000186850629868906222604A685968DB685D
:1097B000626051629362012010BD002010BD00BFA5
:1097C0008C00FF1FD432FF1F780AFF1F8814FF1F71
:1097D000012805D820B9034B1B681B680B60704734
:1097E00008207047780AFF1F012810B5144608D0DA
:1097F000022813D10A4B0B4ADB68506A1B681B6AAC
:1098000005E0074B074ADB68106A1B681B6A98472C
:10981000003018BF01202060002010BD042010BDC2
:109820000C5502008814FF1F022804BF0B4B93F84D
:10983000D00020B90A4BDB681B685B690AE001288D
:109840000BD1064B93F8D030012B06D1044BDB68CB
:109850001B689B69034A106918477047C82EFF1F91
:109860000C5502008814FF1F70B50020FFF7DCFFC5
:109870000A4B0B4CDD6820692B689B6898472B6866
:10988000206A9B6898472B68606A9B68984715F028
:10989000D7FE044BBDE870405B6818470C550200CA
:1098A0008814FF1FC409FF1F2DE9F843184C9DF8C9
:1098B00020609DF82450984623680F469B6800213D
:1098C00047F0800091469847236800219B684846EE
:1098D0009847236800219B684046984723680021E9
:1098E0009B6830469847236828469B680121984723
:1098F000084B1B6848EA092807F07F0746EA082654
:1099000003EB870745EA06257D60BDE8F88300BFC5
:10991000D832FF1FD432FF1F07B5D3B20193C2F371
:1099200007230093C2F30743120EFFF7BDFF03B0F6
:109930005DF804FB0A4601460020FFF7EDBF38B58D
:10994000234B01F07F04234493F81432DB0705D442
:10995000204B1B6803EB8404606838BD1E4D2B68E8
:1099600000219B68204698472B6800219B68084689
:1099700098472B6800219B68084698472B68002170
:109980009B68084698472B6801219B6800209847F0
:109990002B6800219B68204698472B6800219B6814
:1099A000084698472B68002104029B6808469847A0
:1099B0002B680021204304029B68084698472B68C7
:1099C000204304029B68012100209847204338BDB2
:1099D000E82FFF1FD432FF1FD832FF1F10B50C46EF
:1099E00001460020FFF7ABFF206010BD012838B50D
:1099F00004460D4618D80021FFF7A1FF002140F0D2
:109A000006022046FFF788FF084B53F82430002059
:109A1000187683F84C009A685A645A6C1A610122CD
:109A20009D6483F84C2038BD082038BD8C00FF1F92
:109A3000012838B504460D4611D80021FFF77FFFF5
:109A4000002140F006022046FFF766FF054B53F861
:109A5000243000201D61187683F84C0038BD0820A2
:109A600038BD00BF8C00FF1F012808D8054A52F8F6
:109A700020309A680B6813440B601946D8E7082019
:109A8000704700BF8C00FF1FA32A2DE9F041044658
:109A90000D461E4600F0C8812DD8072A00F0D98057
:109AA0000DD8032A00F0868003D8012A64D055D946
:109AB00071E0052A00F09F8040F28B80AAE0182A0E
:109AC00000F0088108D8162A00F0E88000F2F4803F
:109AD000082A00F0DC80B6E31D2A00F02D8103D8AF
:109AE0001C2A00F00B81AEE38C2A00F02C81A22A04
:109AF00000F07781A7E3AC2A00F0C88215D8A72A26
:109B000000F03F8205D8A52A00F0CA8140F2AA8160
:109B100003E2A92A00F06082C0F04182AA2A00F084
:109B20007982AB2A00F094828DE3B42A00F02C8372
:109B300008D8AE2A00F0E582C0F0C582B32A00F052
:109B4000068380E3B62A00F0A980C0F02A83B82AF1
:109B500000F04783CE2A00F0688374E320B9B04B4D
:109B600053F821301B69DFE2012801BFAC4B32689A
:109B700053F821301A6155E320B9A94B53F821302D
:109B80009B68D1E2012840F04D83A54B326853F821
:109B900021309A6046E320B9A14B53F82130DB68AD
:109BA000C2E2012840F03E839D4B326853F82130D9
:109BB000DA6037E348B99A4B53F821301A6812F447
:109BC000000318BF4FF07F43ADE2012C00F03B8350
:109BD00028E320B9924B53F821305B69A4E20128B5
:109BE00040F020838E4B53F821203368002BB8BF00
:109BF0005B42536116E320B9894B53F821305B680F
:109C000092E2012840F00E83854B326853F82130F0
:109C10005A6007E350B92021A94041F01001C9B2B0
:109C20002846FFF78CFEC0F304200AE3012840F029
:109C3000F98220248C4044F01004E4B221462846E6
:109C4000FFF77DFE33681B0203F4F85320F4F8524B
:109C5000E3E250B92021A94041F01001C9B22846E1
:109C6000FFF76DFE00F01F00EBE2012840F0DA8202
:109C700020248C4044F01004E4B221462846FFF72B
:109C80005EFE336820F01F0203F01F03C5E20028C8
:109C90009BD1634B53F821305B7E45E224B92021F0
:109CA000A94041F011011AE0012C40F0BB822021B3
:109CB000A94041F011011EE020B92021A94041F046
:109CC00012010CE0012840F0AD822021A94041F0B2
:109CD000120110E040B92021A94041F01301C9B29E
:109CE0002846FFF72CFEACE2012840F09B822021A1
:109CF000A94041F013013268C9B290E250B909019C
:109D000041F06C0101F0FC012846FFF718FEC0F39A
:109D1000804096E2012840F085820C0144F06C04FA
:109D2000E4B221462846FFF70AFE33689B0403F499
:109D3000802320F4802270E200287FF446AF394B64
:109D40001B681B68F0E150B9090141F06C0101F09A
:109D5000FC012846FFF7F3FDC0F3036071E2012820
:109D600040F060821B68102B1FD00CDC022B18D037
:109D700003DC012B1FD108231FE0042B13D0082B79
:109D800019D1052319E0402B11D003DC202B12D16F
:109D9000032312E0802B0CD0B3F5807F0BD100237E
:109DA0000BE0072309E0062307E0042305E0022374
:109DB00003E0306002E04FF0FF333360336801337B
:109DC00000F030822C0144F06C04E4B221462846B5
:109DD000FFF7B5FD33681B0603F0706320F0706277
:109DE0001BE250B9090141F06C0101F0FC01284669
:109DF000FFF7A5FDC0F3C13023E2012840F0128235
:109E00000C0144F06C04E4B221462846FFF797FDAC
:109E10003368DB0303F4C03320F4C032FDE100BF3C
:109E20008C00FF1F780AFF1F50B9090141F06C0137
:109E300001F0FC012846FFF782FDC0F3803000E20C
:109E4000012840F0EF810C0144F06C04E4B221469B
:109E50002846FFF774FD33689B0303F4804320F426
:109E60008042DAE150B9090141F06C0101F0FC01D6
:109E70002846FFF764FDC0F30030E2E1012840F01E
:109E8000D1810C0144F06C04E4B221462846FFF76E
:109E900056FD33681B0303F4805320F48052BCE169
:109EA0000F0147F06C07FFB239462846FFF747FD20
:109EB000804674B918F4804F3946284640D1FFF7E0
:109EC0003EFD18F4006FC0F3021018BF40F0080008
:109ED000B7E1012C40F0A68118F4804839462846A5
:109EE00044D1FFF72CFD3268120120F0700002F01F
:109EF0007002024339462846FFF70EFD39462846D0
:109F0000FFF71DFD336813F0080F20F4006218BF3F
:109F10004FF4006842EA080231E00F0147F06C0795
:109F2000FFB239462846FFF70AFD74B910F4804F96
:109F30003946284604D0FFF702FDC0F3021080E145
:109F4000FFF7FDFCC0F3C3107BE1012C40F06A81F8
:109F500010F480443946284608D0FFF7F0FC3368F7
:109F60001B0103F0700320F0700207E0FFF7E7FC2D
:109F70003368DB0103F4F06320F4F0621A433946DE
:109F80004DE128B9090141F06C0101F0FC0183E0C9
:109F9000012840F047810C0144F06C0488E050B97E
:109FA000090141F06D0101F0FD012846FFF7C7FCF2
:109FB000C0F3C03045E1012840F034810C0144F089
:109FC0006D04E4B221462846FFF7B9FC3368DB0391
:109FD0009BB220F4004220E150B9090141F06D012B
:109FE00001F0FD012846FFF7AAFCC0F3413028E14B
:109FF000012840F017810C0144F06D04E4B22146C1
:10A000002846FFF79CFC33685B0303F4C04320F44D
:10A01000C04202E150B9090141F06D0101F0FD01BA
:10A020002846FFF78CFCC0F303200AE1012840F02A
:10A03000F9800C0144F06D04E4B221462846FFF794
:10A040007EFC33681B0203F4706320F47062E4E06A
:10A0500050B9090141F06D0101F0FD012846FFF7FB
:10A060006EFCC0F34110ECE0012840F0DB800C01F5
:10A0700044F06D04E4B221462846FFF760FC3368E3
:10A080005B0103F0600320F06002C6E050B90901F3
:10A0900041F06D0101F0FD012846FFF750FC00F092
:10A0A0000F00CEE0012840F0BD800C0144F06D04AB
:10A0B000E4B221462846FFF742FC336820F00F0245
:10A0C00003F00F03A9E050B9090141F06D0101F05F
:10A0D000FD012846FFF733FCC0F30060B1E0012822
:10A0E00040F0A0800C0144F06D04E4B22146284603
:10A0F000FFF725FC33681B0603F0807320F08072A5
:10A100008BE098B9090141F06D0101F0FD0128468D
:10A11000FFF715FC001410F0400F00F07F0214BF91
:10A120006FF0FF030023134333607BE0012879D1F4
:10A130000C0144F06D04E4B221462846FFF7FFFB12
:10A1400033681B0403F4FE0320F4FE0265E050B9FB
:10A15000090141F06C0101F0FC012846FFF7EFFB1B
:10A16000C0F340406DE001285CD10C0144F06C0468
:10A17000E4B221462846FFF7E2FB33685B0403F4B0
:10A18000003320F4003248E000287FF41EAD0901BE
:10A1900041F06F01C9B22846FFF7D1FBC0F304407C
:10A1A0004FE020B9294B53F82130DB69BCE7012887
:10A1B00038D120248C4064B244F0110144F01404DE
:10A1C0001A68C9B22846E4B2FFF7A6FB2146284622
:10A1D000FFF7B5FB33689B0203F4806320F48062D1
:10A1E0001BE050B9090141F06C0101F0FC01284667
:10A1F000FFF7A5FBC0F3403023E0012812D10C018A
:10A2000044F06C04E4B221462846FFF798FB33681B
:10A210005B0303F4005320F400521A4321462846FE
:10A22000FFF77AFB0020BDE8F08100287FF4CDAC79
:10A23000090141F06F01C9B22846FFF780FBC0F366
:10A2400009003060EEE70420BDE8F0818C00FF1FBC
:10A2500007B50129019205D8024601AB0120FFF79D
:10A2600013FC00E0082003B05DF804FB012913464D
:10A2700002D80246002007E408207047012838B5BC
:10A2800004460D4610D80021FFF759FB002140F08D
:10A2900006022046FFF740FB044B53F8243001220E
:10A2A0001A760020DD6038BD082038BD8C00FF1F05
:10A2B0000021E3E74942E1E7E0E770B5554E564833
:10A2C000564C15F011FBF5686B6803F164022261CE
:10A2D00003F1E402626203F58272226203F5A27264
:10A2E000A26003F5B27203F59270626003F5C27268
:10A2F00003F50173A3622B68E260DB682060984776
:10A300002B68A068DB6898472B686068DB68984713
:10A310002B68E068DB6898472B682069DB68984702
:10A320002B68A06ADB683E4D984733693D4A03F1CC
:10A3300010011160A26A5A613B4B3C4A1A6002202C
:10A3400015F01EF93A4920680B683A4A5862A0682D
:10A35000986213604B68536062685A62E2689A625E
:10A36000354B3649DA6FC2F804123549C2F8081283
:10A370000024012111705470324AC3F88820324AF7
:10A38000C3F88420314AC3F88020314AC3F88C20B6
:10A39000304AC3F8A020304AC3F89C202F4AC3F8A3
:10A3A00090202F4AC3F894202E4AC3F898202E4AB2
:10A3B000C3F8B0202D4AC3F8AC202D4AC3F8BC2006
:10A3C0002C4AC3F8B8202C4AC3F8B4202B4AC3F84F
:10A3D000C8202B4AC3F8C42032225A674FF48C722B
:10A3E00002201A67274AC3F8C02083F87800FFF7D5
:10A3F0001BFA2B689847AB682046984721462046B1
:10A40000FFF79DFA214640F006022046BDE8704065
:10A41000FFF782BA0C550200E82FFF1F8814FF1FB8
:10A42000C409FF1FD832FF1FD432FF1F2C10FF1F9B
:10A43000780AFF1F8C00FF1FC82EFF1F7D970000AA
:10A44000719700007DA20000B9A20000B5A2000033
:10A45000B1A200006DA2000051A20000319A0000DC
:10A46000699A0000ED99000035990000DD9900001F
:10A4700045970000E9970000D19700002998000057
:10A48000399700006998000028B9044B1B68012225
:10A490001A76D96070470820704700BF9400FF1FEC
:10A4A000F2E74942F0E70021EEE730B9044B1B68C0
:10A4B0001961187683F84C0070470820704700BF78
:10A4C0009400FF1F014B0846DB6B18470800FF1F75
:10A4D000034B10B51B6C0C469847206010BD00BFA5
:10A4E0000800FF1F07B5034B68461B6B984703B076
:10A4F0005DF804FB0800FF1F70B50020FFF7F2FFB6
:10A500001E4B1F4CDD68206B2B689B6898472B689F
:10A51000E06A9B6898472B68E0689B6898472B68BF
:10A52000A0689B6898472B6860689B6898472B6871
:10A5300020689B6898472B68A0699B6898472B68A0
:10A54000E0699B6898472B68A06A9B6898472B68CE
:10A5500060699B6898472B68206A9B6898472B68BE
:10A56000606A9B6898472B6820699B68984715F03C
:10A5700067F8044BBDE870405B6818470C55020053
:10A58000C014FF1FC409FF1F38B9054B1B689A6828
:10A590000B6813440B60194687E70820704700BF1B
:10A5A0009400FF1F062873B505460C465CD80229A7
:10A5B00003D901285AD10F2958DC2E4E6846336B37
:10A5C00098473346052D4AD8DFE805F003063E419B
:10A5D00044478DF8004042E0082C40D8DFE804F002
:10A5E000050A11161B20252A2F00F2788DF801206C
:10A5F000327B03E032798DF80120727B8DF80220E6
:10A600002DE072798DF80120B27BF7E7B2798DF8F1
:10A610000120F27BF2E7F2798DF80120327CEDE740
:10A62000727A8DF80120B27CE8E7B27A8DF80120C9
:10A63000F27CE3E7327A8DF80120727CDEE7F27A71
:10A640008DF80120327DD9E78DF8034007E08DF8C1
:10A65000044004E08DF8054001E08DF806406846AE
:10A66000DB6A9847002002E0042000E0102002B0DE
:10A6700070BD00BF0800FF1F73B5444E0546336B25
:10A6800068460C4698473346062D7AD8DFE805F031
:10A6900076046A6D707376009DF80120F17891421E
:10A6A00008D13A499DF80200097B884202D1002076
:10A6B000206069E01979914207D134499DF8020080
:10A6C000497B884201D101235AE05979914207D14F
:10A6D0002E499DF80200897B884201D102234FE078
:10A6E0009979914207D129499DF80200C97B884296
:10A6F00001D1032344E0D979914207D123499DF840
:10A700000200097C884201D1042339E0597A914240
:10A7100007D11E499DF80200897C884201D105239A
:10A720002EE0997A914207D118499DF80200C97C20
:10A73000884201D1062323E0197A914207D11349B7
:10A740009DF80200497C884201D1072318E0DB7A9A
:10A75000934218D10D4B9DF802201B7D9A4212D1D5
:10A7600008230DE09DF803300AE09DF8043007E06F
:10A770009DF8053004E09DF8063001E09DF80030BA
:10A780002360002000E0102002B070BD0800FF1F11
:10A7900030B585B00C46019200295CD10B2814D845
:10A7A000062836D2022829D007D818B3012854D158
:10A7B0002B4B1B689A601A614BE0042822D00528B5
:10A7C0004BD1274B1B685A6043E0132806D80E284C
:10A7D00039D20C281FD00D282CD03EE08C283CD13B
:10A7E00001A90120FFF748FF1E4B04469B6B02A8FE
:10A7F00098472EE01A4B1B681A612FE0184B1B6814
:10A80000DA6026E0164B002A1B68B8BF52425A6134
:10A810001FE0063818E01546134A144BD268126838
:10A820001DB15269D86A904713E0D86A926990477F
:10A83000284613E042F210739A420ED80C4B90B2A5
:10A840009B68984705E00E381146C0B2FFF7AAFE94
:10A8500004E0204602E0082000E0042005B030BDFE
:10A860009400FF1F0800FF1F0C550200C014FF1FBB
:10A87000C409FF1F10B51446002946D1132846D835
:10A88000DFE800F00A0E12161A1E222222222222CD
:10A8900029303C3C3C3C3C3C1E4B1B681B6918E08F
:10A8A0001C4B1B689B6814E01A4B1B68DB6810E0AC
:10A8B000184B1B681B680CE0164B1B685B6908E0B3
:10A8C000144B1B685B6804E0082820D1114B1B68FF
:10A8D0005B7E236017E0104B104ADB68D06A1B6870
:10A8E0001B6A05E00C4B0D4ADB68106B1B681B6A8A
:10A8F0009847003018BF0120206004E00E38114650
:10A90000C0B2FFF7B9FE002010BD082010BD042022
:10A9100010BD00BF9400FF1F0C550200C014FF1FA4
:10A920005F4B2DE9F041DF685E4C786800F5E2731B
:10A93000236300F5D273E36200F52173E36000F551
:10A940002973A36000F51973636000F50173236038
:10A9500000F55973A36100F55173E36100F16403DD
:10A96000A36200F5A273636100F56973236200F5C9
:10A97000717363623B6800F59270DB6820619847F1
:10A980003B686069DB6898473B68206BDB689847E9
:10A990003B68E06ADB6898473B68206A1B69984718
:10A9A0003B68606A1B6998473F4BE1685A6C1160CD
:10A9B0005A6CA16851605A6C616891605A6C216848
:10A9C000D1605A6CA16911615A6CE16951615A6C8C
:10A9D000A16A916100251E46726C3B685059DB6884
:10A9E0009847726C3B6850599B69043598471C2DF9
:10A9F000F2D12E4DDFF8F480EB6F00221A700120A7
:10AA000014F0BEFD2A4B22695B68C8F800305A6218
:10AA100062699A62274BC5F88830274BC5F88430A5
:10AA2000264BC5F88030264BC5F88C30254BC5F831
:10AA3000A030254BC5F89C30244BC5F89030244BF2
:10AA4000C5F89430234BC5F8B030234BC5F8AC3073
:10AA5000224BC5F8C830012385F878300220204BFE
:10AA6000C5F8C030FFF73EFDD8F800301B6813B1C1
:10AA70001C4B9B780BB1B36A98473B68206BDB6833
:10AA80009847206B184C042343753B681B68984714
:10AA900023689847A3680020BDE8F041184700BF2D
:10AAA0000C550200C014FF1F0800FF1FC82EFF1F17
:10AAB000780AFF1F89A40000A1A40000A3A400003D
:10AAC000A7A4000075A8000091A70000ABA4000097
:10AAD00089A50000C5A40000D1A40000E5A40000E1
:10AAE000F9A40000400AFF1FC409FF1F9400FF1FC4
:10AAF00028B9044B1B6801221A76D96070470820D8
:10AB0000704700BF9800FF1FF2E74942F0E70021BD
:10AB1000EEE730B9044B1B681961187683F84C00D6
:10AB200070470820704700BF9800FF1F10B5042829
:10AB300004D8DFE800F0052321333F00042010BDD6
:10AB4000146844F620639C426AD8364B364ADB6868
:10AB5000106A1B6842F210718C42DB6994BF0021BD
:10AB60000121984742F21170B4FBF0F300FB13404F
:10AB70002E4B80B29B689847002010BD294B14686B
:10AB8000DB6858681B6824B1DB69002100F5F270AE
:10AB90000EE09B6800F5F2709847EDE7214B1168D5
:10ABA000DB68214A1B681069DB69003118BF01218D
:10ABB0009847E1E714681E4B0020032C20D8DFE8FB
:10ABC00004F002070E1553F8213083F84C00D3E748
:10ABD000184A53F82130126892685A64CCE7154A33
:10ABE00053F82130126892689A64C5E753F821300F
:10ABF000012283F84C205A6C1A610020187610BD8F
:10AC000053F821300B4983F84C000968896859646E
:10AC100012689A645A6C1A61012283F84C20ABE7DF
:10AC2000102010BD0C5502000015FF1FC409FF1FA6
:10AC30009800FF1F780AFF1F1B4B70B5DD681B4C87
:10AC40002B68A0685B6998472B6820689B689847C9
:10AC50002B6860689B6898472B68206A9B689847B8
:10AC60002B68606A9B6898472B68E0689B689847E8
:10AC70002B6820699B6898472B6860699B68984798
:10AC80002B68A0699B6898472B68E0699B68984788
:10AC90002B68A0689B68984714F0D2FC044BBDE871
:10ACA00070405B68184700BF0C5502000015FF1F7D
:10ACB000C409FF1F014B186814F0EEBE6035FF1F7A
:10ACC0000C4B1A68126810B51C4612B10A4B9878E2
:10ACD00078B10A4B186814F0D6FE012014F050FC2D
:10ACE000074B084A1B6811685268236059629A62D0
:10ACF000012010BD9800FF1F400AFF1F6035FF1F95
:10AD0000780AFF1F0015FF1F38B9054B1B689A68AA
:10AD10000B6813440B601946FBE60820704700BF20
:10AD20009800FF1F78B9094B094A1B68126818760A
:10AD300083F84C0092685A645A6C1A610122996433
:10AD400083F84C2070470820704700BF9800FF1F11
:10AD5000780AFF1F20B9034B1B681B680B60704704
:10AD600008207047780AFF1F022804BF0B4B93F896
:10AD7000D00020B90A4BDB681B685B690AE0012838
:10AD80000BD1064B93F8D030012B06D1044BDB6876
:10AD90001B689B69034A906818477047C82EFF1FBD
:10ADA0000C5502000015FF1F2DE9F0471C4D9DF8C2
:10ADB00020709DF82460994655F820300446884656
:10ADC0009B68002148F080009246984755F824304F
:10ADD00000219B685046984755F8243000219B6815
:10ADE0004846984755F8243000219B6838469847D4
:10ADF00055F8243030469B6801219847094B53F899
:10AE0000243049EA0A2908F07F0847EA092703EBBA
:10AE1000880846EA0726C8F80460BDE8F08700BF46
:10AE20006435FF1F6035FF1F07B5D3B20193C2F32E
:10AE300007230093C2F30743120EFFF7B5FF03B0D9
:10AE40005DF804FB0A4601460020FFF7EDBF70B530
:10AE50002B4A4FF4217301F07F0403FB00232344AA
:10AE6000054693F80432DB0706D4264B53F820300E
:10AE700003EB8404606870BD234E56F82030002137
:10AE80009B682046984756F8253000219B68084665
:10AE9000984756F8253000219B680846984756F891
:10AEA000253000219B680846984756F82530012137
:10AEB0009B680020984756F8253000219B68204663
:10AEC000984756F8253000219B680846984756F861
:10AED0002530002104029B680846984756F8253023
:10AEE0000021204304029B680846984756F8253005
:10AEF000204304029B68012100209847204370BD35
:10AF0000DC32FF1F6035FF1F6435FF1F38B5104B63
:10AF1000104C1B68104A0146002014F0ADFD236858
:10AF200093F8302002F0FF0582B993F840306BB1FE
:10AF30006F212846FFF78BFF6F212846FFF787FF19
:10AF4000C30142BF2368012283F8302038BD00BF0F
:10AF50006035FF1F780AFF1FDC32FF1F10B50C465B
:10AF600001460020FFF773FF206010BDA62AF8B548
:10AF700004460D461E4600F06A8251D8172A00F09A
:10AF8000308124D8042A00F0CE800CD8012A00F0A9
:10AF9000A280C0F09280022A00F0AD80032A00F067
:10AFA000B98000F064BC072A00F0F48007D8052AB5
:10AFB00000F0CB80062A00F0D78000F058BC082AA9
:10AFC00000F0FF80152A00F0038100F050BC1D2A1C
:10AFD00000F0658110D81A2A00F0248104D8182ABC
:10AFE00000F0148100F043BC1B2A00F02C811C2AC5
:10AFF00000F03F8100F03BBCA32A00F0B78107D8E6
:10B000008C2A00F05381A22A00F09A8100F02FBC14
:10B01000A42A00F0C781A52A00F0DA8100F027BC3D
:10B02000B52A00F0268323D8AB2A00F0A1820CD8E1
:10B03000A82A00F05C82C0F04A82A92A00F06C8243
:10B04000AA2A00F07F8200F012BCAE2A00F0D18262
:10B0500007D8AC2A00F0A282AD2A00F0B48200F03A
:10B0600006BCB32A00F0E582B42A00F0F882FEE3C1
:10B07000BB2A00F06E830ED8B82A00F0228303D8D2
:10B08000B62A00F00B83F2E3B92A00F02A83BA2A29
:10B0900000F03783EBE3C02A00F0AB8306D8BC2A6C
:10B0A00000F07D83BF2A00F08C83E0E3CC2A00F01F
:10B0B000B883CE2A00F0D083D9E320B9AF4B53F840
:10B0C00021301B69DAE2012840F0C483AB4B3268BF
:10B0D00053F821300DE020B9A84B53F821309B687C
:10B0E000CCE2012840F0B683A44B326853F82130FB
:10B0F0009A601A61AEE320B9A04B53F82130DB68A7
:10B10000BCE2012840F0A6839C4B326853F8213002
:10B11000DA609FE318B9994B53F82130C4E0012C51
:10B1200000F0A58396E320B9944B53F821305B6976
:10B13000A4E2012840F08E83904B53F8212033681D
:10B14000002BB8BF5B42536184E320B98B4B53F8AB
:10B1500021305B6892E2012840F07C83874B3268A3
:10B1600053F821305A6075E330B910212846FFF7B3
:10B170006EFEC0F3042078E3012840F06B831021B9
:10B180002846FFF764FE33681B0203F4F85320F4EB
:10B19000F85213E030B910212846FFF758FE00F0AE
:10B1A0001F0062E3012840F0558310212846FFF775
:10B1B0004EFE336820F01F0203F01F031A431021D4
:10B1C00045E30028ABD16D4B53F821305B7E55E24F
:10B1D000002800F04C83012840F03C831A681121BC
:10B1E00035E308B915218EE2012840F033831B684E
:10B1F000002B08BF01234FF0807494FBF3F4604BE5
:10B200009C42A8BF1C46224615219DE220B933214D
:10B210002846FFF71CFE28E3012840F01B831A682C
:10B22000332114E308B96C21E5E2012840F01283D0
:10B230006C212846FFF70BFE33689B0403F4802340
:10B2400020F4802240E130B96C212846FFF7FFFD51
:10B25000C0F3C04009E3012840F0FC826C2128467D
:10B26000FFF7F5FD3368DB0403F4002320F400222C
:10B270002AE130B901462846FFF7E9FDC0F3400056
:10B28000F3E2012840F0E68200212846FFF7DFFDC7
:10B2900033685B0003F0020320F002027CE2002826
:10B2A0007FF43DAF374B1B681B68E7E150B96C2159
:10B2B0002846FFF7CCFD4FF48073C0F3036043FAD8
:10B2C00000F0D2E2012840F0C5821B68102B1FD08D
:10B2D0000CDC022B18D003DC012B1FD108231FE04C
:10B2E000042B13D0082B19D1052319E0402B11D0C2
:10B2F00003DC202B12D1032312E0802B0CD0B3F5FA
:10B30000807F0BD100230BE0072309E0062307E031
:10B31000042305E0022303E0306002E04FF0FF3336
:10B3200033603368013300F0A4826C212846FFF7B4
:10B330008EFD33681B0603F0706320F07062C3E07B
:10B3400030B96C212846FFF782FDC0F3C1308CE292
:10B35000012840F07F826C212846FFF778FD336892
:10B36000DB0303F4C03320F4C032ADE060B96C21DC
:10B370002846FFF76CFDC0F3803076E29800FF1F8F
:10B38000FFFF0F00780AFF1F012840F063826C2145
:10B390002846FFF75CFD33689B0303F4804320F4E9
:10B3A000804291E030B96C212846FFF750FDC0F390
:10B3B00000305AE2012840F04D826C212846FFF708
:10B3C00046FD33681B0303F4805320F480527BE076
:10B3D000D0B96C212846FFF73AFD10F4804F4FF0AA
:10B3E0006C01284604D0FFF732FDC0F3C3103CE2E5
:10B3F000FFF72DFD6C2107462846FFF728FD17F4BF
:10B40000006FC0F302103DE0012840F023826C2160
:10B410002846FFF71CFD10F480444FF06C012846CD
:10B420004AD1FFF714FD6C212846FFF710FD336861
:10B4300013F0080F20F4006218BF4FF400646C2171
:10B4400028462243FFF7F0FC6C2128462BE0E8B9A0
:10B450006C212846FFF7FBFC10F480474FF06C018D
:10B46000284604D0FFF7F3FCC0F30210FDE1FFF71C
:10B47000EEFC6C2104462846FFF7E9FC14F4006F4B
:10B48000C0F3C31018BF40F00800EEE1012840F0FF
:10B49000E1816C212846FFF7DAFC10F480444FF07C
:10B4A0006C01284608D0FFF7D2FC33681B0103F07B
:10B4B000700320F0700207E0FFF7C9FC3368DB017E
:10B4C00003F4F06320F4F0621A436C21BFE108B981
:10B4D0006C2165E0012840F0BD816C212846FFF712
:10B4E000B6FC336820F00F0203F00F03ECE730B92D
:10B4F0006D212846FFF7ABFCC0F3C030B5E1012851
:10B5000040F0A8816D212846FFF7A1FC3368DB03DA
:10B510009BB220F4004289E030B96D212846FFF744
:10B5200096FCC0F34130A0E1012840F093816D21E9
:10B530002846FFF78CFC33685B0303F4C04320F418
:10B54000C04273E030B96D212846FFF780FCC0F39C
:10B5500003208AE1012840F07D816D212846FFF714
:10B5600076FC33681B0203F4706320F470625DE0C4
:10B5700030B96D212846FFF76AFCC0F3411074E131
:10B58000012840F067816D212846FFF760FC336891
:10B590005B0103F0600320F0600247E030B96D21E9
:10B5A0002846FFF754FC00F00F005EE1012840F050
:10B5B00051816D212846FFF74AFC336820F00F02C5
:10B5C00003F00F0332E030B96D212846FFF73FFC4E
:10B5D000C0F3006049E1012840F03C816D2128461C
:10B5E000FFF735FC33681B0603F0807320F0807290
:10B5F0001CE070B96D212846FFF729FC001410F0FB
:10B60000400F00F07F0214BF6FF07F03002313434D
:10B6100034E0012840F01E816D212846FFF717FC19
:10B6200033681B0403F4FE0320F4FE021A436D2169
:10B630000DE130B96C212846FFF709FCC0F340400A
:10B6400013E1012840F006816C212846FFF7FFFB3B
:10B6500033685B0403F4003320F4003234E700283D
:10B660007FF45DAD6F212846FFF7F1FBC0F3044086
:10B67000FBE028B9804B53F82130DB693360E9E007
:10B68000012840F0E7807C4B326853F82130DA61C2
:10B690007A4B1B68002483F83040DBE008B91421A2
:10B6A00031E0012840F0D6801A68754C32B14FF075
:10B6B000807393FBF2F39C42A8BF1C4622461421E0
:10B6C00042E030B96C212846FFF7C1FBC0F340309F
:10B6D000CBE0012840F0BE801A68520302F4005209
:10B6E000F3E630B96C212846FFF7B1FBC0F30350F5
:10B6F000BBE0012840F0AE801A68120502F4700227
:10B70000E3E680B913212846FFF7A1FB4FF08073D1
:10B71000002808BF012093FBF0F0594B9842D4BF9A
:10B720003060336096E0012840F094801B68002B65
:10B7300008BF01234FF0807494FBF3F4504B9C42FC
:10B74000A8BF1C46224613212846FFF76DFB346034
:10B7500080E030B970212846FFF779FBC0F307205D
:10B7600083E0012876D170212846FFF770FB32680C
:10B77000120220F47F4092B2024370212846FFF764
:10B7800053FB00212846FFF762FB3368002B20F0B3
:10B790000402CCBF042300231A43002157E028B938
:10B7A00070212846FFF753FBC0B25EE0012851D15B
:10B7B00070212846FFF74BFB327820F0FF00024350
:10B7C00044E030B970212846FFF741FBC0F3014047
:10B7D0004BE001283ED11B68032B4AD87021284634
:10B7E000FFF735FB33681B0403F4403320F4403289
:10B7F0002BE030B970212846FFF729FBC0F38040C9
:10B8000033E0012826D11B68012B32D8702128464D
:10B81000FFF71DFB33689B0403F4802320F4802290
:10B8200013E030B970212846FFF711FBC0F3015037
:10B830001BE001280ED170212846FFF708FB336872
:10B840001B0503F4401320F440121A4370212846CC
:10B85000FFF7EAFA0020F8BD00287FF460AC6F2102
:10B860002846FFF7F4FAC0F309003060F2E704203D
:10B87000F8BD1020F8BD00BF9800FF1F780AFF1F19
:10B88000FFFF0F0007B5019229B9024601AB012065
:10B89000FFF76CFB00E0082003B05DF804FB10B478
:10B8A00013460446084619B9224610BCFFF75EBB92
:10B8B000082010BC70472DE9F041654D6548664C85
:10B8C00014F0A6F8EE68736803F16402A26003F551
:10B8D0009272226003F5A272626003F5D272226254
:10B8E00003F5E272626203F55172E26003F5597288
:10B8F00003F56970226103F5617203F57173E36109
:10B90000336862611B69A06198473368E0691B690D
:10B910009847336860691B69984733682068DB681B
:10B92000984733686068DB6898473368A068DB68CD
:10B93000984733682069DB6898473368E068DB68BC
:10B9400098473368606ADB6898473368206ADB6829
:10B9500098473368606A9B6998473368206A9B6997
:10B960009847336860699B6998473368E0689B69CA
:10B9700098472A69394B3A4D02F1100119607368F2
:10B9800003F501735361374BEA6F1A60012013F01E
:10B99000F7FD354B354A1B68136022685A626268AE
:10B9A0009A62EB6F324AC3F80422324AC3F8082283
:10B9B000002701221A705F702F4BC5F888302F4B7B
:10B9C000C5F884302E4BC5F880302E4BC5F88C302E
:10B9D0002D4BC5F8A0302D4BC5F89C302C4BC5F82D
:10B9E00090302C4BC5F894302B4BC5F898302B4B2E
:10B9F000C5F8B0302A4BC5F8AC302A4BC5F8BC307E
:10BA0000294BC5F8B830294BC5F8B430284BC5F8D8
:10BA1000C83032236B674FF4F0732B670220254B3D
:10BA200085F87820C5F8C030FFF79EF93368606A62
:10BA3000DB689847606A204C0423437533681B68B1
:10BA4000984723689847A3683846BDE8F0411847EF
:10BA50000C550200DC32FF1F0015FF1F6435FF1F6D
:10BA6000C82EFF1F6035FF1F780AFF1F9800FF1FB9
:10BA7000C1AC0000B5AC0000F1AA000009AB0000A9
:10BA80000BAB00000FAB00009FB8000085B80000B2
:10BA900013AB000009AD000025AD000045AE00006D
:10BAA0005DAF00000DAF00002DAB000055AD0000F4
:10BAB00069AD000039AC0000C409FF1F10B50B4C84
:10BAC00001440023884204D010F8012B5340E35C6A
:10BAD000F8E70822002003F0010101EB4000013AE1
:10BAE00000F0FF004FEA5303F5D110BD00530200F0
:10BAF00028B9044B1B6801221A76D96070470820C8
:10BB0000704700BF9C00FF1FF2E74942F0E70021A9
:10BB1000EEE720B9034B1B681961187670470820BF
:10BB2000704700BF9C00FF1FF7B505238DF800305C
:10BB300060F07F038DF802300B168DF803300B1484
:10BB40008DF804308DF806100B1206460D460024C1
:10BB5000072168460E4F8DF805308DF80140FFF73C
:10BB6000ADFF3B688DF807009B6998473B681DF85F
:10BB700004009B6801349847082CF7D1054B1B68DB
:10BB800026F0800603EB8606756003B0F0BD00BFAB
:10BB90006C35FF1F6835FF1F014B0022DA667047C6
:10BBA000C82EFF1F00207047F0B5314B00F07F0614
:10BBB000334485B093F80C32DB070D4605D42D4B8A
:10BBC0001B6803EB860673684EE0052303218DF89E
:10BBD0000430294C8DF80660002301A88DF805304B
:10BBE000FFF76CFF23688DF807009B69984723686F
:10BBF00004211B690DEB0100984710F015FC074666
:10BC00002368DB699847072805D8384610F01CFCE4
:10BC10000A28F5D929E0184B1B6808215B690DEB50
:10BC200001009847072102A8FFF748FF9DF80F4041
:10BC300084421AD19DF80830052B16D19DF80930A1
:10BC4000FF2B12D19DF80A30B3420ED19DF80C3073
:10BC50009DF80B201B0443EA02639DF80E2013435A
:10BC60009DF80D2043EA02232B6005B0F0BD00BF14
:10BC70007035FF1F6835FF1F6C35FF1F034B044AEB
:10BC80001B680146002013F04BBF00BF6835FF1F43
:10BC90007035FF1F014B186813F05ABF6835FF1F3E
:10BCA000014B186813F04BBF6835FF1F38B9054BBF
:10BCB0001B689A680B6813440B60194629E7082033
:10BCC000704700BF9C00FF1F022804BF0B4B93F876
:10BCD000D00020B90A4BDB681B685B690AE00128C9
:10BCE0000BD1064B93F8D030012B06D1044BDB6807
:10BCF0001B689B69034A106818477047C82EFF1FCE
:10BD00000C5502003415FF1F38B50020FFF7DCFF8B
:10BD1000114B124CDD6820682B689B6898472B6894
:10BD200060689B6898472B68A0689B6898472B6859
:10BD3000E0689B6898472B6820699B6898472B6848
:10BD400060699B6898472B68A0699B689847BDE825
:10BD5000384013F075BC00BF0C5502003415FF1FAE
:10BD600001BB052820D8DFE800F003070B0F1317ED
:10BD70000E4B1B681B6912E00C4B1B689B680EE0A6
:10BD80000A4B1B68DB680AE0084B1B681B6806E06F
:10BD9000064B1B685B6902E0044B1B685B68136021
:10BDA0000020704708207047042070479C00FF1F48
:10BDB000F1B905281ED8DFE800F003060B1D1017A7
:10BDC0000D4B1B6802E00C4B1B689A601A6102E085
:10BDD000094B1B68DA6000207047074B002A1B687C
:10BDE000B8BF52425A61F6E7034B1B685A60F2E74C
:10BDF00008207047042070479C00FF1F94E6D3E69C
:10BE000070B5484E4848494C13F050FEF5686B68D1
:10BE100003F59272626003F5A272A26003F1C4029C
:10BE2000E26003F1E40203F16400226103F18402A1
:10BE3000A433A3612B686261DB68206098472B689C
:10BE40006068DB6898472B68A068DB6898472B68B8
:10BE5000E068DB6898472B682069DB6898472B68A7
:10BE600060691B6998472B68A0691B699847F56A48
:10BE70002B6898472E4B2F491D602F4BDA6F0A60B5
:10BE80002E49C2F804122E49C2F8081201250021D9
:10BE9000157051702B4AC3F888202B4AC3F88420B0
:10BEA0002A4AC3F880202A4AC3F88C20294AC3F8BA
:10BEB000A020294AC3F89C20284AC3F89020284A89
:10BEC000C3F89420274AC3F8B020274AC3F8AC200F
:10BED000264AC3F8B820264AC3F8C820254AC3F822
:10BEE000C42032225A674FF4C3721A67224AC3F839
:10BEF000C0202846214A83F87850C3F8BC2013F0AC
:10BF00003FFB1F4B1F4A1B68136062685A62A2689E
:10BF10009A624FF448425A6128465A60BDE8704020
:10BF2000D2E600BF0C5502007035FF1F3415FF1F0D
:10BF30006C35FF1F6835FF1FC82EFF1FA1BC000016
:10BF400095BC0000F1BA000009BB00000BBB00006B
:10BF50000FBB000061BD0000B1BD000013BB0000BD
:10BF6000ADBC000029BB0000A9BB0000A5BB0000C0
:10BF7000C9BC000099BB000009BD00007DBC0000E9
:10BF8000780AFF1F9C00FF1F10B50B4C01440023D3
:10BF9000884204D010F8012B5340E35CF8E70822F4
:10BFA000002003F0010101EB4000013A00F0FF0026
:10BFB0004FEA5303F5D110BD0054020028B9044BD9
:10BFC0001B6801221A76D96070470820704700BFAD
:10BFD000A000FF1FF2E74942F0E70021EEE720B999
:10BFE000034B1B681961187670470820704700BF23
:10BFF000A000FF1FF7B505238DF8003060F07F0328
:10C000008DF802300B168DF803300B148DF80430C8
:10C010008DF806100B1206460D46002407216846CF
:10C020000E4F8DF805308DF80140FFF7ADFF3B68EE
:10C030008DF807009B6998473B681DF804009B68D2
:10C0400001349847082CF7D1054B1B6826F0800671
:10C0500003EB8606756003B0F0BD00BF8C3AFF1F8E
:10C06000903AFF1F014B0022DA667047C82EFF1F6F
:10C0700000207047F0B5314B00F07F06334485B0A7
:10C0800093F80C32DB070D4605D42D4B1B6803EBF0
:10C09000860673684EE0052303218DF80430294C91
:10C0A0008DF80660002301A88DF80530FFF76CFFBE
:10C0B00023688DF807009B699847236804211B6952
:10C0C0000DEB0100984710F0AFF907462368DB69D4
:10C0D0009847072805D8384610F0B6F91428F5D93E
:10C0E00029E0184B1B6808215B690DEB010098479C
:10C0F000072102A8FFF748FF9DF80F4084421AD19C
:10C100009DF80830052B16D19DF80930FF2B12D170
:10C110009DF80A30B3420ED19DF80C309DF80B20EB
:10C120001B0443EA02639DF80E2013439DF80D2083
:10C1300043EA02232B6005B0F0BD00BFFC37FF1FB0
:10C14000903AFF1F8C3AFF1F034B044A1B680146BD
:10C15000002013F043BD00BF903AFF1FFC37FF1FC4
:10C16000014B186813F052BD903AFF1F014B18683D
:10C1700013F043BD903AFF1F38B9054B1B689A680E
:10C180000B6813440B60194629E70820704700BF6D
:10C19000A000FF1F022804BF0B4B93F8D00020B96A
:10C1A0000A4BDB681B685B690AE001280BD1064B70
:10C1B00093F8D030012B06D1044BDB681B689B69D8
:10C1C000034A106818477047C82EFF1F0C5502001D
:10C1D0005C15FF1F70B5144E144C0020FFF7DAFFFA
:10C1E000F56820682B689B6898472B6860689B6897
:10C1F00098472B68A0689B6898472B68E0689B6805
:10C2000098472B6820699B6898472B6860699B68F2
:10C2100098472B68A0699B689847F36A5B689847C2
:10C22000BDE8704013F00CBA0C5502005C15FF1FFE
:10C2300001BB052820D8DFE800F003070B0F131718
:10C240000E4B1B681B6912E00C4B1B689B680EE0D1
:10C250000A4B1B68DB680AE0084B1B681B6806E09A
:10C26000064B1B685B6902E0044B1B685B6813604C
:10C27000002070470820704704207047A000FF1F6F
:10C28000F1B905281ED8DFE800F003070B1D1017D1
:10C290000D4B1B681A6106E00B4B1B689A6002E0AD
:10C2A000094B1B68DA6000207047074B002A1B68A7
:10C2B000B8BF52425A61F6E7034B1B685A60F2E777
:10C2C0000820704704207047A000FF1F92E6D1E6C7
:10C2D00070B5484E4848494C13F044FCF5686B680B
:10C2E00003F59272626003F5A272A26003F1C402C8
:10C2F000E26003F1E40203F16400226103F18402CD
:10C30000A433A3612B686261DB68206098472B68C7
:10C310006068DB6898472B68A068DB6898472B68E3
:10C32000E068DB6898472B682069DB6898472B68D2
:10C3300060691B6998472B68A0691B699847F56A73
:10C340002B6898472E4B2F491D602F4BDA6F0A60E0
:10C350002E49C2F804122E49C2F808120125002104
:10C36000157051702B4AC3F888202B4AC3F88420DB
:10C370002A4AC3F880202A4AC3F88C20294AC3F8E5
:10C38000A020294AC3F89C20284AC3F89020284AB4
:10C39000C3F89420274AC3F8B020274AC3F8AC203A
:10C3A000264AC3F8B820264AC3F8C820254AC3F84D
:10C3B000C42032225A674FF4C3721A67224AC3F864
:10C3C000C0202846214A83F87850C3F8BC2013F0D7
:10C3D000D7F81F4B1F4A1B68136062685A62A26835
:10C3E0009A624FF448425A6128465A60BDE870404C
:10C3F000D0E600BF0C550200FC37FF1F5C15FF1F85
:10C400008C3AFF1F903AFF1FC82EFF1F6DC100001E
:10C4100061C10000BDBF0000D5BF0000D7BF000054
:10C42000DBBF000031C2000081C20000DFBF00009E
:10C4300079C10000F5BF000075C0000071C00000A8
:10C4400095C1000065C00000D5C1000049C10000D1
:10C45000780AFF1FA000FF1F48B101280ED1136802
:10C46000074AB3FA83F35B0913600020704713682F
:10C47000044AB3FA83F35B09937270470420704750
:10C48000A400FF1F943AFF1F20B9034B5B6819619A
:10C490001876704708207047A400FF1F10B50D4B99
:10C4A0000D4C1B6822460146002013F0DAFB237A6C
:10C4B0000A4A1BB1D36E43F0010302E0D36E23F0AE
:10C4C0000103617A11B143F0020301E023F002039A
:10C4D000D36610BDD83AFF1F943AFF1FC82EFF1F26
:10C4E000014B186813F031BCD83AFF1F40B9054B17
:10C4F00058721872044B5B6801221A76D960704733
:10C5000008207047943AFF1FA400FF1FEEE749423E
:10C51000ECE70021EAE738B9044B5B689A680B68DE
:10C5200013440B601946AFE708207047A400FF1FB3
:10C5300020B9034B1B681B680B60704708207047CD
:10C54000780AFF1F022804BF0B4B93F8D00020B9D4
:10C550000A4BDB681B685B690AE001280BD1064BBC
:10C5600093F8D030012B06D1044BDB681B689B6924
:10C57000034AD06818477047C82EFF1F0C550200A9
:10C580008415FF1F38B50020FFF7DCFF0F4B104C60
:10C59000DD68E0682B685B6998472B6820689B68BA
:10C5A00098472B68A0689B6898472B68E0689B6851
:10C5B00098472B6820699B6898472B6860689B6840
:10C5C0009847BDE8384013F03BB800BF0C55020057
:10C5D0008415FF1F38B50A4D6B681C6874B9094B88
:10C5E0000948196813F094FB6B68022083F8304007
:10C5F00001242C60FFF7A6FF204638BD002038BD7F
:10C60000A400FF1FD83AFF1F943AFF1F2DE9F843FB
:10C61000830C04460ED0C0F34243062B0AD1294BAB
:10C620005A7A20F01F040AB11B7800E0DB7A03F08D
:10C630001F031C43244F254E254D3B68D6F8008030
:10C6400095F818909B680021C4F3074098472A7E0C
:10C65000336808EB890803EB8203C8F804005A68C2
:10C6600012025A603B6800219B68C4F30720984778
:10C6700033682A7E03EB82020121536818430002CB
:10C680003B6850609B68E0B298473268297E02EBB5
:10C6900081014B6818430011A30C4860106107D05A
:10C6A000C4F34243072B09D1C4F30111297605E0F5
:10C6B000082302EB83035C60BDE8F88343F00803C2
:10C6C000F7E700BF943AFF1FD43AFF1FD83AFF1F85
:10C6D0008415FF1FC2F31300830C0B4A05D04314CB
:10C6E000062B04BF00F01F03D372084B01F0770143
:10C6F0001B6841F0080103EB81014860937A0BB994
:10C70000FFF784BF704700BF943AFF1FD83AFF1F5E
:10C710000A4601460020FFF7DDBF10B5074B9B7AA4
:10C7200001F07F0423B90B0702D4204600F00AF879
:10C73000034B186800EB8400406810BD943AFF1F5B
:10C74000D83AFF1F38B50F2104460020FFF7E5FF58
:10C750000323B4FBF3F303EB4303E41A240105467C
:10C7600004F0300420F030002043FFF74FFF28464C
:10C77000BDE83840FFF74ABF10B50C46014600201F
:10C78000FFF7CBFF206010BDA82A38B504461D4630
:10C7900000F0738242D81D2A00F029811CD8042A97
:10C7A00000F0CA800BD8012A00F08F807AD3022AC9
:10C7B00000F09E80032A00F0AF8000F06CBC062AD7
:10C7C00000F0E380C0F0CE80072A00F0F980082A4C
:10C7D00000F0048100F05FBCA32A00F0BD8110D8F6
:10C7E000A02A00F05C8104D88C2A00F0098100F0B6
:10C7F00052BCA12A00F07081A22A00F08B8100F0C7
:10C800004ABCA52A00F0E281C0F0C381A62A00F04C
:10C81000FA81A72A00F0158200F03DBCB22A00F090
:10C8200047831DD8AD2A00F0AB820CD8AA2A00F0AD
:10C830005D82C0F03E82AB2A00F07582AC2A00F027
:10C84000908200F028BCAF2A00F0DB82C0F0B582F5
:10C85000B02A00F0F282B12A00F00D8300F01BBC78
:10C86000B72A00F093830CD8B42A00F05B83C0F0A1
:10C870003C83B52A00F06183B62A00F0748300F08F
:10C880000ABCCE2A50D006D8B82A00F09B83B92A19
:10C8900000F0B683FFE3D02A00F0E683D62A00F04A
:10C8A000EE83F8E330B9AA4B03EB81014B681B69B7
:10C8B0002B6038BD012840F0F083A54B2A6803EBBC
:10C8C000810100204B681A6138BD30B9A04B03EBE1
:10C8D00081014B689B682B6038BD012840F0DF83E5
:10C8E0009B4B2A6803EB810100204B689A6038BD9E
:10C8F00038B9974B03EB810100204B68DB682B6054
:10C9000038BD012840F0CD83914B2A6803EB8101AB
:10C9100000204B68DA6038BD48B98D4B03EB8101CC
:10C920004B681B682B6038BD002800F08683012C03
:10C9300014BF0020042038BD30B9854B03EB8101C2
:10C940004B685B692B6038BD012840F0AC83804B9D
:10C9500003EB81012B684A68002BB8BF5B4253612F
:10C96000002038BD30B97A4B03EB81014B685B681E
:10C970002B6038BD012840F09883754B2A6803EB83
:10C98000810100204B685A6038BD18B9714BDB7AC1
:10C990002B6038BD012840F08A831A686D4B0E2148
:10C9A0000020DA72FFF7B9FE2B6820F01F0203F0B7
:10C9B0001F031A430E210020FFF78CFE002038BD14
:10C9C00020B9644B1B782B60002038BD012840F053
:10C9D00070831A685F4B1A70002038BD0028A6D1FA
:10C9E0005B4B03EB81014B685B7E2B6038BD0028FD
:10C9F0009DD1574B03EB81014B681B682B6038BD01
:10CA000050B908210020FFF788FE00F00F00C0F1A8
:10CA100008002860002038BD012840F04C831B68C6
:10CA2000102B1FD00CDC022B18D003DC012B1FD1E4
:10CA300008231FE0042B13D0082B19D1052319E07C
:10CA4000402B11D003DC202B12D1032312E0802BCA
:10CA50000CD0B3F5807F0BD100230BE0072309E056
:10CA6000062307E0042305E0022303E0286002E038
:10CA70004FF0FF332B602B68013300F01E83082139
:10CA80000020FFF74AFE2B6820F00F0203F00F038F
:10CA90001A4308210020FFF71DFE002038BD38B9D9
:10CAA0000821FFF73AFEC0F340202860204638BD39
:10CAB000012840F0048308210020FFF72EFE2B6898
:10CAC0005B0203F4007320F400721A430821002073
:10CAD000FFF700FE002038BD40B908210020FFF715
:10CAE0001CFEC0F300202860002038BD012840F063
:10CAF000E88208210020FFF710FE2B681B0203F4D8
:10CB0000807320F480721A4308210020FFF7E2FDB1
:10CB1000002038BD38B90C21FFF7FFFDC0F3C1304C
:10CB20002860204638BD012840F0CD820C2100202D
:10CB3000FFF7F3FD2B68DB0303F4C03320F4C032AE
:10CB40001A430C210020FFF7C5FD002038BD00BFAF
:10CB5000A400FF1F943AFF1F38B90C21FFF7DDFD39
:10CB6000C0F380302860204638BD012840F0AD82F7
:10CB70000C210020FFF7D1FD2B689B0303F48043B9
:10CB800020F480421A430C210020FFF7A3FD00206F
:10CB900038BD38B90C21FFF7C0FDC0F3C1202860B3
:10CBA000204638BD012840F092820C210020FFF77A
:10CBB000B4FD2B68DB0203F4C05320F4C0521A43C7
:10CBC0000C210020FFF786FD002038BD38B90C216C
:10CBD000FFF7A3FDC0F3C3102860204638BD01282D
:10CBE00040F077820C210020FFF797FD2B68DB01D6
:10CBF00003F4F06320F4F0621A430C210020FFF7E5
:10CC000069FD002038BD40B90C210020FFF785FDEB
:10CC1000C0F302102860002038BD012840F05B827C
:10CC20000C210020FFF779FD2B681B0103F0700336
:10CC300020F070021A430C210020FFF74BFD00206A
:10CC400038BD38B90C21FFF768FD00F00F002860EF
:10CC5000204638BD012840F040820C210020FFF71B
:10CC60005CFD2B6820F00F0203F00F031A430C2128
:10CC70000020FFF72FFD002038BD38B90521FFF750
:10CC80004CFDC0F3C0302860204638BD012840F07C
:10CC900026820D210020FFF740FD2B68DB039BB2AD
:10CCA00020F400421A430D210020FFF713FD00205D
:10CCB00038BD38B90521FFF730FDC0F34130286099
:10CCC000204638BD012840F00C820D210020FFF7DE
:10CCD00024FD2B685B0303F4C04320F4C0421A43D5
:10CCE0000D210020FFF7F6FC002038BD38B90521E2
:10CCF000FFF713FDC0F303202860204638BD01284C
:10CD000040F0F1810D210020FFF707FD2B681B0289
:10CD100003F4706320F470621A430D210020FFF7C2
:10CD2000D9FC002038BD40B905210020FFF7F5FCF3
:10CD3000C0F341102860002038BD012840F0D581A3
:10CD40000D210020FFF7E9FC2B685B0103F0600375
:10CD500020F060021A430D210020FFF7BBFC0020E9
:10CD600038BD20B9BE4B1B685B6B2B6038BD0128FA
:10CD700040F0BD81BA4B2A681B6800205A6338BD59
:10CD800038B90621FFF7C9FCC0F3004028602046EF
:10CD900038BD012840F0AD810E210020FFF7BDFC19
:10CDA0002B681B0403F4803320F480321A430E21D5
:10CDB0000020FFF78FFC002038BD70B90621FFF777
:10CDC000ACFC000A00F07F0310F0400018BF6FF0C9
:10CDD0007F0018432860204638BD012840F08B8131
:10CDE0000E210020FFF799FC2B681B0203F4FE4381
:10CDF00020F4FE421A430E210020FFF76BFC0020B6
:10CE000038BD38B90721FFF788FCC0F381302860AE
:10CE1000204638BD012840F070810F210020FFF727
:10CE20007CFC2B689B039BB220F440421A430F21E9
:10CE30000020FFF74FFC002038BD40B9072100203B
:10CE4000FFF76BFCC0F301302860002038BD0128DB
:10CE500040F055810F210020FFF75FFC2B681B037A
:10CE600003F4405320F440521A430F210020FFF7EF
:10CE700031FC002038BD38B90721FFF74EFCC0F364
:10CE800080202860204638BD012840F03A810F21DB
:10CE90000020FFF742FC2B689B0203F4806320F420
:10CEA00080621A430F210020FFF714FC002038BDD8
:10CEB00038B90721FFF731FCC0F301202860204674
:10CEC00038BD012840F01F810F210020FFF725FC0D
:10CED0002B681B0203F4407320F440721A430F21A5
:10CEE0000020FFF7F7FB002038BD38B90721FFF716
:10CEF00014FCC0F380102860204638BD012840F0A3
:10CF000004810F210020FFF708FC2B689B0103F030
:10CF1000400320F040021A430F210020FFF7DAFB04
:10CF2000002038BD00287FF402AD0221FFF7F5FB99
:10CF3000C0F384202860204638BD38B9494B03EB44
:10CF4000810100204B68DB692B6038BD012840F06F
:10CF5000DE80444B2A6803EB810100204B68DA61D4
:10CF600083F8300038BD30B93E4B03EB81014B688C
:10CF70001B6A2B6038BD012840F0CB80394B2A68F2
:10CF800003EB810100204B681A6238BD38B90721D4
:10CF9000FFF7C3FBC0F3C0102860204638BD01284E
:10CFA00040F0B9800F210020FFF7B7FB2B68DB01B1
:10CFB000DBB220F080021A430F210020FFF78AFB2A
:10CFC000002038BD40B904210020FFF7A6FBC0F3C4
:10CFD00040302860002038BD012840F09E800C21A0
:10CFE0000020FFF79AFB2B685B0303F4005320F447
:10CFF00000521A430C210020FFF76CFB002038BDC3
:10D0000038B90721FFF789FBC0F3004028602046AC
:10D0100038BD012840F083800F210020FFF77DFB01
:10D020002B681B0403F4803320F480321A430F2151
:10D030000020FFF74FFB002038BD0A4B1B6833B1BF
:10D040000221FFF76AFB800A00F4787004E00121F6
:10D05000FFF763FBC0F389202860002038BD00BFC4
:10D06000780AFF1FA400FF1F00287FF460AC032193
:10D070000020FFF752FBC0B22860002038BD18B96D
:10D08000294B5B682B6038BD01284AD11A68264BB2
:10D0900000205A6038BD042038BD002038BD002073
:10D0A00038BD002038BD002038BD002038BD00202C
:10D0B00038BD002038BD002038BD102038BD00200C
:10D0C00038BD002038BD002038BD002038BD00200C
:10D0D00038BD002038BD002038BD002038BD0020FC
:10D0E00038BD002038BD002038BD002038BD0020EC
:10D0F00038BD002038BD002038BD002038BD0020DC
:10D1000038BD002038BD002038BD002038BD0020CB
:10D1100038BD002038BD002038BD002038BD0020BB
:10D1200038BD002038BD00BF943AFF1F07B50192FB
:10D1300029B9024601AB0120FFF726FB00E00820D9
:10D1400003B05DF804FB10B413460446084619B951
:10D15000224610BCFFF718BB082010BC704710B562
:10D160000D2104460020FFF7D8FA04F00F0420F048
:10D170000F0222430D210020BDE81040FFF7AABA9C
:10D180002DE9F8438B0C0C460ED0C1F34243062B1D
:10D190000AD1294B5A7A21F01F040AB11B7800E00A
:10D1A000DB7A03F01F031C43244F254E254D3B68BB
:10D1B000D6F8008095F819909B680021C4F30740C9
:10D1C00098476A7E336808EB890803EB8203C8F846
:10D1D00004005A6812025A603B6800219B68C4F33D
:10D1E0000720984733686A7E03EB82020121536867
:10D1F000184300023B6850609B68E0B29847326871
:10D20000697E02EB81014B6818430011A30C486052
:10D21000106107D0C4F34243072B09D1C4F30111B5
:10D22000697605E0082302EB83035C60BDE8F883C0
:10D2300043F00803F7E700BF943AFF1FD43AFF1FFB
:10D24000D83AFF1F8415FF1F2DE9F843494FDFF837
:10D250008481DFF88491484C01263846C8F8006084
:10D2600012F0DEFCD9F80C506B6803F16402E26046
:10D2700003F1840203F59270226103F5A27203F5B3
:10D28000017323602B68A260DB68606098472B689D
:10D29000A068DB6898472B68E068DB6898472B68D4
:10D2A00020691B6998472B682068DB689847D9F884
:10D2B0001030324A03F11001116022685A610523CF
:10D2C0003B7030464FF47A737B6012F059F92C4B67
:10D2D00062681B68C8F804305A62A2689A622269C0
:10D2E000DA620021274A1A659963274B2748DA6FCB
:10D2F00002602748C2F80802264811705170C2F82F
:10D300000402254AC3F88820244AC3F88420244A0A
:10D31000C3F88020234AC3F88C20234AC3F8A020F6
:10D32000224AC3F89C20224AC3F89020214AC3F81D
:10D330009420214AC3F8B020204AC3F8AC20204AE8
:10D34000C3F8BC201F4AC3F8B8201F4AC3F8B42052
:10D350001E4AC3F8C82032225A6740F2251283F8C9
:10D3600078601A671A4AC3F8C0200220BDE8F84363
:10D37000FFF7E8B8943AFF1F8415FF1FD43AFF1F48
:10D38000780AFF1F5FD10000C82EFF1FD83AFF1F89
:10D39000E1C40000D5C50000EDC400000DC50000CB
:10D3A0000FC5000013C5000047D100002DD10000BB
:10D3B00089C4000017C5000011C7000079C700002C
:10D3C0009DC4000059C4000031C5000045C50000DF
:10D3D00085C50000A400FF1F0C550200014B002270
:10D3E0005A607047C82EFF1F0128F8B5144633D085
:10D3F0000BD3FF2843D1244CE36FD3F80432984772
:10D400006369D3F8043298472FE0136833F00302BE
:10D4100037D113F0010F1D4D1D4E03D0F3681B686B
:10D420001B6906E0F76828693B68DB6898473B683A
:10D430009B6928699847206810F0020403D0F368BC
:10D440001B681B6906E0F66868693368DB68984703
:10D4500033689B69686907E014680C4D0C4B34B164
:10D46000DB681B681B69E86898470020F8BDDE6828
:10D47000E8683368DB68984733689B69F3E7042002
:10D48000F8BD1020F8BD00BFC82EFF1FAC15FF1F50
:10D490000C55020070B5144E144CF56860682B688A
:10D4A0009B6998472B6860699B6898472B6820693F
:10D4B0009B6898472B68E0689B6898472B68A06832
:10D4C0009B6898472B68A0699B6898472B682068E1
:10D4D0009B6898472B6860689B6898473369BDE8EC
:10D4E0007040DB69184700BF0C550200AC15FF1FE8
:10D4F0002DE9F843194C9DF820501E4623688946B3
:10D5000007469B68002140F0800090469847144BE6
:10D5100083F8E002236800219B6848469847236807
:10D5200000219B6840469847236800219B6830464D
:10D530009847236828469B6801219847094B1B6838
:10D5400048EA092807F07F0746EA082603EB870721
:10D5500045EA06257D60BDE8F88300BFDC3AFF1F81
:10D56000E43AFF1FE03AFF1F07B5CBB20093C1F3C7
:10D570000742C1F30723090EFFF7BAFF03B05DF8B6
:10D5800004FBFFF7F1BF10B50F4C104A2368D268B7
:10D59000197812680E4B31B9926958689047236820
:10D5A00001221A700EE05868526990470421102039
:10D5B000FFF7DAFF236800221A70064BDB6FD3F8FF
:10D5C00004329847012010BDE03AFF1F0C550200BD
:10D5D000AC15FF1FC82EFF1F10B5064C0649226868
:10D5E00012F0ACFD23681B7813B1BDE81040CAE708
:10D5F00010BD00BFE03AFF1FE43AFF1F10B500293D
:10D6000040F08880122867D01AD805284CD007D857
:10D61000012837D033D3022837D0042835D07BE017
:10D620000F2847D007D80E2876D1002A14BF022130
:10D63000012120204CE010283FD0112843D06BE07E
:10D6400017285BD009D814284FD048D315284FD0BD
:10D65000162861D111462D203AE01A2854D006D858
:10D6600018284ED0192857D11146302030E01B28F9
:10D670004DD0D62850D12A491520514328E01146D3
:10D68000372025E01146212022E082EAE271254B75
:10D69000A1EBE271994204DD234911EA220238BF6D
:10D6A0001A461102242013E0940DA405B4BB910086
:10D6B00028200DE0114625200AE0940DA40574BB36
:10D6C00091002A2004E0930D9B053BBB910029208B
:10D6D000FFF74AFF002010BD11462720F8E7940D00
:10D6E000A405DCB991002B20F2E711462620EFE7D4
:10D6F000940DA40594B911462C20E9E711462E207B
:10D70000E6E711462F20E3E711463320E0E7114614
:10D710003420DDE7082010BD042010BD102010BD0E
:10D720000071020000127A0000EE85FF70B5254EF0
:10D7300000F07F04331993F80C32DB0705D4224B39
:10D740001B6803EB8404606870BD204D2B680021CA
:10D750009B68204698472B6800219B68084698479D
:10D760002B6800219B68084698472B6800219B681E
:10D77000084698472B6801219B68002098472B6832
:10D7800000219B68204698472B6886F8E00200211C
:10D790009B68084698472B68002104029B6808464E
:10D7A00098472B680021204304029B68084698474D
:10D7B0002B68204304029B680121002098472043E6
:10D7C00070BD00BFE43AFF1FE03AFF1FDC3AFF1FC5
:10D7D00010B50C46FFF7AAFF206010BD38B50D4606
:10D7E000044668B92020FFF7A1FF40F00401202083
:10D7F000FFF7BAFE29463720FFF7B6FE204638BDB0
:10D80000082038BD38B50C4605462120FFF78EFFAD
:10D810002368C11821602846BDE83840DEE738B5E6
:10D8200015460C4600296CD1112852D01ED8042868
:10D8300041D008D801283CD039D302283BD0032856
:10D8400061D1222058E00E283CD009D8052837D0D5
:10D85000082858D10F20FFF769FF00F001004DE0C4
:10D860000F2834D010284ED12A2036E017283CD07B
:10D870000ED8142835D005D812282CD0132842D120
:10D880002B202AE015282ED016283CD12D2033E05D
:10D890001A282ED005D8182829D0192833D130209D
:10D8A0002AE01B2827D0D6282DD1152024E03720A8
:10D8B00022E0212020E02420FFF738FF00121DE0A5
:10D8C00028200AE02020FFF731FF400016E0252045
:10D8D00012E0292001E027200EE0FFF727FF80104B
:10D8E0000CE0262008E02C2006E02E2004E02F206B
:10D8F00002E0332000E03420FFF718FF28602046C4
:10D9000038BD082038BD042038BD10B50C46C8B954
:10D910002020FFF70BFF20F004012020FFF724FE5A
:10D9200084EAE472084BA2EBE4729A4204DD074AEF
:10D9300012EA240438BF1C4621022420FFF714FEFB
:10D94000002010BD082010BD00127A0000EE85FFF7
:10D950000021DAE74942D8E7D7E770B53F4E4048A3
:10D96000404C12F003FBF5686B6803F58272A2610C
:10D9700003F55172626103F55972226103F5617218
:10D9800003F57970E26003F5697203F204432360E2
:10D990002B68A260DB68606098472B686069DB6871
:10D9A00098472B682069DB6898472B68E068DB683C
:10D9B00098472B68A068DB6898472B6860685B69AC
:10D9C00098472B6860695B6998472B6820695B6999
:10D9D00098472B68E0685B6998472B68A0685B698B
:10D9E00098472B68A0691B6998472B6820681B69BA
:10D9F0001D4C98471D4B32691A606B6803F53173F3
:10DA000053601B4B62691A6001212020FFF7ACFDB7
:10DA10006369184AC3F8042200225A7001221A705E
:10DA2000154B2362154BE361154BA361154B6362E4
:10DA3000154BA363154B6363154BA362154BE36250
:10DA4000154BA364154B6364154B6365154B236538
:10DA5000154BE3652274154BA36570BD0C55020090
:10DA6000E43AFF1FAC15FF1FC82EFF1FDC3AFF1F53
:10DA7000E03AFF1F87D500000BD9000059D90000FC
:10DA800055D9000051D900001FD80000FDD5000075
:10DA9000DDD7000005D8000083D50000D1D70000F5
:10DAA000D9D50000E9D30000DDD3000095D40000F3
:10DAB000014B00225A607047C82EFF1F0128F8B59D
:10DAC000144633D00BD3FF2843D1244CE36FD3F853
:10DAD000043298476369D3F8043298472FE01368FB
:10DAE00033F0030237D113F0010F1D4D1D4E03D04B
:10DAF000F3681B681B6906E0F76828693B68DB6808
:10DB000098473B689B6928699847206810F0020491
:10DB100003D0F3681B681B6906E0F6686869336820
:10DB2000DB68984733689B69686907E014680C4DA7
:10DB30000C4B34B1DB681B681B69E8689847002010
:10DB4000F8BDDE68E8683368DB68984733689B692E
:10DB5000F3E70420F8BD1020F8BD00BFC82EFF1F5A
:10DB6000D815FF1F0C55020070B5164E164CF568FF
:10DB700060682B689B6998472B6860699B68984729
:10DB80002B6820699B6898472B68E0689B689847DA
:10DB90002B68A0689B6898472B68E0699B6898474A
:10DBA0002B68A0699B6898472B6820689B689847FA
:10DBB0002B6860689B6898473369BDE87040DB69F3
:10DBC000184700BF0C550200D815FF1F38B50A4B87
:10DBD0000A4CDD6860682B689B69984701200EF04D
:10DBE00029FC2B6860685B699847054B186812F040
:10DBF00009FB012038BD00BF0C550200D815FF1FDE
:10DC0000C83DFF1F38B50A4B0A4CDD6860682B68B9
:10DC10009B69984701200EF00DFC2B6860685B69DA
:10DC20009847054B186812F0E4FA012038BD00BF90
:10DC30000C550200D815FF1FC83DFF1F2DE9F84302
:10DC4000194D9DF820909DF8244098462B680E466B
:10DC50009B68002146F0800017469847134B83F8D5
:10DC6000E0022B6800219B68384698472B6800210A
:10DC70009B68404698472B6800219B684846984718
:10DC80002B6801219B6820469847094B1B6806F0CA
:10DC90007F0644EA092203EB860642EA084242EA8A
:10DCA00007627260BDE8F883CC3DFF1FD03DFF1FC7
:10DCB000C83DFF1F07B5D3B20193C2F307230093FA
:10DCC000C2F30743120EFFF7B9FF03B05DF804FB80
:10DCD00070B5174C174A23681D780146002012F0D2
:10DCE0003BFB1DB323681A7802BB134C94F86830D1
:10DCF000012B06D0032B0BBF002228220D230F235C
:10DD000000E00B2343F0884343F0401343EA4232E0
:10DD100004210020FFF7CEFFE36F012D0CBFD3F8E5
:10DD20000432D3F80832BDE87040184770BD00BF18
:10DD3000C83DFF1FD03DFF1FC82EFF1F0A460146EA
:10DD40000020FFF7B7BF38B514460D4600297ED135
:10DD5000122863D01AD8052848D007D8012834D013
:10DD600031D3022833D0042831D072E00F2843D0B9
:10DD700007D80E286DD1002A14BF022201222021CB
:10DD800063E010283AD011283ED062E0172855D021
:10DD900008D814284AD043D3152849D0162858D17A
:10DDA0002D2152E01A284DD005D8182848D019281E
:10DDB0004FD1302149E01B2846D0D62849D1274AE7
:10DDC0001521624341E037213FE021213DE084EA13
:10DDD000E472234BA2EBE4729A4204DD214A12EA78
:10DDE000240438BF1C462202242112E0950DAD0503
:10DDF0008DBB9200282128E0252126E0950DAD0558
:10DE000055BB92002A2120E0930D9B051BBB92007D
:10DE100029210020FFF74EFF002038BD272114E004
:10DE2000950DAD05BDB992002B210EE026210CE029
:10DE3000940DA4057CB92C212046EBE72E2104E0AB
:10DE40002F2102E0332100E034212846E2E70820B8
:10DE500038BD042038BD102038BD00BF007102005D
:10DE600000127A0000EE85FF70B5254E01F07F04A8
:10DE7000331993F80C32DB0705D4224B1B6803EBF4
:10DE80008404606870BD204D2B6800219B6820468B
:10DE900098472B6800219B68084698472B6800210B
:10DEA0009B68084698472B6800219B68084698475E
:10DEB0002B6801219B68002098472B6800219B68F4
:10DEC000204698472B6886F8E00200219B680846A8
:10DED00098472B68002104029B68084698472B68E6
:10DEE0000021204304029B68084698472B68204382
:10DEF00004029B68012100209847204370BD00BFA9
:10DF0000D03DFF1FC83DFF1FCC3DFF1F10B50C4685
:10DF100001460020FFF7A8FF206010BD38B50D4670
:10DF2000044678B92021FFF79FFF202140F004022A
:10DF30002046FFF7BFFE20462A463721FFF7BAFEEC
:10DF4000204638BD082038BD38B50C46212105468D
:10DF5000FFF78AFF2168014421602846BDE8384068
:10DF6000DCE738B515460C46002975D1112859D083
:10DF70001FD8042842D008D801283DD03AD302281F
:10DF80003CD003286AD1222160E00E283ED00AD876
:10DF9000052839D0082861D10F212046FFF764FFFA
:10DFA00000F0010055E00F283AD0102856D12A2160
:10DFB0003CE0172843D00ED814283CD005D81228AE
:10DFC00032D013284AD12B2130E0152835D016281D
:10DFD00044D12D213AE01A2835D005D8182830D060
:10DFE00019283BD1302131E01B282ED0D62835D13D
:10DFF00015212BE0372129E0212127E0242120468B
:10E00000FFF732FF001224E028210FE020212046F4
:10E01000FFF72AFF00F00300831E5842584118E022
:10E02000252113E0292101E027210FE02046FFF7F9
:10E030001BFF80100DE0262108E02C2106E02E2198
:10E0400004E02F2102E0332100E034212046FFF7D5
:10E050000BFF2860204638BD082038BD042038BD9D
:10E0600038B50C460546D8B92021FFF7FDFE202122
:10E0700020F004022846FFF71DFE84EAE472094BF3
:10E08000A2EBE4729A4204DD074A12EA240438BF84
:10E090001C46220224210020FFF70CFE002038BD80
:10E0A000082038BD00127A0000EE85FF0021D7E776
:10E0B0004942D5E7D4E7354B2DE9F0415E6A1A6A4B
:10E0C000350245EA12651402C6B293F82820586B4F
:10E0D000264300271C6B2F430132050E000240EA45
:10E0E0001460D2B224021C63C3E9086783F82820B5
:10E0F00058631C46002945D0042A04D93A466D21AC
:10E100000020FFF7D7FD226ADFF880806C21002015
:10E11000FFF7D0FD01200EF08DF9226A6C2100205E
:10E12000FFF7C8FD01200EF085F900230022C4E9A5
:10E130000C2394F82830042B0AD96F210020FFF714
:10E1400093FED8E90C23002632430343C8E90C238D
:10E150006E210020FFF788FED4E90C6794F8282090
:10E160000346C2F10802D20047EAE371304316F0D9
:10E1700075F800230022C4E90C01C4E90823002338
:10E1800084F828302846BDE8F08100BFD815FF1F6D
:10E1900070B5464E4648474C11F0E2FFF5686B6893
:10E1A00003F1E402E26103F58272A26103F55172A8
:10E1B000626103F55972226103F5617203F57970AA
:10E1C000E26003F5697203F2044323602B68A260E6
:10E1D000DB68606098472B686069DB6898472B684C
:10E1E0002069DB6898472B68E068DB6898472B68F4
:10E1F000A068DB6898472B6860685B6998472B6864
:10E2000060695B6998472B6820695B6998472B6850
:10E21000E0685B6998472B68A0685B6998472B6842
:10E22000E0691B6998472B68A0691B6998472B68B0
:10E2300020681B69204C9847204B32691A606B6834
:10E2400003F5317353601E4B62691A60202101226D
:10E250000020FFF72FFD6369002159701949C3F8A9
:10E260000412012218491A70C3F80812174B63668A
:10E27000174B2362174BE361174BA361174B636284
:10E28000174BA363174B6363174BA362174BE362F0
:10E29000174BA364174B6364174B6365174B2365D8
:10E2A000174BE3652274174BA36570BD0C55020034
:10E2B000D03DFF1FD815FF1FC82EFF1FCC3DFF1FED
:10E2C000C83DFF1F05DC0000CDDB0000B7E000000B
:10E2D00061E00000B5E00000B1E00000ADE000004A
:10E2E00063DF000047DD00001DDF000049DF0000A4
:10E2F0003DDD00000DDF0000D1DC0000BDDA0000D4
:10E30000B1DA000069DB0000014B00225A6070475F
:10E31000C82EFF1F70B5184E184CF56860682B6842
:10E320009B6998472B68A0699B6898472B68606930
:10E330009B6898472B6820699B6898472B68E06822
:10E340009B6898472B68A0689B6898472B68206A51
:10E350009B6898472B68E0699B6898472B68206802
:10E360009B6898472B6860689B6898473369BDE84D
:10E370007040DB69184700BF0C5502002016FF1FD4
:10E380000228F8B514464CD003D880B1012835D006
:10E3900060E0032856D0FF285CD12F4CE36FD3F800
:10E3A000043298476369D3F8043298472FE0136822
:10E3B00033F003022BD113F0010F284D284E03D068
:10E3C000F3681B681B6906E0F76868693B68DB68EF
:10E3D00098473B689B6968699847206810F0020479
:10E3E00003D0F3681B681B6906E0F668A869336808
:10E3F000DB68984733689B69A86907E01468174D84
:10E40000174B34B1DB681B681B69286998470020EB
:10E41000F8BDDE6828693368DB68984733689B6914
:10E42000F3E714680D4D0E4B1CB1DB681B681B69CC
:10E4300006E0DE68A8683368DB68984733689B6944
:10E44000A868E3E7012012F017F820600028DED169
:10E450002020F8BD0420F8BDC82EFF1F2016FF1F86
:10E460000C55020038B50A4B0A4CDD6860682B6811
:10E470009B69984701200DF0DDFF2B6860685B69A0
:10E480009847054B186811F0CCFF012038BD00BF3C
:10E490000C5502002016FF1FB440FF1F38B50A4B71
:10E4A0000A4CDD6860682B689B69984701200DF075
:10E4B000C1FF2B6860685B699847054B186811F0CD
:10E4C000A7FF012038BD00BF0C5502002016FF1F1A
:10E4D000B440FF1F2DE9F843194D9DF8204099469F
:10E4E0002B680F4606469B68002140F0800090464E
:10E4F0009847144B83F8E0022B6800219B6838464C
:10E5000098472B6800219B68404698472B6800215C
:10E510009B68484698472B6801219B68204698478E
:10E52000094B1B6806F07F0644EA092103EB8606C7
:10E5300041EA084141EA07617160BDE8F88300BF24
:10E54000B840FF1FBC40FF1FB440FF1F07B5CBB250
:10E550000093C1F30742C1F30723090EFFF7BAFF87
:10E5600003B05DF804FB70B5154C164922681578A8
:10E5700011F0ECFF15B323681978F9B9124C94F82F
:10E580006830012B06D0032B0BBF002128210D235F
:10E590000F2300E00B2343F0884343F0401343EA8A
:10E5A00041310420FFF7D2FFE36F012D0CBFD3F8F8
:10E5B0000432D3F80832BDE87040184770BD00BF80
:10E5C000B440FF1FBC40FF1FC82EFF1FFFF7BEBF98
:10E5D00070B5254E00F07F04331993F80C32DB0739
:10E5E00005D4224B1B6803EB8404606870BD204D8A
:10E5F0002B6800219B68204698472B6800219B6868
:10E60000084698472B6800219B68084698472B6866
:10E6100000219B68084698472B6801219B680020D1
:10E6200098472B6800219B68204698472B6886F8FE
:10E63000E00200219B68084698472B6800210402ED
:10E640009B68084698472B680021204304029B687A
:10E65000084698472B68204304029B68012100204C
:10E660009847204370BD00BFBC40FF1FB440FF1F50
:10E67000B840FF1F10B50C46FFF7AAFF206010BD81
:10E6800038B50D46044668B92020FFF7A1FF40F0D9
:10E6900004012020FFF75AFF29463720FFF756FFD5
:10E6A000204638BD082038BD38B50C460546212027
:10E6B000FFF78EFF2368C11821602846BDE8384067
:10E6C000DEE76F2970B50446154600F0BA8155D8CB
:10E6D000122900F02A8127D8052900F0D88011D806
:10E6E000022900F0B48006D8002900F09E8001299C
:10E6F00000F0A480F0E2032900F0AF80042900F0CC
:10E70000A680E9E20F2900F0E98006D8082900F088
:10E71000CD800E2900F0D280DEE2102900F0E780E3
:10E72000112900F0F380D7E2182900F0428111D8B6
:10E73000152900F01E8106D8132900F0FF80142946
:10E7400000F00E81C8E2162900F02181172900F09F
:10E750002781C1E21B2900F0478106D8192900F062
:10E7600031811A2900F03781B6E26D2900F04E811F
:10E7700000F255816C2900F04081ADE27D2900F066
:10E78000048227D8752900F0AF8111D8722900F0D2
:10E79000838106D8702900F06581712900F06B81B2
:10E7A0009AE2732900F08A81742900F0928193E241
:10E7B000782900F0D28106D8762900F0B181772936
:10E7C00000F0C38188E2792900F0CF817C2900F034
:10E7D000D48181E2882900F0218211D8842900F0B7
:10E7E000058206D87E2900F0D881812900F0EC81CD
:10E7F00072E2852900F0FF81862900F007826BE232
:10E80000C82900F0388106D8892900F019828A29A0
:10E8100000F02D8260E2D42900F04682D62900F073
:10E820004E82D12940F0588234E208B9372033E2D1
:10E83000012840F0B981116837204AE208B9212047
:10E840002AE2012840F0B0811168212041E25CB940
:10E850002420FFF7BDFE0012A5E108B922201BE22B
:10E86000012C00F039829FE1012C40F09D81296844
:10E87000A14B81EAE172A2EBE1729A4204DD9F4A68
:10E8800012EA210138BF19460902242021E208B901
:10E89000282055E0012840F0878111688C0DA405DF
:10E8A000002C40F01B828900282012E20028D7D1DA
:10E8B0000F20FFF78DFE00F0010074E120B9202049
:10E8C000FFF786FE40006EE1012840F06D8113687D
:10E8D000002B14BF022101212020FAE108B92520D4
:10E8E000DAE1012840F0608111682520F1E108B9E2
:10E8F0002A2025E0012840F0578111688C0DA405DD
:10E90000002C40F0EB8189002A20E2E108B929209F
:10E9100016E0012840F0488111688C0DA405002CF8
:10E9200040F0DC8189002920D3E108B92720B3E138
:10E93000012840F0398111682720CAE120B92B2035
:10E94000FFF746FE80102EE1012840F02D8111686E
:10E950008C0DA405002C40F0C18189002B20B8E16A
:10E9600008B9262098E1012840F01E811168262070
:10E97000AFE108B92C208FE1012840F01581116822
:10E980008B0D9B05002B40F0A9812C20A1E108B93B
:10E990002D2081E1012840F0078111682D2098E1A8
:10E9A00008B92E2078E1012840F0FE8011682E2061
:10E9B0008FE108B92F206FE1012840F0F580116840
:10E9C0002F2086E108B9302066E1012840F0EC8074
:10E9D000116830207DE108B933205DE1012840F065
:10E9E000E3801168332074E108B9342054E1012830
:10E9F00040F0DA80116834206BE108B960204BE107
:10EA0000012840F0D1801168602062E108B96120DE
:10EA100042E1012840F0C8801168612059E120B925
:10EA20001C20FFF7D5FD0014BDE0012840F0BC809C
:10EA30001C20FFF7CDFD2968C0F3080040EA014122
:10EA40000EE008B91C2018E0012840F0AD801C2021
:10EA5000FFF7BEFD2B6800F47F01C3F308031943E1
:10EA60001C2036E108B9592016E1012840F09C80AD
:10EA7000116859202DE124B90620FFF7A9FDC0B285
:10EA800091E0012C40F090800620FFF7A1FD29784D
:10EA900020F0FF00014395E028B90620FFF798FD1C
:10EAA000C0F307207FE001287ED10620FFF790FD0C
:10EAB0002B681B0220F47F419BB282E020B9104BEF
:10EAC0001B68D3F86C3109E001286DD111685A2018
:10EAD000FFE028B90A4B1B68D3F870312B6063E064
:10EAE000012861D111682EE060B9054B1B68D3F88D
:10EAF0007031C3F30E03F1E700127A0000EE85FFD8
:10EB0000B440FF1F01284FD1754B11681B68D3F823
:10EB1000703123F4FF4323F07F03C1F30E0111E0B2
:10EB200020B96F4B1B6893F87231D7E701283BD1AE
:10EB30006B4B1B68D3F8701113681B0421F47F0121
:10EB400003F47F0319435B20C3E008B95E20A3E010
:10EB5000012829D111685E20BBE008B918209BE08C
:10EB6000012821D111681820B3E008B9192093E0D9
:10EB7000012819D111681920ABE008B95C208BE09D
:10EB8000012811D111685C20A3E008B95F2083E05F
:10EB9000012809D111685F209BE038B90620FFF7F2
:10EBA00017FDC0F307402860002070BD0128FBD18D
:10EBB0000620FFF70DFD2B681B0420F47F0103F4F2
:10EBC0007F031943062084E00128EDD1166836B191
:10EBD00011F052FC28600028E6D1202070BD0720EB
:10EBE000FFF7F6FC20F48001072072E000287FF494
:10EBF00037AE652050E00028D6D10720FFF7E8FCAB
:10EC0000C0F38150431E58425841CCE708B9522006
:10EC100042E00128C8D1116852205AE020B9304B97
:10EC20001B6893F8903159E70128BDD12C4B11682E
:10EC30001B68D3F8903101F00F0123F0FF0313E0BC
:10EC400030B9274B1B68D3F89031C3F3032345E752
:10EC50000128A9D1224B1B68D3F8901113681B021D
:10EC600021F4706103F470631943632031E020B92B
:10EC70001B4B1B6893F8923130E7012894D1184B55
:10EC80001B68D3F8901113681B0421F47F0103F46F
:10EC90007F03E9E718B95020FFF79AFC83E70128C2
:10ECA00082D11168502014E018B90D4B1B68DB6944
:10ECB00014E701287FF478AF1168532009E008B900
:10ECC0001520E9E701287FF46FAF13680549152087
:10ECD0005943FFF73BFC67E7042070BD102070BD6F
:10ECE000B440FF1F0071020007B5019229B9014627
:10ECF00001AA0120FFF7E5FC00E0082003B05DF861
:10ED000004FB0B4611B901461846DAE408207047A7
:10ED100010B50C46C8B92020FFF75AFC20F00401BA
:10ED20002020FFF713FC84EAE472094BA2EBE472A3
:10ED30009A4204DD074A12EA240438BF1C46210225
:10ED40002420FFF703FC002010BD082010BD00BFE9
:10ED500000127A0000EE85FF0021D9E74942D7E78B
:10ED6000D6E7324B2DE9F041DE6A9A6A350245EA70
:10ED700012651402C6B293F83020D86B26430027E0
:10ED80009C6B2F430132050E000240EA1460D2B2A0
:10ED900024029C63C3E90A6783F83020D8631C46C9
:10EDA000002940D0042A03D939466D20FFF7CEFB55
:10EDB000A16ADFF878806C20FFF7C8FB01200DF016
:10EDC00039FBA16A6C20FFF7C1FB01200DF032FB7B
:10EDD00000230022C4E90E2394F83030042B09D913
:10EDE0006F20FFF7F5FBD8E90E23002632430343DB
:10EDF000C8E90E236E20FFF7EBFBD4E90E6794F809
:10EE000030200346C2F10802D20047EAE3713043E2
:10EE100015F024FA00230022C4E90E01C4E90A23F4
:10EE2000002384F830302846BDE8F0812016FF1F0B
:10EE300070B54B4E4B484C4C11F0A0FAF5686B681E
:10EE400003F1E402226203F58272E26103F551727A
:10EE5000A26103F55972626103F56172226103F5E3
:10EE6000697203F57970E26003F5717203F204438D
:10EE700023602B68A260DB68606098472B68A069FC
:10EE8000DB6898472B686069DB6898472B682069C6
:10EE9000DB6898472B68E068DB6898472B68A068B8
:10EEA000DB6898472B6860685B6998472B68A069A6
:10EEB0005B6998472B6860695B6998472B68206994
:10EEC0005B6998472B68E0685B6998472B68A06886
:10EED0005B6998472B68206A1B6998472B68E06933
:10EEE0001B6998472B6820681B69204C9847204B6A
:10EEF00032691A606B6803F5317353601D4B6269A8
:10EF00001A6001212020FFF721FB6369002159705D
:10EF10001949C3F80412012218491A70C3F80812DB
:10EF2000174B6366174B2362174BE361174BA361C3
:10EF3000174B6362174BA363174B6363174BA362B3
:10EF4000174BE362174BA364174B6364174B63655E
:10EF5000174B2365174BE3652274174BA36570BDF0
:10EF60000C550200BC40FF1F2016FF1FC82EFF1FBC
:10EF7000B840FF1FB440FF1F9DE4000065E400009F
:10EF800063ED000011ED000061ED00005DED00009B
:10EF900059ED000003ED0000E9EC000081E60000FF
:10EFA000A9E60000CDE5000075E6000067E5000079
:10EFB00081E3000009E3000015E30000014B00229B
:10EFC0005A607047C82EFF1F70B5184E184CF56870
:10EFD00060682B689B6998472B68A0699B68984775
:10EFE0002B6860699B6898472B6820699B689847E5
:10EFF0002B68E0689B6898472B68A0689B689847D7
:10F000002B68206A9B6898472B68E0699B68984743
:10F010002B6820689B6898472B6860689B689847B6
:10F020003369BDE87040DB69184700BF0C5502002A
:10F030007016FF1F0228F8B514464CD003D880B1D3
:10F04000012835D060E0032856D0FF285CD12F4C32
:10F05000E36FD3F8043298476369D3F804329847D2
:10F060002FE0136833F003022BD113F0010F284D6A
:10F07000284E03D0F3681B681B6906E0F7686869CF
:10F080003B68DB6898473B689B69686998472068DC
:10F0900010F0020403D0F3681B681B6906E0F668F1
:10F0A000A8693368DB68984733689B69A86907E0FB
:10F0B0001468174D174B34B1DB681B681B6928694E
:10F0C00098470020F8BDDE6828693368DB689847F8
:10F0D00033689B69F3E714680D4D0E4B1CB1DB6878
:10F0E0001B681B6906E0DE68A8683368DB68984720
:10F0F00033689B69A868E3E7012011F0B7FA206044
:10F100000028DED12020F8BD0420F8BDC82EFF1F46
:10F110007016FF1F0C55020038B50A4B0A4CDD680B
:10F1200060682B689B69984701200DF083F92B6874
:10F1300060685B699847054B186811F06CFA01200C
:10F1400038BD00BF0C5502007016FF1F8846FF1F18
:10F1500038B50A4B0A4CDD6860682B689B69984794
:10F1600001200DF067F92B6860685B699847054BD3
:10F17000186811F047FA012038BD00BF0C55020095
:10F180007016FF1F8846FF1F2DE9F843194D9DF8A3
:10F19000204099462B680F4606469B68002140F0A8
:10F1A000800090469847144B83F8E0022B680021BA
:10F1B0009B68384698472B6800219B6840469847D3
:10F1C0002B6800219B68484698472B6801219B6863
:10F1D00020469847094B1B6806F07F0644EA092140
:10F1E00003EB860641EA084141EA07617160BDE828
:10F1F000F88300BF8446FF1FA043FF1F8846FF1F00
:10F2000007B5CBB20093C1F30742C1F30723090E40
:10F21000FFF7BAFF03B05DF804FB70B5154C164953
:10F220002268157811F08CFA15B323681978F9B9AA
:10F23000124C94F86830012B06D0032B0BBF002131
:10F2400028210D230F2300E00B2343F0884343F0D4
:10F25000401343EA41310420FFF7D2FFE36F012D51
:10F260000CBFD3F80432D3F80832BDE87040184719
:10F2700070BD00BF8846FF1FA043FF1FC82EFF1FA1
:10F28000FFF7BEBF70B5254E00F07F04331993F829
:10F290000C32DB0705D4224B1B6803EB8404606847
:10F2A00070BD204D2B6800219B68204698472B6835
:10F2B00000219B68084698472B6800219B680846F8
:10F2C00098472B6800219B68084698472B680121C6
:10F2D0009B68002098472B6800219B682046984730
:10F2E0002B6886F8E00200219B68084698472B6847
:10F2F000002104029B68084698472B6800212043A0
:10F3000004029B68084698472B68204304029B68C8
:10F31000012100209847204370BD00BFA043FF1F7C
:10F320008846FF1F8446FF1F10B50C46FFF7AAFF53
:10F33000206010BD38B50D46044668B92020FFF79F
:10F34000A1FF40F004012020FFF75AFF2946372093
:10F35000FFF756FF204638BD082038BD38B50C46AB
:10F3600005462120FFF78EFF2368C118216028463B
:10F37000BDE83840DEE76F2970B50446154600F059
:10F38000BA8155D8122900F02A8127D8052900F022
:10F39000D88011D8022900F0B48006D8002900F0E6
:10F3A0009E80012900F0A480F0E2032900F0AF80E4
:10F3B000042900F0A680E9E20F2900F0E98006D8D0
:10F3C000082900F0CD800E2900F0D280DEE210295D
:10F3D00000F0E780112900F0F380D7E2182900F04F
:10F3E000428111D8152900F01E8106D8132900F09A
:10F3F000FF80142900F00E81C8E2162900F0218157
:10F40000172900F02781C1E21B2900F0478106D8A7
:10F41000192900F031811A2900F03781B6E26D29EF
:10F4200000F04E8100F255816C2900F04081ADE280
:10F430007D2900F0048227D8752900F0AF8111D80A
:10F44000722900F0838106D8702900F06581712946
:10F4500000F06B819AE2732900F08A81742900F030
:10F46000928193E2782900F0D28106D8762900F0C3
:10F47000B181772900F0C38188E2792900F0CF813A
:10F480007C2900F0D48181E2882900F0218211D802
:10F49000842900F0058206D87E2900F0D8818129D0
:10F4A00000F0EC8172E2852900F0FF81862900F0EE
:10F4B00007826BE2C82900F0388106D8892900F05C
:10F4C00019828A2900F02D8260E2D42900F0468258
:10F4D000D62900F04E82D12940F0588234E208B992
:10F4E000372033E2012840F0B981116837204AE221
:10F4F00008B921202AE2012840F0B08111682120BA
:10F5000041E25CB92420FFF7BDFE0012A5E108B975
:10F5100022201BE2012C00F039829FE1012C40F0F7
:10F520009D812968A14B81EAE172A2EBE1729A42C6
:10F5300004DD9F4A12EA210138BF1946090224203E
:10F5400021E208B9282055E0012840F087811168A0
:10F550008C0DA405002C40F01B828900282012E2AB
:10F560000028D7D10F20FFF78DFE00F0010074E1D5
:10F5700020B92020FFF786FE40006EE1012840F010
:10F580006D811368002B14BF022101212020FAE1B4
:10F5900008B92520DAE1012840F0608111682520B2
:10F5A000F1E108B92A2025E0012840F057811168CF
:10F5B0008C0DA405002C40F0EB8189002A20E2E1AB
:10F5C00008B9292016E0012840F0488111688C0D07
:10F5D000A405002C40F0DC8189002920D3E108B982
:10F5E0002720B3E1012840F0398111682720CAE1C2
:10F5F00020B92B20FFF746FE80102EE1012840F0B5
:10F600002D8111688C0DA405002C40F0C18189006A
:10F610002B20B8E108B9262098E1012840F01E818E
:10F6200011682620AFE108B92C208FE1012840F0B5
:10F63000158111688B0D9B05002B40F0A9812C20B2
:10F64000A1E108B92D2081E1012840F0078111686E
:10F650002D2098E108B92E2078E1012840F0FE80A5
:10F6600011682E208FE108B92F206FE1012840F0AA
:10F67000F58011682F2086E108B9302066E1012865
:10F6800040F0EC80116830207DE108B933205DE165
:10F69000012840F0E3801168332074E108B9342078
:10F6A00054E1012840F0DA80116834206BE108B998
:10F6B00060204BE1012840F0D1801168602062E1B8
:10F6C00008B9612042E1012840F0C880116861203A
:10F6D00059E120B91C20FFF7D5FD0014BDE0012839
:10F6E00040F0BC801C20FFF7CDFD2968C0F3080066
:10F6F00040EA01410EE008B91C2018E0012840F062
:10F70000AD801C20FFF7BEFD2B6800F47F01C3F322
:10F71000080319431C2036E108B9592016E10128D5
:10F7200040F09C80116859202DE124B90620FFF794
:10F73000A9FDC0B291E0012C40F090800620FFF7B7
:10F74000A1FD297820F0FF00014395E028B90620AB
:10F75000FFF798FDC0F307207FE001287ED1062047
:10F76000FFF790FD2B681B0220F47F419BB282E0E3
:10F7700020B9104B1B68D3F86C3109E001286DD11A
:10F7800011685A20FFE028B90A4B1B68D3F8703182
:10F790002B6063E0012861D111682EE060B9054B50
:10F7A0001B68D3F87031C3F30E03F1E700127A003F
:10F7B00000EE85FF8846FF1F01284FD1754B116869
:10F7C0001B68D3F8703123F4FF4323F07F03C1F3A8
:10F7D0000E0111E020B96F4B1B6893F87231D7E727
:10F7E00001283BD16B4B1B68D3F8701113681B04C5
:10F7F00021F47F0103F47F0319435B20C3E008B9C0
:10F800005E20A3E0012829D111685E20BBE008B981
:10F8100018209BE0012821D111681820B3E008B915
:10F82000192093E0012819D111681920ABE008B91B
:10F830005C208BE0012811D111685C20A3E008B99D
:10F840005F2083E0012809D111685F209BE038B96F
:10F850000620FFF717FDC0F307402860002070BDA9
:10F860000128FBD10620FFF70DFD2B681B0420F4B7
:10F870007F0103F47F031943062084E00128EDD1C2
:10F88000166836B110F0F2FE28600028E6D120207C
:10F8900070BD0720FFF7F6FC20F48001072072E01E
:10F8A00000287FF437AE652050E00028D6D107202D
:10F8B000FFF7E8FCC0F38150431E58425841CCE7A3
:10F8C00008B9522042E00128C8D1116852205AE0FC
:10F8D00020B9304B1B6893F8903159E70128BDD10E
:10F8E0002C4B11681B68D3F8903101F00F0123F005
:10F8F000FF0313E030B9274B1B68D3F89031C3F3F3
:10F90000032345E70128A9D1224B1B68D3F89011A6
:10F9100013681B0221F4706103F4706319436320C0
:10F9200031E020B91B4B1B6893F8923130E7012876
:10F9300094D1184B1B68D3F8901113681B0421F461
:10F940007F0103F47F03E9E718B95020FFF79AFC21
:10F9500083E7012882D11168502014E018B90D4BBB
:10F960001B68DB6914E701287FF478AF1168532026
:10F9700009E008B91520E9E701287FF46FAF1368A3
:10F98000054915205943FFF73BFC67E7042070BD8C
:10F99000102070BD8846FF1F0071020007B501925C
:10F9A00029B9014601AA0120FFF7E5FC00E0082083
:10F9B00003B05DF804FB0B4611B901461846DAE4C2
:10F9C0000820704710B50C46C8B92020FFF75AFC34
:10F9D00020F004012020FFF713FC84EAE472094BB5
:10F9E000A2EBE4729A4204DD074A12EA240438BF0B
:10F9F0001C4621022420FFF703FC002010BD082034
:10FA000010BD00BF00127A0000EE85FF0021D9E78B
:10FA10004942D7E7D6E7314B2DE9F041DE6A9A6AD1
:10FA2000350245EA12651402C6B293F83020D86B4D
:10FA3000264300279C6B2F430132050E000240EA4B
:10FA40001460D2B224029C63C3E90A6783F83020B1
:10FA5000D8631C4600293DD0042A03D939466D20BD
:10FA6000FFF7CEFBA16ADFF874806C20FFF7C8FBBC
:10FA700001200CF0DFFCA16A6C20FFF7C1FB002322
:10FA80000022C4E90E2394F83030042B09D96F20EA
:10FA9000FFF7F8FBD8E90E23002632430343C8E9F9
:10FAA0000E236E20FFF7EEFBD4E90E6794F83020AA
:10FAB0000346C2F10802D20047EAE371304314F072
:10FAC000CDFB00230022C4E90E01C4E90A23002370
:10FAD00084F830302846BDE8F08100BF7016FF1F63
:10FAE00070B54B4E4B484C4C10F042FDF5686B68BE
:10FAF00003F1E402226203F58272E26103F55172BE
:10FB0000A26103F55972626103F56172226103F526
:10FB1000697203F57970E26003F5717203F20443D0
:10FB200023602B68A260DB68606098472B68A0693F
:10FB3000DB6898472B686069DB6898472B68206909
:10FB4000DB6898472B68E068DB6898472B68A068FB
:10FB5000DB6898472B6860685B6998472B68A069E9
:10FB60005B6998472B6860695B6998472B682069D7
:10FB70005B6998472B68E0685B6998472B68A068C9
:10FB80005B6998472B68206A1B6998472B68E06976
:10FB90001B6998472B6820681B69204C9847204BAD
:10FBA00032691A606B6803F5317353601D4B6269EB
:10FBB0001A6001212020FFF723FB6369002159709F
:10FBC0001949C3F80412012218491A70C3F808121F
:10FBD000174B6366174B2362174BE361174BA36107
:10FBE000174B6362174BA363174B6363174BA362F7
:10FBF000174BE362174BA364174B6364174B6365A2
:10FC0000174B2365174BE3652274174BA36570BD33
:10FC10000C550200A043FF1F7016FF1FC82EFF1FC8
:10FC20008446FF1F8846FF1F51F1000019F10000B4
:10FC300017FA0000C5F9000015FA000011FA0000DB
:10FC40000DFA0000B7F900009DF9000035F300003F
:10FC50005DF3000081F2000029F300001BF20000B8
:10FC600035F00000BDEF0000C9EF00000020704734
:10FC700001207047014B00225A607047C82EFF1FB9
:10FC800010B50C460DF056F8206010BD0DF07EB892
:10FC900038B50D46044620B910F01DFE28602046F8
:10FCA00038BD082038BDF0B589B004AC374D0746E3
:10FCB00010220021204615F05FFA2B68FB1A092B51
:10FCC00006D9AA682F60642353436B600023AB609E
:10FCD000AB680133AB602E4BA3F1080633F8081C68
:10FCE000727A0291B11D0191B188009100203946CC
:10FCF00010F00CFF0FF044FD20B100221146104619
:10FD00000FF0CAFD0FF036FD00283CD00FF0B2FD19
:10FD1000032838D8DFE800F0120A021D002010F096
:10FD2000FDFD0490002010F000FE10E0002010F017
:10FD3000C6FD0490002010F0CEFD08E0718900207F
:10FD400010F055FD71890490002010F05AFD0590C7
:10FD500015E0EB685BB1012B11D164230493C82338
:10FD600005934FF4967306934FF4C87306E00A2385
:10FD70000493142305931E2306932823079394E8E2
:10FD80000F000FF017FD09B0F0BD00BFBC16FF1F3C
:10FD90009446FF1F10B5044620B9096810F0ADFD68
:10FDA000204610BD082010BD10B5044618B910F04B
:10FDB00097FD204610BD082010BD10B5044618B9A7
:10FDC00010F070FD204610BD082010BD0021F4E7A2
:10FDD0004942F2E7F1E7022804BF0C4B93F8D00048
:10FDE00020B90B4BDB681B689B690AE001280BD12B
:10FDF000064B93F8D030012B06D1054BDB681B680E
:10FE00005B69044A10681847704700BFC82EFF1F7F
:10FE10000C550200E42FFF1F10B50020FFF7DBFF99
:10FE2000044B054ADB6810681B68BDE810409B69FD
:10FE3000184700BF0C550200E42FFF1F043A38B5E5
:10FE400004461D460846FB2A00F28E87DFE812F0C2
:10FE5000FC008C078C078C078C078C078C070C0127
:10FE600013018C0717018C078C078C078C078C07F4
:10FE70008C078C078C078C078C078C078C078C07EA
:10FE80008C078C078C078C078C078C078C078C07DA
:10FE90008C078C078C078C078C078C078C078C07CA
:10FEA0008C078C078C078C078C078C071B012E0195
:10FEB0008C07410154018C078C078C078C078C0739
:10FEC0008C078C078C078C078C078C078C078C079A
:10FED0008C078C078C078C078C078C078C078C078A
:10FEE0008C078C078C078C078C078C078C078C077A
:10FEF0008C078C078C078C078C078C078C078C076A
:10FF00008C078C078C078C078C078C078C078C0759
:10FF100067017801850192019F01AC01B901C60119
:10FF2000D301E001ED01FA010802160224023202B7
:10FF300040024B0256028C0761026C027702820279
:10FF40008D029C02AB02BA02C4028C078C078C079C
:10FF5000CE02D702E002EB02F6028C078C078C0778
:10FF6000FF02080311038C078C078C078C078C0792
:10FF70008C078C071C03270332033D038C078C0777
:10FF80008C078C078C078C07480353035E036903B7
:10FF900074038C078C078C078C078C077F038A03FC
:10FFA0009D03B003B903C803D303DF03EA03F203DD
:10FFB00000040D041A042704340441044E045B04B5
:10FFC0008C07680476048C049904A704B404C10463
:10FFD000CE04DB04E804F704060515052405330503
:10FFE0004205540563057205810590059F05AE0520
:10FFF000BD05CC05DB05EA05F905080616068C07E4
:020000021000EC
:100000008C078C078C078C078C078C078C078C0758
:100010008C078C07240633064206510660066F06DD
:100020007E068D069C06AA06B806C606D406E2061B
:10003000F006FE060C0719072607330740074D0791
:100040005E0771077A0784072CB960200CF072FEF6
:100050002860204638BD012C40F088862968602041
:100060000CF094FE002038BD002C40F08186002466
:100070002C60204638BD002CF9D0002038BD002C63
:10008000F5D0002038BD3CB9214608200CF0DDFE3B
:1000900000B22860204638BD012C40F06B862A88CB
:1000A000002108200CF003FF002038BD3CB9214698
:1000B00009200CF0CAFE00B22860204638BD012C91
:1000C00040F05A862A88002109200CF0F0FE00201A
:1000D00038BD3CB9012108200CF0B7FE00B2286001
:1000E000204638BD012C40F049862A882146082048
:1000F0000CF0DDFE002038BD3CB9012109200CF0D8
:10010000A4FE00B22860204638BD012C40F038869D
:100110002A88214609200CF0CAFE002038BD54B9B7
:10012000012103200CF032FE214602200CF08DFE4E
:100130002860204638BD012C14BF0020042038BDA3
:10014000002CF8D1012103200CF020FE0121022017
:100150000CF07BFE2860204638BD002CEBD102213C
:1001600003200CF013FE214602200CF06EFE2860E6
:10017000204638BD002CDED1214603200CF006FEBF
:10018000214602200CF061FE2860204638BD002C7C
:10019000D1D1214603200CF0F9FD012102200CF001
:1001A00054FE2860204638BD002CC4D103210846E7
:1001B0000CF0ECFD214602200CF047FE28602046A2
:1001C00038BD002CB7D1042103200CF0DFFD2146FF
:1001D00002200CF03AFE2860204638BD002CAAD13F
:1001E000042103200CF0D2FD012102200CF02DFE91
:1001F0002860204638BD002C9DD1052103200CF03D
:10020000C5FD214602200CF020FE2860204638BDA6
:10021000002C90D1052103200CF0B8FD0121022013
:100220000CF013FE2860204638BD002C83D1062137
:1002300003200CF0ABFD214602200CF006FE2860E6
:10024000204638BD002C7FF476AF072103200CF048
:100250009DFD214602200CF0F8FD2860204638BDA7
:10026000002C7FF468AF072103200CF08FFD0121E3
:1002700002200CF0EAFD2860204638BD002C7FF4F7
:100280005AAF082103200CF081FD214602200CF01A
:10029000DCFD2860204638BD002C7FF44CAF0821DF
:1002A00003200CF073FD012102200CF0CEFD28602C
:1002B000204638BD002C7FF43EAF092103200CF00E
:1002C00065FD214602200CF0C0FD2860204638BDA7
:1002D000002C7FF430AF214612200CF0B6FD00B2A6
:1002E0002860204638BD002C7FF425AF0121122064
:1002F0000CF0ABFD00B22860204638BD002C7FF426
:100300001AAF214613200CF0A0FD00B22860204651
:1003100038BD002C7FF40FAF214615200CF095FD61
:1003200000B22860204638BD002C7FF404AF0121C4
:1003300015200CF08AFD00B22860204638BD002C44
:100340007FF4F9AE214616200CF07FFD00B2286044
:10035000204638BD002C7FF4EEAE012116200CF0B3
:1003600074FD00B22860204638BD002C7FF4E3AE57
:100370000A2103200CF00AFD214602200CF065FD45
:1003800000B22860204638BD002C7FF4D4AE0A218C
:1003900003200CF0FBFC012102200CF056FD00B202
:1003A0002860204638BD002C7FF4C5AE0B21032009
:1003B0000CF0ECFC214602200CF047FD00B2286056
:1003C000204638BD002C7FF4B6AE214606200CF046
:1003D0003CFD2860204638BD002C7FF4ACAE0121E6
:1003E00006200CF032FD2860204638BD002C7FF43A
:1003F000A2AE41200CF09EFC2860204638BD002CA7
:100400007FF499AE42200CF095FC2860204638BD60
:10041000002C7FF490AE012146200CF016FD00B2B6
:100420002860204638BD002C7FF485AE214646204A
:100430000CF00BFD00B22860204638BD002C7FF484
:100440007AAE47200CF076FC2860204638BD002CA0
:100450007FF471AE21200CF06DFC2860204638BD81
:10046000002C7FF468AE22200CF064FC286020464B
:1004700038BD002C7FF45FAE214623200CF0E5FC54
:1004800000B22860204638BD002C7FF454AE2720EF
:100490000CF050FC20F07F402860204638BD002C36
:1004A0007FF449AE28200CF045FC20F07F40286006
:1004B000204638BD002C7FF43EAE01212A200CF0EE
:1004C000C4FC00B22860204638BD002C7FF433AE57
:1004D00021462A200CF0B9FC00B22860204638BD25
:1004E000002C7FF428AE214639200CF0AEFC00B27F
:1004F0002860204638BD002C7FF41DAE0121392034
:100500000CF0A3FC00B22860204638BD002C7FF41C
:1005100012AE21463D200CF098FC00B22860204627
:1005200038BD002C7FF407AE21463F200CF08DFC37
:1005300000B22860204638BD002C7FF4FCAD214677
:100540003A200CF082FC00B22860204638BD002C16
:100550007FF4F1AD214653200CF077FC00B2286007
:10056000204638BD3CB9012164200CF06EFC00B27D
:100570002860204638BD012C40F004842A8821469A
:1005800064200CF094FC002038BD3CB92146642066
:100590000CF05BFC00B22860204638BD012C40F016
:1005A000F3832A88002164200CF081FC002038BDF0
:1005B000002C7FF4C0AD66200CF0BCFB2860204608
:1005C00038BD2CB968200CF0B5FB2860204638BD3A
:1005D000012C40F0DB83296810F082F9002038BD3F
:1005E000002C7FF4A8AD012169200CF02EFC00B294
:1005F0002860204638BD002C7FF49DADBD4B03EB39
:100600000113598910F0FDF82860204638BD002CF0
:100610007FF491AD214669200CF017FC00B22860F0
:10062000204638BD002C7FF486AD10F054F92860C8
:10063000204638BD24B910F078F92860204638BD2E
:10064000012C40F0A583296810F06BF9002038BD1B
:10065000002C7FF470AD21466D200CF097FB6C20D0
:100660000CF068FB2860204638BD002C7FF463AD99
:1006700001216D200CF08AFB6C200CF05BFB2860E4
:10068000204638BD002C7FF456AD02216D200CF0C1
:100690007DFB6C200CF04EFB2860204638BD002C02
:1006A0007FF449AD03216D200CF070FB6C200CF041
:1006B00041FB2860204638BD002C7FF43CAD04216E
:1006C0006D200CF063FB6C200CF034FB286020469E
:1006D00038BD002C7FF42FAD05216D200CF056FBAA
:1006E0006C200CF027FB2860204638BD002C7FF4DE
:1006F00022AD06216D200CF049FB6C200CF01AFB9A
:100700002860204638BD002C7FF415AD07216D20F0
:100710000CF03CFB6C200CF00DFB2860204638BD33
:1007200024B910F03DF82860204638BD012C40F077
:100730003183296810F026F8002038BD44B96D4B8C
:1007400003EB0113598910F052F82860204638BD98
:10075000012C40F02183674B2A6803EB0113598970
:1007600010F033F8002038BD002C7FF4E4AC0121F8
:100770006F200CF00BFB6E200CF0DCFA286020469A
:1007800038BD24B910F09BF82860204638BD012CF4
:1007900040F00483296810F085F8002038BD002C53
:1007A0007FF4C9AC03216F200CF0F0FA6E200CF03E
:1007B000C1FA2860204638BD002C7FF4BCAC04216F
:1007C0006F200CF0E3FA6E200CF0B4FA286020469B
:1007D00038BD002C7FF4AFAC05216F200CF0D6FAA9
:1007E0006E200CF0A7FA2860204638BD002C7FF45C
:1007F000A2AC06216F200CF0C9FA6E200CF09AFA18
:100800002860204638BD002C7FF495AC07216F206E
:100810000CF0BCFA6E200CF08DFA2860204638BD32
:10082000002C7FF488AC08216F200CF0AFFA214631
:100830006E200CF00AFB00B22860204638BD002C68
:100840007FF479AC08216F200CF0A0FA01216E2012
:100850000CF0FBFA00B22860204638BD002C7FF473
:100860006AAC09216F200CF091FA21466E200CF041
:10087000ECFA00B22860204638BD002C7FF45BAC57
:100880000A216F200CF082FA21466E200CF0DDFA6E
:1008900000B22860204638BD002C7FF44CAC0A2101
:1008A0006F200CF073FA01216E200CF0CEFA00B22A
:1008B0002860204638BD002C7FF43DAC0B216F2012
:1008C0000CF064FA21466E200CF0BFFA00B22860EA
:1008D000204638BD002C7FF42EAC0B216F200CF08D
:1008E00055FA01216E200CF0B0FA00B228602046C3
:1008F00038BD00BF8C46FF1F002C7FF41CAC0C21C0
:100900006F200CF043FA21466E200CF09EFA00B2E4
:100910002860204638BD002C7FF40DAC0C216F20E0
:100920000CF034FA01216E200CF08FFA00B228602E
:10093000204638BD002C7FF4FEAB0D216F200CF05B
:1009400025FA21466E200CF080FA00B2286020467D
:1009500038BD002C7FF4EFAB0D216F200CF016FAA0
:1009600001216E200CF071FA00B22860204638BDDB
:10097000002C7FF4E0AB0E216F200CF007FA21462B
:100980006E200CF062FA00B22860204638BD002CC0
:100990007FF4D1AB0E216F200CF0F8F901216E200D
:1009A0000CF053FA00B22860204638BD002C7FF4CA
:1009B000C2AB0F216F200CF0E9F921466E200CF03C
:1009C00044FA00B22860204638BD002C7FF4B3AB57
:1009D0000F216F200CF0DAF901216E200CF035FAAE
:1009E00000B22860204638BD002C7FF4A4AB102153
:1009F0006F200CF0CBF921466E200CF026FA00B2E5
:100A00002860204638BD002C7FF495AB11216F2063
:100A10000CF0BCF921466E200CF017FA00B22860E9
:100A2000204638BD002C7FF486AB11216F200CF0DE
:100A3000ADF901216E200CF008FA00B228602046C2
:100A400038BD002C7FF477AB12216F200CF09EF99B
:100A500021466E200CF0F9F900B22860204638BD1E
:100A6000002C7FF468AB13216F200CF08FF9214626
:100A70006E200CF0EAF92860204638BD002C7FF487
:100A80005AAB13216F200CF081F901216E200CF07C
:100A9000DCF92860204638BD002C7FF44CABC02127
:100AA0006F200CF073F921466E200CF0CEF900B2E5
:100AB0002860204638BD002C7FF43DABC0216F205C
:100AC0000CF064F901216E200CF0BFF900B228602F
:100AD000204638BD002C7FF42EABC1216F200CF0D6
:100AE00055F921466E200CF0B0F900B2286020467E
:100AF00038BD002C7FF41FABC1216F200CF046F9EC
:100B000001216E200CF0A1F900B22860204638BD0A
:100B1000002C7FF410ABC2216F200CF037F9214676
:100B20006E200CF092F900B22860204638BD002CEF
:100B30007FF401ABC2216F200CF028F901216E2057
:100B40000CF083F900B22860204638BD002C7FF4F9
:100B5000F2AAC3216F200CF019F921466E200CF087
:100B600074F900B22860204638BD002C7FF4E3AA57
:100B7000C3216F200CF00AF901216E200CF065F9F9
:100B800000B22860204638BD002C7FF4D4AAC421CE
:100B90006F200CF0FBF821466E200CF056F928600F
:100BA000204638BD002C7FF4C6AAC4216F200CF06B
:100BB000EDF801216E200CF048F92860204638BD80
:100BC000002C7FF4B8AAC5216F200CF0DFF8214675
:100BD0006E200CF03AF92860204638BD002C7FF4D6
:100BE000AAAAC5216F200CF0D1F801216E200CF0CB
:100BF0002CF92860204638BD002C7FF49CAAC62121
:100C00006F200CF0C3F821466E200CF01EF928600E
:100C1000204638BD002C7FF48EAAC6216F200CF030
:100C2000B5F801216E200CF010F92860204638BD7F
:100C3000002C7FF480AAC7216F200CF0A7F8214672
:100C40006E200CF002F92860204638BD002C7FF49D
:100C500072AAC7216F200CF099F801216E200CF0C8
:100C6000F4F82860204638BD002C7FF464AAC8211F
:100C70006F200CF08BF86E200CF05CF8286020469A
:100C800038BD002C7FF457AAC9216F200CF07EF8E4
:100C90006E200CF04FF82860204638BD002C7FF401
:100CA0004AAACA216F200CF071F86E200CF042F8AD
:100CB0002860204638BD002C7FF43DAACB216F2050
:100CC0000CF064F86E200CF035F82860204638BD32
:100CD00024B9374BDB682B60204638BD012C5FD12F
:100CE000334B2A68DA60002038BD34B9314A02EB50
:100CF000011043892B60204638BD012C52D12D4A6A
:100D00002B6802EB01104381002038BD34B9294A19
:100D100002EB0110437A2B60204638BD012C43D1F1
:100D2000254A287802EB0112511C0FF0F9FE002031
:100D300038BD002C3AD11F4A02EB0110037A2B6018
:100D4000204638BD002C7FF4F6A91A4A02EB0110A8
:100D5000C3882B60204638BD002C7FF4ECA9144BCF
:100D60005B682B60204638BD042038BD002038BDAC
:100D7000002038BD002038BD002038BD002038BD1F
:100D8000002038BD002038BD002038BD002038BD0F
:100D9000002038BD002038BD002038BD002038BDFF
:100DA000002038BD002038BD002038BD002038BDEF
:100DB000BC16FF1F8C46FF1F9446FF1F10B413463E
:100DC0000446084619B9224610BCFFF737B8082078
:100DD00010BC70470120704707B5019229B902463F
:100DE00001AB0120FFF72AF800E0082003B05DF80E
:100DF00004FB08460BF09EBF084611460BF0C6BF29
:100E0000084611460CF021B8084611461A460CF067
:100E10004EB838B5274B284DDC68606823686430CD
:100E20002860DB689847236828685B699847234BEC
:100E300023495A690A602349C2F804122249C2F8B8
:100E40000812002111705170204A1A62204ADA619A
:100E5000204A9A61204A5A62204ADA64204A9A63F8
:100E6000204A5A63204A9A62204ADA62204A9A64E7
:100E7000204A5A64204A5A65204A1A65204A1A664E
:100E8000204ADA65204A9A653222DA60012040F26F
:100E90008A229A6018741D4B4FF47A729A8041F23C
:100EA00070721A6059724FF480725A81BDE83840EE
:100EB000FEF791BF0C550200E42FFF1FC82EFF1F45
:100EC0009C46FF1FD50D010071FC0000BBFD00001A
:100ED000D5FD0000D1FD0000CDFD000091FC00001B
:100EE000BD0D0100D90D0100A9FD000095FD000018
:100EF0008DFC000081FC0000A7FC00006DFC0000E0
:100F0000D7FD000075FC000019FE00008C46FF1F95
:100F10000020704701207047014B00225A60704743
:100F2000C82EFF1F10B50C460BF004FF206010BD4B
:100F30000BF02CBF38B50D46044620B90FF03CFF2E
:100F40002860204638BD082038BD30B589B004ACD3
:100F5000054610220021204614F00EF9384B1A687D
:100F6000AA1A092A06D999681D6064224A435A6060
:100F700000229A609A6801329A60324B33F8060C6C
:100F80005A780290981E019033F8041C00910020BA
:100F9000294610F02DF80EF0F3FB20B10022114687
:100FA00010460EF079FC0EF0E5FB002845D00EF05F
:100FB00061FC032841D8DFE800F0130A0229002071
:100FC0000FF01DFF049000200FF020FF06E000202E
:100FD0000FF0EFFE049000200FF0EEFE059028E0E9
:100FE00000216F200BF0D2FE6E200BF0A3FE01213A
:100FF000049069200BF029FF0021054669200BF0C1
:1010000024FF00B200FA85F5059512E076200BF07A
:1010100091FE6423C0F30222C0F302505A434343BB
:10102000A3F52F730593084B0693A3F5FA63049277
:10103000079394E80F000EF0BDFB09B030BD00BF70
:10104000D816FF1F9246FF1FF0D8FFFF10B50446C9
:1010500020B909680FF0C2FE204610BD082010BD5F
:1010600010B5044618B90FF0ACFE204610BD08209C
:1010700010BD10B5044618B90FF08EFE204610BD05
:10108000082010BD0021F4E74942F2E7F1E7022809
:1010900004BF0C4B93F8D00020B90B4BDB681B68E6
:1010A0009B690AE001280BD1064B93F8D030012B45
:1010B00006D1054BDB681B685B69044A106818475A
:1010C000704700BFC82EFF1F0C550200E42FFF1F02
:1010D00010B50020FFF7DBFF044B054ADB68106802
:1010E0001B68BDE810409B69184700BF0C55020003
:1010F000E42FFF1F043A38B504461D460846FB2A74
:1011000001F21D80DFE812F0FC001B081B081B0821
:101110001B081B081B080C0113011B0817011B08E7
:101120001B081B081B081B081B081B081B081B08A7
:101130001B081B081B081B081B081B081B081B0897
:101140001B081B081B081B081B081B081B081B0887
:101150001B081B081B081B081B081B081B081B0877
:101160001B081B081B012D011B083F0152011B0816
:101170001B081B081B081B081B081B081B081B0857
:101180001B081B081B081B081B081B081B081B0847
:101190001B081B081B081B081B081B081B081B0837
:1011A0001B081B081B081B081B081B081B081B0827
:1011B0001B081B081B081B081B081B081B081B0817
:1011C0001B081B081B081B086501760183011B080F
:1011D0001B081B081B081B081B081B081B08900189
:1011E0009D01AA011B081B08B701C101CB011B0807
:1011F000D501DF01E9011B08F30101021B080F0201
:1012000019021B081B081B0823022C02350240028E
:101210004B021B081B081B0854025D0266021B08D8
:101220001B081B081B081B081B081B0871027C02FB
:10123000870292029D02B502CD02E80203031E035B
:10124000380343034E03590364031B081B081B08A0
:101250001B081B086F037A038D03A003A903B203C5
:10126000BD03CA03D503DD03EC03F903060413042D
:1012700020042D043A0447041B08540462047A0431
:1012800087049404A104AE04BB04C804D504E40498
:10129000F3040205110520052F0540054F055E05E5
:1012A0006D057C058B059A05A905B805C705D6050A
:1012B000E505F40502061B081006280640065B0635
:1012C00076069106AC061B081B081B08B906C80663
:1012D000D706E606F50604071307220731073F077E
:1012E0004D075B076907770785079307A107AE07D7
:1012F000BB07C8071B08D507E807FE07080813083F
:101300002CB960200BF016FD2860204638BD012C5A
:1013100040F01787296860200BF038FD002038BDA9
:10132000002C40F0108700242C60204638BD002C93
:10133000F9D0002038BD002CF5D0002038BD34B9DC
:10134000214608200BF081FD2860204638BD012C85
:1013500040F0FB862A88002108200BF0A8FD002021
:1013600038BD34B9214609200BF06FFD28602046B6
:1013700038BD012C40F0EB862A88002109200BF0B3
:1013800096FD002038BD3CB9012108200BF05DFD21
:1013900000B22860204638BD012C40F0DA862A8849
:1013A000214608200BF083FD002038BD3CB9012107
:1013B00009200BF04AFD00B22860204638BD012C00
:1013C00040F0C9862A88214609200BF070FD0020D4
:1013D00038BD54B9012103200BF0D8FC214602206E
:1013E0000BF033FD2860204638BD012C14BF0020CF
:1013F000042038BD002CF8D1012103200BF0C6FCDD
:10140000012102200BF021FD2860204638BD002C70
:10141000EBD1022103200BF0B9FC214602200BF096
:1014200014FD2860204638BD002CDED102210320A7
:101430000BF0ACFC012102200BF007FD28602046D8
:1014400038BD002CD1D1032108460BF09FFC0121AF
:1014500002200BF0FAFC2860204638BD002CC4D1D5
:10146000032108460BF092FC214602200BF0EDFC14
:101470002860204638BD002CB7D1214612200BF041
:10148000E4FC00B22860204638BD002CADD101211B
:1014900012200BF0DAFC00B22860204638BD002C88
:1014A000A3D1214613200BF0D0FC00B228602046C7
:1014B00038BD002C99D1214615200BF0C6FC00B296
:1014C0002860204638BD002C8FD1012115200BF05B
:1014D000BCFC00B22860204638BD002C85D12146D6
:1014E00016200BF0B2FC00B22860204638BD002C5C
:1014F0007FF47BAF214603200BF048FC21460220FD
:101500000BF0A3FC2860204638BD002C7FF46DAFA3
:10151000214603200BF03AFC012102200BF095FC40
:101520002860204638BD002C7FF45FAF21460B2099
:101530000BF08BFC2860204638BD002C7FF455AFA3
:1015400001210B200BF081FC2860204638BD002CC7
:101550007FF44BAF41200BF0EDFB2860204638BDF7
:10156000002C7FF442AF42200BF0E4FB28602046C1
:1015700038BD002C7FF439AF012146200BF065FC0B
:1015800000B22860204638BD002C7FF42EAF2146E3
:1015900046200BF05AFC00B22860204638BD002CD3
:1015A0007FF423AF47200BF0C5FB2860204638BDF1
:1015B000002C7FF41AAF21200BF0BCFB28602046E2
:1015C00038BD002C7FF411AF22200BF0B3FB286054
:1015D000204638BD002C7FF408AF214623200BF0B5
:1015E00034FC00B22860204638BD002C7FF4FDAEEC
:1015F00027200BF09FFB20F07F402860204638BD5D
:10160000002C7FF4F2AE28200BF094FB20F07F40FA
:101610002860204638BD002C7FF4E7AE01212A2047
:101620000BF013FC00B22860204638BD002C7FF47C
:10163000DCAE21462A200BF008FC00B228602046D0
:1016400038BD4CB9D4216F200BF0A0FB6E200BF0FD
:1016500071FB2860204638BD012C40F07E85D421E6
:101660006F200BF093FB29686E200BF08FFB00209E
:1016700038BD4CB9D5216F200BF088FB6E200BF0E4
:1016800059FB2860204638BD012C40F06885D521E3
:101690006F200BF07BFB29686E200BF077FB00209E
:1016A00038BD5CB9D6216F200BF070FB21466E204F
:1016B0000BF0CBFB00B22860204638BD012C40F077
:1016C0005085D6216F200BF061FB2A8800216E2007
:1016D0000BF0EDFB002038BD5CB9D6216F200BF07C
:1016E00055FB01216E200BF0B0FB00B228602046B4
:1016F00038BD012C40F03785D6216F200BF046FB1A
:101700002A8821466E200BF0D2FB002038BD5CB940
:10171000D7216F200BF03AFB21466E200BF095FB92
:1017200000B22860204638BD012C40F01E85D7212C
:101730006F200BF02BFB2A8800216E200BF0B7FBEB
:10174000002038BD54B9D7216F200BF01FFB0121B9
:101750006E200BF07AFB2860204638BD012C40F04B
:101760000685D7216F200BF011FB2A8821466E20B9
:101770000BF09DFB002038BD002C7FF436AE2146D7
:1017800039200BF062FB00B22860204638BD002CE7
:101790007FF42BAE012139200BF057FB00B22860FB
:1017A000204638BD002C7FF420AE21463D200BF0B2
:1017B0004CFB00B22860204638BD002C7FF415AEEB
:1017C00021463F200BF041FB00B22860204638BD87
:1017D000002C7FF40AAE21463A200BF036FB00B213
:1017E0002860204638BD002C7FF4FFAD21465320F1
:1017F0000BF02BFB00B22860204638BD3CB901211C
:1018000064200BF022FB00B22860204638BD012C7A
:1018100040F0AF842A88214664200BF048FB00206A
:1018200038BD3CB9214664200BF00FFB00B22860A4
:10183000204638BD012C40F09E842A880021642077
:101840000BF035FB002038BD002C7FF4CEAD6620B8
:101850000BF070FA2860204638BD002C7FF4C5AD2F
:1018600068200BF067FA2860204638BD002C7FF412
:10187000BCAD012169200BF0E8FA00B228602046D7
:1018800038BD002C7FF4B1ADBE4A0C2303FB01230D
:1018900019890FF030FA2860204638BD002C7FF4FB
:1018A000A4AD214669200BF0D0FA00B22860204692
:1018B00038BD002C7FF499AD0FF07EFA28602046E9
:1018C00038BD24B90FF0A2FA2860204638BD012C9B
:1018D00040F0538429686B200BF058FA002038BD83
:1018E000002C7FF482AD21466D200BF04FFA6C2066
:1018F0000BF020FA2860204638BD002C7FF475AD2F
:1019000001216D200BF042FA6C200BF013FA2860D5
:10191000204638BD002C7FF468AD02216D200BF00D
:1019200035FA6C200BF006FA2860204638BD002CF2
:101930007FF45BAD03216D200BF028FA6C200BF0D7
:10194000F9F92860204638BD002C7FF44EAD042103
:101950006D200BF01BFA6C200BF0ECF92860204690
:1019600038BD002C7FF441AD05216D200BF00EFA3F
:101970006C200BF0DFF92860204638BD002C7FF486
:1019800034AD06216D200BF001FA6C200BF0D2F97A
:101990002860204638BD002C7FF427AD07216D203C
:1019A0000BF0F4F96C200BF0C5F92860204638BD27
:1019B00024B90FF06FF92860204638BD012C40F0A3
:1019C000DE8329680FF058F9002038BD4CB96D4A04
:1019D0000C2303FB012319890FF083F928602046AB
:1019E00038BD012C40F0CD83664A0C2303FB012354
:1019F0002A6819890FF063F9002038BD002C7FF4A4
:101A0000F4AC01216F200BF0C1F96E200BF092F9BC
:101A10002860204638BD002C7FF4E7AC02216F20FF
:101A20000BF0B4F96E200BF085F92860204638BD24
:101A3000002C7FF4DAAC03216F200BF0A7F96E20A5
:101A40000BF078F92860204638BD002C7FF4CDAC2F
:101A500004216F200BF09AF96E200BF06BF92860CF
:101A6000204638BD002C7FF4C0AC05216F200BF060
:101A70008DF96E200BF05EF92860204638BD002CF1
:101A80007FF4B3AC06216F200BF080F96E200BF0D1
:101A900051F92860204638BD002C7FF4A6AC072100
:101AA0006F200BF073F96E200BF044F9286020468C
:101AB00038BD002C7FF499AC08216F200BF066F93B
:101AC00021466E200BF0C1F900B22860204638BDD7
:101AD000002C7FF48AAC08216F200BF057F901210C
:101AE0006E200BF0B2F900B22860204638BD002C01
:101AF0007FF47BAC09216F200BF048F921466E2062
:101B00000BF0A3F900B22860204638BD002C7FF40A
:101B10006CAC0A216F200BF039F921466E200BF0D6
:101B200094F900B22860204638BD002C7FF45DACEB
:101B30000A216F200BF02AF901216E200BF085F9A4
:101B400000B22860204638BD002C7FF44EAC0B213B
:101B50006F200BF01BF921466E200BF076F900B2D6
:101B60002860204638BD002C7FF43FAC0B216F204D
:101B70000BF00CF901216E200BF067F900B2286020
:101B8000204638BD8C46FF1F002C7FF42EAC0C2164
:101B90006F200BF0FBF821466E200BF056F900B2D7
:101BA0002860204638BD002C7FF41FAC0C216F202C
:101BB0000BF0ECF801216E200BF047F900B2286021
:101BC000204638BD002C7FF410AC0D216F200BF0A7
:101BD000DDF821466E200BF038F900B2286020466F
:101BE00038BD002C7FF401AC0D216F200BF0CEF836
:101BF00001216E200BF029F900B22860204638BD83
:101C0000002C7FF4F2AB0E216F200BF0BFF82146C1
:101C10006E200BF01AF900B22860204638BD002C67
:101C20007FF4E3AB0E216F200BF0B0F801216E20A2
:101C30000BF00BF900B22860204638BD002C7FF471
:101C4000D4AB0F216F200BF0A1F821466E200BF0D2
:101C5000FCF800B22860204638BD002C7FF4C5ABEC
:101C60000F216F200BF092F801216E200BF0EDF8A0
:101C700000B22860204638BD002C7FF4B6AB10219E
:101C80006F200BF083F821466E200BF0DEF800B2D7
:101C90002860204638BD002C7FF4A7AB11216F20AF
:101CA0000BF074F821466E200BF0CFF800B22860DC
:101CB000204638BD002C7FF498AB11216F200BF02B
:101CC00065F801216E200BF0C0F800B228602046B4
:101CD00038BD002C7FF489AB12216F200BF056F831
:101CE00021466E200BF0B1F800B22860204638BDC6
:101CF000002C7FF47AAB13216F200BF047F82146BC
:101D00006E200BF0A2F82860204638BD002C7FF42E
:101D10006CAB13216F200BF039F801216E200BF012
:101D200094F82860204638BD4CB9D0216F200BF0C4
:101D30002DF86E200AF0FEFF2860204638BD012CE9
:101D400040F02182D0216F200BF020F829686E200E
:101D50000BF01CF8002038BD4CB9D1216F200BF0DE
:101D600015F86E200AF0E6FF2860204638BD012CE9
:101D700040F00B82D1216F200BF008F829686E200B
:101D80000BF004F8002038BD5CB9D2216F200AF0B6
:101D9000FDFF21466E200BF058F800B22860204667
:101DA00038BD012C40F0F381D2216F200AF0EEFF04
:101DB0002A8800216E200BF07AF8002038BD5CB92B
:101DC000D2216F200AF0E2FF01216E200BF03DF8D6
:101DD00000B22860204638BD012C40F0DA81D221C3
:101DE0006F200AF0D3FF2A8821466E200BF05FF89F
:101DF000002038BD5CB9D3216F200AF0C7FF21460F
:101E00006E200BF022F800B22860204638BD012C6D
:101E100040F0C181D3216F200AF0B8FF2A88002149
:101E20006E200BF044F8002038BD5CB9D3216F2040
:101E30000AF0ACFF01216E200BF007F800B2286019
:101E4000204638BD012C40F0A881D3216F200AF034
:101E50009DFF2A8821466E200BF029F8002038BD0E
:101E6000002C7FF4C2AA1D216F200AF08FFF6E2084
:101E70000AF060FF2860204638BD002C7FF4B5AA28
:101E8000C0216F200AF082FF21466E200AF0DDFF9C
:101E900000B22860204638BD002C7FF4A6AAC021DD
:101EA0006F200AF073FF01216E200AF0CEFF00B20E
:101EB0002860204638BD002C7FF497AAC1216F20EE
:101EC0000AF064FF21466E200AF0BFFF00B22860CE
:101ED000204638BD002C7FF488AAC1216F200AF06B
:101EE00055FF01216E200AF0B0FF00B228602046A5
:101EF00038BD002C7FF479AAC2216F200AF046FF7A
:101F000021466E200AF0A1FF00B22860204638BDAD
:101F1000002C7FF46AAAC2216F200AF037FF01214A
:101F20006E200AF092FF00B22860204638BD002CD7
:101F30007FF45BAAC3216F200AF028FF21466E20A0
:101F40000AF083FF00B22860204638BD002C7FF4E1
:101F50004CAAC3216F200AF019FF01216E200AF05C
:101F600074FF00B22860204638BD002C7FF43DAAE3
:101F7000C4216F200AF00AFF21466E200AF065FF97
:101F80002860204638BD002C7FF42FAAC4216F2082
:101F90000AF0FCFE01216E200AF057FF286020465F
:101FA00038BD002C7FF421AAC5216F200AF0EEFE77
:101FB00021466E200AF049FF2860204638BD002CDB
:101FC0007FF413AAC5216F200AF0E0FE01216E20E4
:101FD0000AF03BFF2860204638BD002C7FF405AA9C
:101FE000C6216F200AF0D2FE21466E200AF02DFF96
:101FF0002860204638BD002C7FF4F7A9C6216F2049
:102000000AF0C4FE01216E200AF01FFF286020465E
:1020100038BD002C7FF4E9A9C7216F200AF0B6FE75
:1020200021466E200AF011FF2860204638BD002CA2
:102030007FF4DBA9C7216F200AF0A8FE01216E20E2
:102040000AF003FF2860204638BD002C7FF4CDA99C
:10205000C8216F200AF09AFE6E200AF06BFE2860FD
:10206000204638BD002C7FF4C0A9C9216F200AF09A
:102070008DFE6E200AF05EFE2860204638BD002CE2
:102080007FF4B3A9CA216F200AF080FE6E200AF007
:1020900051FE2860204638BD002C7FF4A6A9CB2134
:1020A0006F200AF073FE6E200AF044FE286020467E
:1020B00038BD3CB93D490C2303FB001003892B605C
:1020C000204638BD012C6AD138490C2303FB00108F
:1020D0002B680381002038BD3CB934490C2303FB35
:1020E0000010C3792B60204638BD012C59D12F49EF
:1020F0000C2303FB00118A1D287807310EF082FFA4
:10210000002038BD002C4ED128490C2303FB0010C1
:1021100083792B60204638BD002C7FF466A9234BC1
:102120000C2101FB003083882B60204638BD002C39
:102130007FF45BA91E4B5B682B60204638BD0420F2
:1021400038BD002038BD002038BD002038BD00203B
:1021500038BD002038BD002038BD002038BD00202B
:1021600038BD002038BD002038BD002038BD00201B
:1021700038BD002038BD002038BD002038BD00200B
:1021800038BD002038BD002038BD002038BD0020FB
:1021900038BD002038BD002038BD002038BD0020EB
:1021A00038BD002038BD002038BD00BF8C46FF1F61
:1021B000D816FF1F10B413460446084619B9224624
:1021C00010BCFEF797BF082010BC70470120704775
:1021D00007B5019229B9024601AB0120FEF78AFF3B
:1021E00000E0082003B05DF804FB08460AF0A2BD39
:1021F000084611460AF0CABD084611460AF025BE37
:10220000084611461A460AF052BE38B5274B284DEB
:10221000DC686068236864302860DB68984723685E
:1022200028685B699847234B23495A690A60234908
:10223000C2F804122249C2F80812012000211070CD
:102240005170204A1A62204ADA61204A9A61204A73
:102250005A62204ADA64204A9A63204A5A63204A22
:102260009A62204ADA62204A9A64204A5A64204AD2
:102270005A65204A1A65204A1A66204ADA65204AB9
:102280009A653222DA6040F28A229A6018741D4BF5
:102290004FF47A725A8041F270721A80D9714FF4F9
:1022A00080721A81BDE83840FEF7F1BE0C5502007D
:1022B000E42FFF1FC82EFF1FA046FF1FCD210100E6
:1022C000150F0100731001008D100100891001002D
:1022D00085100100350F0100B5210100D121010059
:1022E000611001004D100100310F0100250F0100A8
:1022F0004B0F0100110F01008F100100190F010099
:10230000D11001008C46FF1F00207047012070474C
:10231000014B00225A607047C82EFF1F10B50C46B3
:102320000AF008FD206010BD0AF030BD38B50D463A
:10233000044620B90EF0C6FF2860204638BD0820AC
:1023400038BD30B589B004AC0546102200212046C6
:1023500012F012FF384B1A68AA1A092A06D999688E
:102360001D6064224A435A6000229A609A680132D2
:102370009A60324B33F8060C5A780290981E0190FE
:1023800033F8041C0091002029460FF0B7F80DF037
:10239000F7F920B10022114610460DF07DFA0DF03C
:1023A000E9F9002845D00DF065FA032841D8DFE8A7
:1023B00000F0130A022900200EF0A7FF049000206D
:1023C0000EF0AAFF06E000200EF079FF0490002036
:1023D0000EF078FF059028E000216F200AF0D6FC6F
:1023E0006E200AF0A7FC0121049069200AF02DFD5F
:1023F0000021054669200AF028FD00B200FA85F5A3
:10240000059512E076200AF095FC6423C0F30222C1
:10241000C0F302505A434343A3F52F730593084B6F
:102420000693A3F5FA630492079394E80F000DF066
:10243000C1F909B030BD00BFF016FF1F9246FF1F63
:10244000F0D8FFFF10B5044620B909680EF04CFF24
:10245000204610BD082010BD10B5044618B90EF076
:1024600036FF204610BD082010BD10B5044618B92F
:102470000EF018FF204610BD082010BD0021F4E723
:102480004942F2E7F1E7022804BF0C4B93F8D00071
:1024900020B90B4BDB681B689B690AE001280BD154
:1024A000064B93F8D030012B06D1054BDB681B6837
:1024B0005B69044A10681847704700BFC82EFF1FA9
:1024C0000C550200E42FFF1F10B50020FFF7DBFFC3
:1024D000044B054ADB6810681B68BDE810409B6927
:1024E000184700BF0C550200E42FFF1F043A38B50F
:1024F00004461D460846FB2A01F21D80DFE812F063
:10250000FC001B081B081B081B081B081B080C01F0
:1025100013011B0817011B081B081B081B081B08BD
:102520001B081B081B081B081B081B081B081B0893
:102530001B081B081B081B081B081B081B081B0883
:102540001B081B081B081B081B081B081B081B0873
:102550001B081B081B081B081B081B081B012D015F
:102560001B083F0152011B081B081B081B081B0806
:102570001B081B081B081B081B081B081B081B0843
:102580001B081B081B081B081B081B081B081B0833
:102590001B081B081B081B081B081B081B081B0823
:1025A0001B081B081B081B081B081B081B081B0813
:1025B0001B081B081B081B081B081B081B081B0803
:1025C0006501760183011B081B081B081B081B08FB
:1025D0001B081B081B0890019D01AA011B081B0872
:1025E000B701C101CB011B08D501DF01E9011B08BF
:1025F000F30101021B080F0219021B081B081B082C
:1026000023022C02350240024B021B081B081B0848
:1026100054025D0266021B081B081B081B081B08EE
:102620001B081B0871027C02870292029D02B50200
:10263000CD02E80203031E03380343034E0359038C
:1026400064031B081B081B081B081B086F037A0385
:102650008D03A003A903B203BD03CA03D503DD03A1
:10266000EC03F9030604130420042D043A04470480
:102670001B08540462047A0487049404A104AE0481
:10268000BB04C804D504E404F304020511052005C5
:102690002F0540054F055E056D057C058B059A05E8
:1026A000A905B805C705D605E505F40502061B080A
:1026B0001006280640065B0676069106AC061B0847
:1026C0001B081B08B906C806D706E606F506040768
:1026D0001307220731073F074D075B076907770795
:1026E00085079307A107AE07BB07C8071B08D507D7
:1026F000E807FE07080813082CB960200AF01AFB47
:102700002860204638BD012C40F0178729686020DA
:102710000AF03CFB002038BD002C40F0108700245C
:102720002C60204638BD002CF9D0002038BD002C8C
:10273000F5D0002038BD34B9214608200AF085FBC9
:102740002860204638BD012C40F0FB862A880021F5
:1027500008200AF0ACFB002038BD34B9214609201E
:102760000AF073FB2860204638BD012C40F0EB8650
:102770002A88002109200AF09AFB002038BD3CB9C4
:10278000012108200AF061FB00B22860204638BD14
:10279000012C40F0DA862A88214608200AF087FBBF
:1027A000002038BD3CB9012109200AF04EFB00B2DF
:1027B0002860204638BD012C40F0C9862A88214671
:1027C00009200AF074FB002038BD54B90121032010
:1027D0000AF0DCFA214602200AF037FB2860204686
:1027E00038BD012C14BF0020042038BD002CF8D1C6
:1027F000012103200AF0CAFA012102200AF025FB78
:102800002860204638BD002CEBD1022103200AF0BD
:10281000BDFA214602200AF018FB2860204638BD88
:10282000002CDED1032108460AF0B0FA214602202E
:102830000AF00BFB2860204638BD002CD1D10421C2
:1028400003200AF0A3FA012102200AF0FEFA286010
:10285000204638BD002CC4D1042103200AF096FA8A
:10286000214602200AF0F1FA2860204638BD002CEB
:10287000B7D1214612200AF0E8FA00B228602046BB
:1028800038BD002CADD1012112200AF0DEFA00B2D1
:102890002860204638BD002CA3D1214613200AF021
:1028A000D4FA00B22860204638BD002C99D12146C8
:1028B00015200AF0CAFA00B22860204638BD002C64
:1028C0008FD1012115200AF0C0FA00B228602046FD
:1028D00038BD002C85D1214616200AF0B6FA00B288
:1028E0002860204638BD002C7FF47BAF21460320B2
:1028F0000AF04CFA214602200AF0A7FA2860204686
:1029000038BD002C7FF46DAF214603200AF03EFA5B
:10291000012102200AF099FA2860204638BD002CD7
:102920007FF45FAF21460B200AF08FFA2860204623
:1029300038BD002C7FF455AF01210B200AF085FA39
:102940002860204638BD002C7FF44BAF41200AF0B0
:10295000F1F92860204638BD002C7FF442AF4220B8
:102960000AF0E8F92860204638BD002C7FF439AF22
:10297000012146200AF069FA00B22860204638BDDD
:10298000002C7FF42EAF214646200AF05EFA00B2FA
:102990002860204638BD002C7FF423AF47200AF082
:1029A000C9F92860204638BD002C7FF41AAF2120D9
:1029B0000AF0C0F92860204638BD002C7FF411AF22
:1029C00022200AF0B7F92860204638BD002C7FF499
:1029D00008AF214623200AF038FA00B228602046CA
:1029E00038BD002C7FF4FDAE27200AF0A3F920F0BB
:1029F0007F402860204638BD002C7FF4F2AE2820AE
:102A00000AF098F920F07F402860204638BD002C5D
:102A10007FF4E7AE01212A200AF017FA00B22860FD
:102A2000204638BD002C7FF4DCAE21462A200AF077
:102A30000CFA00B22860204638BD4CB9D4216F2072
:102A40000AF0A4F96E200AF075F92860204638BD16
:102A5000012C40F07E85D4216F200AF097F9296877
:102A60006E200AF093F9002038BD4CB9D5216F20B3
:102A70000AF08CF96E200AF05DF92860204638BD16
:102A8000012C40F06885D5216F200AF07FF9296874
:102A90006E200AF07BF9002038BD5CB9D6216F208A
:102AA0000AF074F921466E200AF0CFF900B22860CE
:102AB000204638BD012C40F05085D6216F200AF009
:102AC00065F92A8800216E200AF0F1F9002038BD4E
:102AD0005CB9D6216F200AF059F901216E200AF065
:102AE000B4F900B22860204638BD012C40F037858B
:102AF000D6216F200AF04AF92A8821466E200AF072
:102B0000D6F9002038BD5CB9D7216F200AF03EF914
:102B100021466E200AF099F900B22860204638BD9F
:102B2000012C40F01E85D7216F200AF02FF92A884A
:102B300000216E200AF0BBF9002038BD54B9D7211E
:102B40006F200AF023F901216E200AF07EF9286037
:102B5000204638BD012C40F00685D7216F200AF0B1
:102B600015F92A8821466E200AF0A1F9002038BD07
:102B7000002C7FF436AE214639200AF066F900B207
:102B80002860204638BD002C7FF42BAE012139206F
:102B90000AF05BF900B22860204638BD002C7FF4B3
:102BA00020AE21463D200AF050F900B228602046B0
:102BB00038BD002C7FF415AE21463F200AF045F9C0
:102BC00000B22860204638BD002C7FF40AAE2146B2
:102BD0003A200AF03AF900B22860204638BD002CAD
:102BE0007FF4FFAD214653200AF02FF900B2286090
:102BF000204638BD3CB9012164200AF026F900B214
:102C00002860204638BD012C40F0AF842A88214638
:102C100064200AF04CF9002038BD3CB921466420FC
:102C20000AF013F900B22860204638BD012C40F0AC
:102C30009E842A88002164200AF039F9002038BDDA
:102C4000002C7FF4CEAD66200AF074F82860204690
:102C500038BD002C7FF4C5AD68200AF06BF8286001
:102C6000204638BD002C7FF4BCAD012169200AF05C
:102C7000ECF800B22860204638BD002C7FF4B1ADDE
:102C8000BE4A0C2303FB012319890EF0BAFA28600F
:102C9000204638BD002C7FF4A4AD214669200AF0FF
:102CA000D4F800B22860204638BD002C7FF499ADDE
:102CB0000EF008FB2860204638BD24B90EF02CFB2E
:102CC0002860204638BD012C40F0538429686B20D1
:102CD0000AF05CF8002038BD002C7FF482AD21465C
:102CE0006D200AF053F86C200AF024F82860204682
:102CF00038BD002C7FF475AD01216D200AF046F837
:102D00006C200AF017F82860204638BD002C7FF4AC
:102D100068AD02216D200AF039F86C200AF00AF83B
:102D20002860204638BD002C7FF45BAD03216D2068
:102D30000AF02CF86C2009F0FDFF2860204638BD11
:102D4000002C7FF44EAD04216D200AF01FF86C209A
:102D500009F0F0FF2860204638BD002C7FF441AD1B
:102D600005216D200AF012F86C2009F0E3FF2860BD
:102D7000204638BD002C7FF434AD06216D200AF0CA
:102D800005F86C2009F0D6FF2860204638BD002CDD
:102D90007FF427AD07216D2009F0F8FF6C2009F0C2
:102DA000C9FF2860204638BD24B90EF0F9F9286023
:102DB000204638BD012C40F0DE8329680EF0E2F990
:102DC000002038BD4CB96D4A0C2303FB012319893F
:102DD0000EF00DFA2860204638BD012C40F0CD835E
:102DE000664A0C2303FB01232A6819890EF0EDF9CA
:102DF000002038BD002C7FF4F4AC01216F2009F0D5
:102E0000C5FF6E2009F096FF2860204638BD002CD3
:102E10007FF4E7AC02216F2009F0B8FF6E2009F0C3
:102E200089FF2860204638BD002C7FF4DAAC0321EE
:102E30006F2009F0ABFF6E2009F07CFF2860204670
:102E400038BD002C7FF4CDAC04216F2009F09EFF2B
:102E50006E2009F06FFF2860204638BD002C7FF4FB
:102E6000C0AC05216F2009F091FF6E2009F062FFD0
:102E70002860204638BD002C7FF4B3AC06216F20BB
:102E800009F084FF6E2009F055FF2860204638BD08
:102E9000002C7FF4A6AC07216F2009F077FF6E208D
:102EA00009F048FF2860204638BD002C7FF499AC1B
:102EB00008216F2009F06AFF21466E2009F0C5FF46
:102EC00000B22860204638BD002C7FF48AAC08216F
:102ED0006F2009F05BFF01216E2009F0B6FF00B200
:102EE0002860204638BD002C7FF47BAC09216F2080
:102EF00009F04CFF21466E2009F0A7FF00B22860C0
:102F0000204638BD002C7FF46CAC0A216F2009F0FC
:102F10003DFF21466E2009F098FF00B22860204650
:102F200038BD002C7FF45DAC0A216F2009F02EFF24
:102F300001216E2009F089FF00B22860204638BDCB
:102F4000002C7FF44EAC0B216F2009F01FFF2146AF
:102F50006E2009F07AFF00B22860204638BD002CB0
:102F60007FF43FAC0B216F2009F010FF01216E2090
:102F700009F06BFF00B22860204638BD8C46FF1F69
:102F8000002C7FF42EAC0C216F2009F0FFFE2146AF
:102F90006E2009F05AFF00B22860204638BD002C90
:102FA0007FF41FAC0C216F2009F0F0FE01216E2090
:102FB00009F04BFF00B22860204638BD002C7FF49A
:102FC00010AC0D216F2009F0E1FE21466E2009F0C2
:102FD0003CFF00B22860204638BD002C7FF401ACD5
:102FE0000D216F2009F0D2FE01216E2009F02DFF86
:102FF00000B22860204638BD002C7FF4F2AB0E21D1
:103000006F2009F0C3FE21466E2009F01EFF00B2BA
:103010002860204638BD002C7FF4E3AB0E216F20E2
:1030200009F0B4FE01216E2009F00FFF00B2286004
:10303000204638BD002C7FF4D4AB0F216F2009F05F
:10304000A5FE21466E2009F000FF00B22860204650
:1030500038BD002C7FF4C5AB0F216F2009F096FE20
:1030600001216E2009F0F1FE00B22860204638BD33
:10307000002C7FF4B6AB10216F2009F087FE2146AB
:103080006E2009F0E2FE00B22860204638BD002C18
:103090007FF4A7AB11216F2009F078FE21466E2046
:1030A00009F0D3FE00B22860204638BD002C7FF422
:1030B00098AB11216F2009F069FE01216E2009F003
:1030C000C4FE00B22860204638BD002C7FF489ABD6
:1030D00012216F2009F05AFE21466E2009F0B5FE3C
:1030E00000B22860204638BD002C7FF47AAB132153
:1030F0006F2009F04BFE21466E2009F0A6FE2860E5
:10310000204638BD002C7FF46CAB13216F2009F0F2
:103110003DFE01216E2009F098FE2860204638BD52
:103120004CB9D0216F2009F031FE6E2009F002FE6B
:103130002860204638BD012C40F02182D0216F202C
:1031400009F024FE29686E2009F020FE002038BD19
:103150004CB9D1216F2009F019FE6E2009F0EAFD6B
:103160002860204638BD012C40F00B82D1216F2011
:1031700009F00CFE29686E2009F008FE002038BD19
:103180005CB9D2216F2009F001FE21466E2009F0C2
:103190005CFE00B22860204638BD012C40F0F3816F
:1031A000D2216F2009F0F2FD2A8800216E2009F05B
:1031B0007EFE002038BD5CB9D2216F2009F0E6FD0B
:1031C00001216E2009F041FE00B22860204638BD82
:1031D000012C40F0DA81D2216F2009F0D7FD2A8836
:1031E00021466E2009F063FE002038BD5CB9D32172
:1031F0006F2009F0CBFD21466E2009F026FE00B2BB
:103200002860204638BD012C40F0C181D3216F20B9
:1032100009F0BCFD2A8800216E2009F048FE00203C
:1032200038BD5CB9D3216F2009F0B0FD01216E20BB
:1032300009F00BFE00B22860204638BD012C40F09A
:10324000A881D3216F2009F0A1FD2A8821466E2094
:1032500009F02DFE002038BD002C7FF4C2AA1D21EC
:103260006F2009F093FD6E2009F064FD2860204670
:1032700038BD002C7FF4B5AAC0216F2009F086FD6F
:1032800021466E2009F0E1FD00B22860204638BDDD
:10329000002C7FF4A6AAC0216F2009F077FD012140
:1032A0006E2009F0D2FD00B22860204638BD002C07
:1032B0007FF497AAC1216F2009F068FD21466E2096
:1032C00009F0C3FD00B22860204638BD002C7FF411
:1032D00088AAC1216F2009F059FD01216E2009F053
:1032E000B4FD00B22860204638BD002C7FF479AAD6
:1032F000C2216F2009F04AFD21466E2009F0A5FD8C
:1033000000B22860204638BD002C7FF46AAAC22192
:103310006F2009F03BFD01216E2009F096FD00B2FF
:103320002860204638BD002C7FF45BAAC3216F20A3
:1033300009F02CFD21466E2009F087FD00B22860BF
:10334000204638BD002C7FF44CAAC3216F2009F021
:103350001DFD01216E2009F078FD00B22860204695
:1033600038BD002C7FF43DAAC4216F2009F00EFD6A
:1033700021466E2009F069FD2860204638BD002CEA
:103380007FF42FAAC4216F2009F000FD01216E20D7
:1033900009F05BFD2860204638BD002C7FF421AA8F
:1033A000C5216F2009F0F2FC21466E2009F04DFD89
:1033B0002860204638BD002C7FF413AAC5216F2059
:1033C00009F0E4FC01216E2009F03FFD2860204651
:1033D00038BD002C7FF405AAC6216F2009F0D6FC69
:1033E00021466E2009F031FD2860204638BD002CB2
:1033F0007FF4F7A9C6216F2009F0C8FC01216E20D7
:1034000009F023FD2860204638BD002C7FF4E9A98F
:10341000C7216F2009F0BAFC21466E2009F015FD86
:103420002860204638BD002C7FF4DBA9C7216F201F
:1034300009F0ACFC01216E2009F007FD2860204650
:1034400038BD002C7FF4CDA9C8216F2009F09EFC67
:103450006E2009F06FFC2860204638BD002C7FF4F8
:10346000C0A9C9216F2009F091FC6E2009F062FC0F
:103470002860204638BD002C7FF4B3A9CA216F20F4
:1034800009F084FC6E2009F055FC2860204638BD08
:10349000002C7FF4A6A9CB216F2009F077FC6E20C9
:1034A00009F048FC2860204638BD3CB93D490C2352
:1034B00003FB001003892B60204638BD012C6AD124
:1034C00038490C2303FB00102B680381002038BD12
:1034D0003CB934490C2303FB0010C3792B60204610
:1034E00038BD012C59D12F490C2303FB00118A1D33
:1034F000287807310EF00CF8002038BD002C4ED192
:1035000028490C2303FB001083792B60204638BD2B
:10351000002C7FF466A9234B0C2101FB003083882B
:103520002B60204638BD002C7FF45BA91E4B5B68E6
:103530002B60204638BD042038BD002038BD002057
:1035400038BD002038BD002038BD002038BD002027
:1035500038BD002038BD002038BD002038BD002017
:1035600038BD002038BD002038BD002038BD002007
:1035700038BD002038BD002038BD002038BD0020F7
:1035800038BD002038BD002038BD002038BD0020E7
:1035900038BD002038BD002038BD002038BD0020D7
:1035A00038BD00BF8C46FF1FF016FF1F10B4134636
:1035B0000446084619B9224610BCFEF797BF0820FA
:1035C00010BC70470120704707B5019229B9024627
:1035D00001AB0120FEF78AFF00E0082003B05DF890
:1035E00004FB084609F0A6BB0846114609F0CEBB0D
:1035F0000846114609F029BC084611461A4609F04A
:1036000056BC38B5274B284DDC68606823686430A9
:103610002860DB689847236828685B699847234BD4
:1036200023495A690A602349C2F804122249C2F8A0
:1036300008120120002110705170204A1A62204A9D
:10364000DA61204A9A61204A5A62204ADA64204AA2
:103650009A63204A5A63204A9A62204ADA62204AD0
:103660009A64204A5A64204A5A65204A1A65204AB8
:103670001A66204ADA65204A9A653222DA6040F2F8
:103680008A229A6018741D4B4FF47A725A8041F264
:1036900070721A80D9714FF480721A81BDE8384077
:1036A000FEF7F1BE0C550200E42FFF1FC82EFF1FCE
:1036B000A446FF1FC53501000D2301006B24010046
:1036C00085240100812401007D2401002D230100B7
:1036D000AD350100C9350100592401004524010020
:1036E000292301001D2301004323010009230100B8
:1036F0008724010011230100C92401008C46FF1F0B
:10370000014B00225A607047C82EFF1F70B5084E4B
:10371000084D336804462A46014600200EF064F83E
:1037200033682A4621460120BDE870400EF05CB89F
:103730004449FF1FA846FF1F014B18680EF0B5B89B
:103740004449FF1F01280CD8074B1A68202303FAAD
:1037500000F040F0020002EB800043680B600020A4
:1037600070470820704700BF4449FF1F012810B56B
:10377000144616D008D302281FD1114B114ADB681A
:1037800090681B681B6A12E014680D4A0D4BD268E2
:10379000126824B15269D8689047002010BD926920
:1037A000F9E7074B074ADB6850681B681B6A9847B4
:1037B000003018BF01202060EFE7042010BD00BFDB
:1037C0000C5502000817FF1F022804BF0B4B93F88B
:1037D000D00020B90A4BDB681B685B690AE001284E
:1037E0000BD1064B93F8D030012B06D1044BDB688C
:1037F0001B689B69034A106818477047C82EFF1F53
:103800000C5502000817FF1F70B50020FFF7DCFF02
:10381000104B114CDD6820682B689B6898472B681B
:1038200060689B6898472B68A0689B6898472B68DE
:10383000A0699B6898472B6820699B6898472B680C
:1038400060699B6898472B68E0689B68BDE870409A
:10385000184700BF0C5502000817FF1F2DE9F84359
:10386000184C9DF820609DF82450984623680F4618
:103870009B68002147F0800091469847236800210B
:103880009B6848469847236800219B6840469847B4
:10389000236800219B6830469847236828469B6828
:1038A00001219847084B1B6848EA092807F07F0761
:1038B00046EA082603EB870745EA06257D60BDE852
:1038C000F88300BF4049FF1F4449FF1F07B5D3B22B
:1038D0000193C2F307230093C2F30743120EFFF7CD
:1038E000BDFF03B05DF804FB0A4601460020FFF768
:1038F000EDBF012873B505460C4623D8134E335C43
:1039000063B1134B202103EB8003814041F0070199
:10391000DA69C9B2FFF7DAFF002373552026AE40FB
:1039200046F00D012246C9B200242846FFF7CEFF1B
:1039300028460194009423462246F1B2FFF78EFFF9
:10394000204600E0082002B070BD00BFAC00FF1FA1
:103950000817FF1F012873B505460E461BD8202403
:10396000844044F0070186EAE672A2EBE672C9B22F
:10397000FFF7ACFF094A0123002E5355E1B2B8BF4F
:103980000223002401932846009423462246FFF791
:1039900065FF204600E0082002B070BDAC00FF1FAC
:1039A0000021D7E74942D5E7D4E738B5234B01F0EA
:1039B0007F04234493F81432DB0705D4204B1B68A3
:1039C00003EB8404606838BD1E4D2B6800219B68A2
:1039D000204698472B6800219B68084698472B682B
:1039E00000219B68084698472B6800219B68084681
:1039F00098472B6801219B68002098472B6800217D
:103A00009B68204698472B6800219B68084698478A
:103A10002B68002104029B68084698472B68002108
:103A2000204304029B68084698472B682043040201
:103A30009B68012100209847204338BDA846FF1FFE
:103A40004449FF1F4049FF1F10B50C4601460020A6
:103A5000FFF7ABFF206010BD38B50D462021814037
:103A600041F00101C9B20446FFF79FFF29680144F4
:103A700029602046BDE838403BE71C2A2DE9F84381
:103A800004460E461F4600F088835DD80C2A00F0DD
:103A9000F8812BD8052A00F0508113D8022A00F0B3
:103AA000EA8007D8002A00F0AD80012A00F0C88023
:103AB00000F0C3BF032A00F0FE80042A00F0138147
:103AC00000F0BBBF082A00F0A58107D8062A00F045
:103AD0005081072A00F0768100F0AFBF0A2A00F07B
:103AE000AA810B2A00F0BA8100F0A7BF122A00F0C9
:103AF000908213D80F2A00F0348207D80D2A00F0E4
:103B0000EA810E2A00F0118200F097BF102A00F01F
:103B10004482112A00F0618200F08FBF152A00F064
:103B2000CC8207D8132A00F09082142A00F0A982D0
:103B300000F083BF172A00F0F882C0F0DA82182A5A
:103B400000F00F8300F079BFAC2A00F09E852AD8E0
:103B5000A52A00F03D8413D8A22A00F0C18307D81B
:103B60001D2A00F042838C2A00F04F8300F065BFCD
:103B7000A32A00F0DD83A42A00F0028400F05DBFD8
:103B8000A82A00F0E38407D8A62A00F07084A72AA8
:103B900000F0B38400F051BFAA2A00F0268540F25D
:103BA000FC8400F04ABDB62A00F0A38213D8B32AE1
:103BB00000F0EA8507D8AD2A00F08E85AE2A00F025
:103BC000B38500F03ABFB42A00F00686B52A00F0AB
:103BD000138600F032BFCE2A00F0968607D8B82AA6
:103BE00000F04286B92A00F0678600F026BFD22A8C
:103BF00000F0B686D32A00F0CF86D12A40F01D8788
:103C000000F092BE58B92021B14041F00D01C9B277
:103C10003046FFF7CAFE38600020BDE8F88301286F
:103C200002D00020BDE8F8832021B14041F00D0111
:103C300030461A68C9B2FFF749FE0020BDE8F88394
:103C400058B92021B14041F00101C9B23046FFF717
:103C5000ACFE38602046BDE8F8830128E1D1202180
:103C6000B14041F0010130461A68C9B2FFF72EFE9B
:103C70000020BDE8F88358B92021B14041F0070188
:103C8000C9B23046FFF791FE38602046BDE8F883A0
:103C90000128C6D13A68C74B2021B140002A41F023
:103CA00007019855B8BF52423046C9B2FFF70EFE21
:103CB0000020BDE8F88388B92021B14041F002011D
:103CC000C9B23046FFF771FE10F4000318BF4FF081
:103CD0007F4303433B600020BDE8F883012CA0D163
:103CE0000420BDE8F88338B9B34800EB8100C3690C
:103CF0003B602046BDE8F883012892D13A68AE4B7C
:103D0000202403EB8103002A04FA01F4B8BF5242D5
:103D1000E1B23046DA61FFF748FE0546002880D15F
:103D20003A6844F00701002A3046B8BF5242C9B28F
:103D3000FFF7CCFD2846BDE8F88358B92021B140F3
:103D400041F00601C9B23046FFF72FFE3860204629
:103D5000BDE8F88301287FF464AF2021B14041F031
:103D6000060130461A68C9B2FFF7B0FD0020BDE871
:103D7000F88368B92021B14041F01001C9B2304642
:103D8000FFF713FEC0F3042038600020BDE8F8837D
:103D900001287FF446AF20248C4044F01004E4B2A4
:103DA00021463046FFF701FE3B681B0203F4F8533F
:103DB00020F4F8521A4330462146FFF787FD0020D1
:103DC000BDE8F88368B92021B14041F01001C9B2C3
:103DD0003046FFF7EAFD00F01F0038602046BDE8DE
:103DE000F88301287FF41DAF20248C4044F0100498
:103DF000E4B221463046FFF7D8FD3B6820F01F02B1
:103E000003F01F0330461A432146FFF75FFD0020F1
:103E1000BDE8F88300287FF461AF2021B14041F074
:103E20001501C9B23046FFF7C0FDC0F3402038602D
:103E30002046BDE8F88300287FF450AF2021B14030
:103E400041F01501C9B23046FFF7AFFDC0F34000A5
:103E500080F0010038600020BDE8F88300287FF47E
:103E60003DAF2021B14041F01501C9B23046FFF706
:103E70009CFD00F0010080F0010038602046BDE8A4
:103E8000F88368B92021B14041F01401C9B230462D
:103E9000FFF78BFDC0F3400038602046BDE8F88393
:103EA00001287FF4BEAE20248C4044F01404E4B218
:103EB00021463046FFF779FD3B68002B0CBF0223FB
:103EC000002320F002021A4330462146FFF7FEFC91
:103ED0000020BDE8F88368B92021B14041F0140109
:103EE000C9B23046FFF761FD00F0010038600020E4
:103EF000BDE8F88301287FF494AE20248C4044F080
:103F00001404E4B221463046FFF74FFD3A6820F032
:103F10000100002A14BF024640F00102214630464B
:103F2000FFF7D4FC0020BDE8F88358B92021B14048
:103F300041F01401C9B23046FFF737FD3860204622
:103F4000BDE8F88301287FF46CAE2021B14041F038
:103F5000140130461A68C9B2FFF7B8FC0020BDE86A
:103F6000F88358B92021B14041F00401C9B230466C
:103F7000FFF71BFD38602046BDE8F88301287FF479
:103F800050AE2021B14041F0040130461A68C9B258
:103F9000FFF79CFC0020BDE8F88378B92021B140F0
:103FA00041F00501C9B23046FFF7FFFC3860002040
:103FB000BDE8F883AC00FF1F0817FF1F01287FF43E
:103FC00030AE2021B14041F0050130461A68C9B237
:103FD000FFF77CFC0020BDE8F88358B92021B140F0
:103FE00041F00801C9B23046FFF7DFFC38602046D7
:103FF000BDE8F88301287FF414AE2021B14041F0E0
:10400000080130461A68C9B2FFF760FC0020BDE81D
:10401000F88358B92021B14041F00A01C9B23046B5
:10402000FFF7C3FC38602046BDE8F88301287FF421
:10403000F8AD2021B14041F00A0130461A68C9B2FA
:10404000FFF744FC0020BDE8F88358B92021B140B7
:1040500041F00301C9B23046FFF7A7FC38600020E9
:10406000BDE8F88301287FF4DCAD2021B14041F0A8
:10407000030130461A68C9B2FFF728FC0020BDE8EA
:10408000F88358B92021B14041F00B01C9B2304644
:10409000FFF78BFC38602046BDE8F88301287FF4E9
:1040A000C0AD2021B14041F00B0130461A68C9B2C1
:1040B000FFF70CFC0020BDE8F88358B92021B1407F
:1040C00041F00C01C9B23046FFF76FFC3860204662
:1040D000BDE8F88301287FF4A4AD2021B14041F070
:1040E0000C0130461A68C9B2FFF7F0FB0020BDE8AA
:1040F000F8835CB92021B14041F01101C9B23046CA
:10410000FFF753FC38600020BDE8F883012C7FF4F2
:1041100088AD2021B14041F0110130463A68C9B262
:10412000FFF7D4FB0020BDE8F88358B92021B14047
:1041300041F01201C9B23046FFF737FC3860002069
:10414000BDE8F88301287FF46CAD2021B14041F037
:10415000120130461A68C9B2FFF7B8FB0020BDE86B
:10416000F88358B92021B14041F01301C9B230465B
:10417000FFF71BFC38602046BDE8F88301287FF478
:1041800050AD2021B14041F0130130461A68C9B248
:10419000FFF79CFB0020BDE8F88368B9090141F0F6
:1041A0006C0101F0FC013046FFF7FFFBC0F38040DB
:1041B00038602046BDE8F88301287FF432AD0C0159
:1041C00044F06C04E4B221463046FFF7EEFB3B6856
:1041D0009B0403F4802320F480221A4330462146B6
:1041E000FFF774FB0020BDE8F88300287FF476AD6C
:1041F000C94B20201B68884040F0020003EB800080
:1042000043683B600020BDE8F88388B9090141F0AC
:104210006C0101F0FC013046FFF7C7FB4FF48073DF
:10422000C0F3036043FA00F038602046BDE8F8832D
:1042300001287FF4F6AC1B68102B1FD00CDC022B7E
:1042400018D003DC012B1FD108231FE0042B13D04F
:10425000082B19D1052319E0402B11D003DC202BAA
:1042600012D1032312E0802B0CD0B3F5807F0BD149
:1042700000230BE0072309E0062307E0042305E001
:10428000022303E0386002E04FF0FF333B603B68FD
:1042900001333FF4C6AC340144F06C04E4B221466F
:1042A0003046FFF782FB3B681B0603F0706320F08B
:1042B00070621A4321463046FFF708FB214630461C
:1042C000FFF773FB3B681B0603F0706320F070621E
:1042D0001A4330462146FFF7F9FA0020BDE8F8837B
:1042E00068B9090141F06C0101F0FC013046FFF7AB
:1042F0005CFBC0F3C13038602046BDE8F88301287C
:104300007FF48FAC0C0144F06C04E4B221463046DB
:10431000FFF74BFB3B68DB0303F4C03320F4C032F0
:104320001A4330462146FFF7D1FA0020BDE8F88352
:1043300068B9090141F06C0101F0FC013046FFF75A
:1043400034FBC0F3803038600020BDE8F8830128DA
:104350007FF467AC0C0144F06C04E4B221463046B3
:10436000FFF723FB3B689B0303F4804320F4804268
:104370001A4330462146FFF7A9FA0020BDE8F8832A
:1043800068B9090141F06C0101F0FC013046FFF70A
:104390000CFBC0F3003038602046BDE8F8830128EC
:1043A0007FF43FAC0C0144F06C04E4B2214630468B
:1043B000FFF7FBFA3B681B0303F4805320F48052A1
:1043C0001A4330462146FFF781FA0020BDE8F88302
:1043D0004FEA011848F06C085FFA88F84146304609
:1043E000FFF7E3FA0546D4B915F480494146304653
:1043F00007D0FFF7DAFAC0F3C31038602046BDE8F3
:10440000F883FFF7D2FA2C05C0F3021001D438600C
:1044100007E440F0080038604846BDE8F883012C06
:104420007FF4FFAB15F48045414630460FD0FFF7CF
:10443000BCFA3B68DB0103F4F06320F4F0621A433A
:1044400030464146FFF742FA0020BDE8F883FFF707
:10445000ACFA3B681B0103F0700320F070021A43B2
:1044600030464146FFF732FA2846BDE8F8830D0191
:1044700045F06C05EDB229463046FFF796FAA4B92F
:1044800010F480442946304607D0FFF78EFAC0F377
:10449000021038600020BDE8F883FFF786FAC0F309
:1044A000C31038602046BDE8F883012C7FF4B9AB17
:1044B00010F48044294630460FD0FFF776FA3B6867
:1044C0001B0103F0700320F070021A4330462946A6
:1044D000FFF7FCF90020BDE8F883FFF766FA3B68B8
:1044E000DB0103F4F06320F4F0621A4330462946FE
:1044F000FFF7ECF92046BDE8F88378B9090141F0EF
:104500006C0101F0FC013046FFF74FFA00F00F009C
:1045100038602046BDE8F8834449FF1F01287FF436
:1045200080AB0C0144F06C04E4B221463046FFF746
:104530003CFA3B6820F00F0203F00F0330461A43A9
:104540002146FFF7C3F90020BDE8F88368B90901E7
:1045500041F06D0101F0FD013046FFF726FAC0F38E
:10456000C03038602046BDE8F88301287FF459AB9D
:104570000C0144F06D04E4B221463046FFF715FA11
:104580003B68DB039BB220F400421A4330462146CD
:10459000FFF79CF90020BDE8F88368B9090141F0F4
:1045A0006D0101F0FD013046FFF7FFF9C0F3413026
:1045B00038602046BDE8F88301287FF432AB0C0157
:1045C00044F06D04E4B221463046FFF7EEF93B6853
:1045D0005B0303F4C04320F4C0421A433046214633
:1045E000FFF774F90020BDE8F88368B9090141F0CC
:1045F0006D0101F0FD013046FFF7D7F9C0F303204C
:1046000038600020BDE8F88301287FF40AAB0C0174
:1046100044F06D04E4B221463046FFF7C6F93B682A
:104620001B0203F4706320F470621A433046214683
:10463000FFF74CF90020BDE8F88368B9090141F0A3
:104640006D0101F0FD013046FFF7AFF9C0F34110F5
:1046500038602046BDE8F88301287FF4E2AA0C0107
:1046600044F06D04E4B221463046FFF79EF93B6802
:104670005B0103F0600320F060021A4330462146DC
:10468000FFF724F90020BDE8F88368B9090141F07B
:104690006D0101F0FD013046FFF787F900F00F00D2
:1046A00038602046BDE8F88301287FF4BAAA0C01DF
:1046B00044F06D04E4B221463046FFF776F93B68DA
:1046C00020F00F0203F00F0330461A432146FFF794
:1046D000FDF80020BDE8F88368B9090141F06D01DB
:1046E00001F0FD013046FFF760F9C0F3006038606B
:1046F0000020BDE8F88301287FF493AA0C0144F060
:104700006D04E4B221463046FFF74FF93B681B06C3
:1047100003F0807320F080721A4330462146FFF781
:10472000D5F80020BDE8F883A8B9090141F06D0172
:1047300001F0FD013046FFF738F9001410F0400F8A
:1047400000F07F0214BF6FF07F03002313433B6030
:104750002046BDE8F88301287FF463AA0C0144F0E9
:104760006D04E4B221463046FFF71FF93B681B0495
:1047700003F4FE0320F4FE021A4330462146FFF7FD
:10478000A5F80020BDE8F88368B9090141F06C0183
:1047900001F0FC013046FFF708F9C0F340403860F3
:1047A0002046BDE8F88301287FF43BAA0C0144F0C1
:1047B0006C04E4B221463046FFF7F7F83B685B042F
:1047C00003F4003320F400321A4330462146FFF749
:1047D0007DF80020BDE8F88300287FF47FAA090156
:1047E00041F06F01C9B23046FFF7DFF8C0F3044073
:1047F00038600020BDE8F88320258D406DB245F07B
:1048000014085FFA88F841463046FFF7CEF87CB9C5
:10481000410509D545F01101C9B23046FFF7C5F889
:1048200038602046BDE8F8833C602046BDE8F88348
:10483000012C7FF4F6A945F011013A683046C9B25F
:10484000FFF744F841463046FFF7AFF83B689B025C
:1048500003F4806320F480621A4330464146FFF738
:1048600035F80020BDE8F88368B9090141F06C0112
:1048700001F0FC013046FFF798F8C0F34030386093
:104880000020BDE8F88301287FF4CBA90C0144F097
:104890006C04E4B221463046FFF787F83B685B03BF
:1048A00003F4005320F400521A4330462146FFF728
:1048B0000DF80020BDE8F88368B9090141F06C01EA
:1048C00001F0FC013046FFF770F8C0F30350386088
:1048D0002046BDE8F88301287FF4A3A90C0144F029
:1048E0006C04E4B221463046FFF75FF83B681B05D5
:1048F00003F4700320F470021A4330462146FEF799
:10490000E5FF0020BDE8F88300287FF4E7A909014E
:1049100041F06F01C9B23046FFF747F8C0F3090014
:1049200038602046BDE8F88358B92021B14041F0F5
:104930001901C9B23046FFF738F838602046BDE8A3
:10494000F88301287FF46DA92021B14041F01901BD
:1049500030461A68C9B2FEF7B9FF0020BDE8F883F7
:1049600058B92021B14041F01A01C9B23046FFF7D1
:104970001CF838600020BDE8F88301287FF451A9B5
:104980002021B14041F01A0130461A68C9B2FEF741
:104990009DFF0020BDE8F883E8B979B101294FD126
:1049A00001463046FFF701F800F06000A0F1200357
:1049B0005842584138602046BDE8F8830846FEF763
:1049C000F4FF00F01800A0F110025042504138608E
:1049D0003046BDE8F88301287FF423A911B10129ED
:1049E00015D02FE00846FEF7E0FF3B6823B120F02A
:1049F000080242F0100203E020F0100242F0080228
:104A000000210846FEF762FF0020BDE8F883002180
:104A10003046FEF7CAFF3B6823B120F0400242F067
:104A2000200203E020F0200242F040020021012099
:104A3000FEF74CFF0020BDE8F8830420BDE8F883B2
:104A4000BDE8F8830020BDE8F88307B5012901928D
:104A500005D8024601AB0120FFF70FF800E008205F
:104A600003B05DF804FB0129134603D80246002079
:104A7000FFF703B80820704708B522210020FEF791
:104A800094FF50B942210120FEF78FFF28B9044B53
:104A90001868BDE808400CF001BF002008BD00BF49
:104AA0004449FF1F70B53D4E3D483E4C0CF05CFE46
:104AB000F5686B6803F58272626003F59272A2601A
:104AC00003F57172E26003F5797203F1640022610B
:104AD00003F2044203F22443A3612B686261DB68A2
:104AE000206098472B68E068DB6898472B68E0688F
:104AF0009B6998472B6860681B6998472B68A0687A
:104B00001B6998472B68A0691B6998472B68206927
:104B10001B6998472B6860691B699847224B32696B
:104B20001A606B68214903F531735360204B5A6951
:104B30000A602049C2F804121F49C2F80812012075
:104B40000021107051701D4A1A621D4ADA611D4A17
:104B50009A611D4A5A621D4A9A631D4A5A631D4A48
:104B60009A621D4ADA621D4A9A641D4A5A641D4AB5
:104B70005A651D4A1A651D4ADA641D4A1A661D4A9D
:104B8000DA6502221A743222DA60B6229A601A4A70
:104B90009A65BDE87040FEF717BE00BF0C550200D5
:104BA000A846FF1F0817FF1F4049FF1F4449FF1F6A
:104BB000C82EFF1F794A010039370100553901001D
:104BC000A9390100A5390100A1390100674A010096
:104BD0004B4A0100F3380100593A0100E93801005D
:104BE000493A01000D3701006D37010045370100DA
:104BF000C9370100013701000938010001289FBFB2
:104C0000034B53F820300B60002088BF082070470A
:104C10005049FF1F014B00225A607047C82EFF1FEA
:104C200070B5084E084D336804462A4601460020F8
:104C30000CF084FE33682A4621460120BDE870400E
:104C40000CF07CBE4849FF1F5049FF1F014B1868FC
:104C50000CF0BFBE4849FF1F012810B5144608D00C
:104C6000022813D10A4B0B4ADB6890681B681B6A49
:104C700005E0074B074ADB6850681B681B6A9847CA
:104C8000003018BF01202060002010BD042010BD9E
:104C90000C5502003817FF1F022804BF0B4B93F876
:104CA000D00020B90A4BDB681B685B690AE0012869
:104CB0000BD1064B93F8D030012B06D1044BDB68A7
:104CC0001B689B69034A106818477047C82EFF1F6E
:104CD0000C5502003817FF1F70B50020FFF7DCFFEE
:104CE000084B094CDD6820682B689B6898472B6847
:104CF00060689B6898472B68A0689B68BDE8704017
:104D0000184700BF0C5502003817FF1F2DE9F84364
:104D1000184C9DF820609DF82450984623680F4653
:104D20009B68002147F08000914698472368002146
:104D30009B6848469847236800219B6840469847EF
:104D4000236800219B6830469847236828469B6863
:104D500001219847084B1B6848EA092807F07F079C
:104D600046EA082603EB870745EA06257D60BDE88D
:104D7000F88300BF4C49FF1F4849FF1F07B5D3B256
:104D80000193C2F307230093C2F30743120EFFF708
:104D9000BDFF03B05DF804FB0A4601460020FFF7A3
:104DA000EDBF0128F7B505460F4627D8154C04443A
:104DB00094F8943273B1144B202181401B6841F068
:104DC000070103EB8103C9B25A68FFF7D7FF00233D
:104DD00084F894322026AE4046F00D0100243A4675
:104DE000C9B22846FFF7CAFF28460194009423461B
:104DF0002246F1B2FFF78AFF204600E0082003B008
:104E0000F0BD00BF5049FF1F4849FF1F012873B57F
:104E100005460C4620D82026864084EAE47246F0F7
:104E20000701A2EBE472C9B2FFF7A8FF0C4B2B44B9
:104E3000002C4FF0010283F894224FF00004ACBF25
:104E40001346022301932846009423462246F1B2DA
:104E5000FFF75CFF204600E0082002B070BD00BFF5
:104E60005049FF1F0021D1E74942CFE7CEE738B5CF
:104E7000234B01F07F04234493F81432DB0705D45D
:104E8000204B1B6803EB8404606838BD1E4D2B6803
:104E900000219B68204698472B6800219B680846A4
:104EA00098472B6800219B68084698472B6800218B
:104EB0009B68084698472B6801219B68002098470B
:104EC0002B6800219B68204698472B6800219B682F
:104ED000084698472B68002104029B6808469847BB
:104EE0002B680021204304029B68084698472B68E2
:104EF000204304029B68012100209847204338BDCD
:104F00005049FF1F4849FF1F4C49FF1F10B50C4671
:104F100001460020FFF7ABFF206010BD38B50D46FD
:104F20002021814041F00101C9B20446FFF79FFFF3
:104F30002968014429602046BDE8384031E71C2A31
:104F40002DE9F84304460E461F4600F039835DD82C
:104F50000C2A00F0D8812BD8052A00F0458113D8FF
:104F6000022A00F0E08007D8002A00F0AE80012A73
:104F700000F0C58000F09BBE032A00F0F480042AF4
:104F800000F0088100F093BE082A00F08C8107D859
:104F9000062A00F03D81072A00F0618100F087BEFB
:104FA0000A2A00F08E810B2A00F09D8100F07FBE5E
:104FB000122A00F0718213D80F2A00F0268207D837
:104FC0000D2A00F0D6810E2A00F00B8200F06FBE91
:104FD000102A00F02E82112A00F04A8200F067BEEB
:104FE000152A00F0978207D8132A00F06882142A45
:104FF00000F07D8200F05BBE172A00F0B682C0F0A0
:105000009C82182A00F0C98200F051BEAB2A00F041
:10501000EF842BD8A52A00F0BF8313D8A22A00F072
:10502000518307D81D2A00F0EE828C2A00F0F3820B
:1050300000F03DBEA32A00F06883A42A00F0898313
:1050400000F035BEA82A00F0678407D8A62A00F031
:10505000F883A72A00F0438400F029BEA92A00F0B3
:105060007F84AA2A00F0A08400F021BEB52A00F0B7
:10507000858513D8AE2A00F0248507D8AC2A00F025
:10508000DA84AD2A00F0FA8400F011BEB32A00F0F1
:105090004485B42A00F0658500F009BECE2A00F0F0
:1050A000B48507D8B62A00F04882B82A00F08B856C
:1050B00000F0FDBDD12AC0F0FA85D22A40F2FD856C
:1050C000D32A00F0AF8500F0F2BD50B92021B140E5
:1050D00041F00D01C9B23046FFF7C9FE386000F05B
:1050E000ECBD012840F0E9852021B14041F00D01DF
:1050F0001A68C9B23046FFF741FE00F0DEBD20B9A4
:105100002021B14041F0010112E0012840F0D58595
:105110002021B14041F001011A68C9B23046FFF7C1
:105120002DFE00F0CABD48B92021B14041F0070171
:10513000C9B23046FFF79BFE00F041BC012840F0A9
:10514000BC85C94B0B44202183F894023A68B140D6
:10515000002A41F00701B8BF5242C9B23046FFF7FA
:105160000DFE00F0AABD80B92021B14041F002013E
:10517000C9B23046FFF77BFE10F4000318BF4FF0B2
:105180007F4303433B6000F098BD012C00F08F8506
:1051900000F093BD50B9B54B20201B68884040F00B
:1051A000070003EB8000436800F09EBC012840F03C
:1051B0008485AE4B3A681B682021B14041F007045A
:1051C00003EB8403002AB8BF52425A60C9B230468A
:1051D000FFF74DFE0546002840F06F853A68002A2B
:1051E000B8BF5242E1B274E320B92021B14041F08E
:1051F00006019DE7012840F060852021B14041F083
:1052000006011A68C9B23046FFF7B8FD00F055BD77
:1052100060B92021B14041F01001C9B23046FFF71A
:1052200026FEC0F30420386000F047BD012840F09E
:10523000448520248C4044F01004E4B221463046DA
:10524000FFF715FE3B681B0203F4F85320F4F852F5
:105250001A4321463046FFF791FD00F02EBD50B9AC
:105260002021B14041F01001C9B23046FFF7FFFDE7
:1052700000F01F00A3E3012840F01F8520248C408C
:1052800044F01004E4B221463046FFF7F0FD3B68DD
:1052900020F01F0203F01F031A4321463046FFF798
:1052A0006DFD00F00ABD00287FF46FAF2021B140F2
:1052B00041F01501C9B23046FFF7D9FDC0F34020D7
:1052C0007DE300287FF461AF2021B14041F015015A
:1052D000C9B23046FFF7CBFDC0F3400080F00100BB
:1052E000386000F0EABC00287FF44FAF2021B140C5
:1052F00041F01501C9B23046FFF7B9FD00F00100D9
:1053000080F001005BE350B92021B14041F014016D
:10531000C9B23046FFF7ABFDC0F340004FE30128B0
:1053200040F0CB8420248C4044F01404E4B22146A5
:105330003046FFF79CFD3B68002B14BF022300237F
:1053400020F002021A4321463046FFF717FD21469E
:105350003046FFF78CFD3B68022B20F008020CBFA3
:10536000082300231A4321463046FFF707FD00F0CB
:10537000A4BC60B92021B14041F01401C9B230464B
:10538000FFF775FD00F00100386000F096BC0128C1
:1053900040F0938420248C4044F01404E4B221466D
:1053A0003046FFF764FD3A6820F00100002A0CBF88
:1053B000024640F0010221463046FFF7DFFC21465D
:1053C0003046FFF754FD3B68022B20F004020CBF6F
:1053D000042300231A4321463046FFF7CFFC00F098
:1053E0006CBC20B92021B14041F01401A0E6012895
:1053F00040F063842021B14041F014011A68C9B221
:105400003046FFF7BBFC00F058BC20B92021B1406A
:1054100041F004018CE6012840F04F842021B14086
:1054200041F004011A68C9B23046FFF7A7FC00F04A
:1054300044BC50B92021B14041F00501C9B2304609
:10544000FFF715FD386000F038BC012840F03584C6
:105450002021B14041F005011A68C9B23046FFF77A
:105460008DFC00F02ABC00BF5049FF1F4849FF1FB8
:1054700020B92021B14041F0080159E6012840F04F
:105480001C842021B14041F008011A68C9B230469D
:10549000FFF774FC00F011BC20B92021B14041F0AD
:1054A0000A0145E6012840F008842021B14041F07E
:1054B0000A011A68C9B23046FFF760FCFDE348B93B
:1054C0002021B14041F00301C9B23046FFF7CFFCC3
:1054D0003860F2E3012840F0F0832021B14041F030
:1054E00003011A68C9B23046FFF748FCE5E320B96A
:1054F0002021B14041F00B011AE6012840F0DD8384
:105500002021B14041F00B011A68C9B23046FFF7C3
:1055100035FCD2E320B92021B14041F00C0107E66F
:10552000012840F0CA832021B14041F00C011A68E3
:10553000C9B23046FFF722FCBFE34CB92021B1408D
:1055400041F01101C9B23046FFF791FC3860B4E375
:10555000012C40F0B2832021B14041F011013A68A2
:10556000C9B23046FFF70AFCA7E348B92021B14091
:1055700041F01201C9B23046FFF779FC38609CE374
:10558000012840F09A832021B14041F012011A68AD
:10559000C9B23046FFF7F2FB8FE320B92021B140BA
:1055A00041F01301C4E5012840F087832021B14078
:1055B00041F013011A68C9B23046FFF7DFFB7CE304
:1055C00050B9090141F06C0101F0FC013046FFF7D0
:1055D0004EFCC0F38040F2E1012840F06E830C01E4
:1055E00044F06C04E4B221463046FFF740FC3B68CF
:1055F0009B0403F4802320F480221A432146304682
:10560000FFF7BCFB59E300287FF4BFADC84B53F84C
:1056100021303B6051E370B9090141F06C0101F0A8
:10562000FC013046FFF723FC4FF48073C0F30360A6
:1056300043FA00F0C3E1012840F03F831B68102BC0
:105640001FD00CDC022B18D003DC012B1FD1082348
:105650001FE0042B13D0082B19D1052319E0402B90
:1056600011D003DC202B12D1032312E0802B0CD0AD
:10567000B3F5807F0BD100230BE0072309E006235D
:1056800007E0042305E0022303E0386002E04FF066
:10569000FF333B603B68013300F00F83340144F07B
:1056A0006C04E4B221463046FFF7E1FB3B681B0681
:1056B00003F0706320F070621A4321463046FFF712
:1056C0005DFBFAE250B9090141F06C0101F0FC0107
:1056D0003046FFF7CCFBC0F3C13070E1012840F049
:1056E000EC820C0144F06C04E4B221463046FFF732
:1056F000BEFB3B68DB0303F4C03320F4C0321A4323
:1057000021463046FFF73AFBD7E258B9090141F08C
:105710006C0101F0FC013046FFF7A9FBC0F38030BB
:105720003860CAE2012840F0C8820C0144F06C04E1
:10573000E4B221463046FFF79AFB3B689B0303F433
:10574000804320F480421A4321463046FFF716FB7F
:10575000B3E250B9090141F06C0101F0FC0130469F
:10576000FFF785FBC0F3003029E1012840F0A58256
:105770000C0144F06C04E4B221463046FFF777FB9D
:105780003B681B0303F4805320F480521A432146E4
:105790003046FFF7F3FA90E20D0145F06C05EDB2EB
:1057A00029463046FFF763FBB4B910F4804206D0B7
:1057B00029463046FFF75BFBC0F3C310FFE003113F
:1057C000010503F0700301D43B6076E243F0080367
:1057D0003B601046BDE8F883012C40F06E8210F467
:1057E0008044294630460DD0FFF741FB3B68DB0182
:1057F00003F4F06320F4F0621A4329463046FFF7C1
:10580000BDFA5AE2FFF733FB3B6813F0080F18BFED
:105810004FF4006420F40062224329463046FFF72B
:10582000ADFA29463046FFF722FB3B681B0103F027
:10583000700320F070021A4329463046FFF79EFAA3
:105840003BE24FEA011848F06C085FFA88F84146DD
:105850003046FFF70CFB8146BCB919F48045414640
:10586000304605D0FFF703FBC0F30210386024E296
:10587000FFF7FDFA19F4006FC0F3C31001D13860CF
:105880001BE240F00800386026E0012C40F0158251
:1058900041463046FFF7EBFA10F48045414630466A
:1058A0000DD0FFF7E4FA3B681B0103F0700320F012
:1058B00070021A4341463046FFF760FAFDE1FFF7F8
:1058C000D6FA3B68DB0103F4F06320F4F0621A437C
:1058D00041463046FFF752FA2846BDE8F88348B9FA
:1058E000090141F06C0101F0FC013046FFF7BFFAFD
:1058F0003C60DFE1012840F0E0810C0144F06C04E1
:10590000E4B221463046FFF7B2FA214620F00F02FA
:105910003046FFF733FAD0E160B9090141F06D017B
:1059200001F0FD013046FFF7A2FAC0F3C03046E0B7
:105930005049FF1F012840F0C0810C0144F06D0464
:10594000E4B221463046FFF792FA3B68DB039BB294
:1059500020F400421A4321463046FFF70FFAACE12B
:1059600058B9090141F06D0101F0FD013046FFF722
:105970007EFAC0F3413038609FE1012840F09D81FC
:105980000C0144F06D04E4B221463046FFF76FFA93
:105990003B685B0303F4C04320F4C0421A43214632
:1059A0003046FFF7EBF988E158B9090141F06D0184
:1059B00001F0FD013046FFF75AFAC0F303203860CA
:1059C00078E1012840F079810C0144F06D04E4B2E3
:1059D00021463046FFF74BFA3B681B0203F4706325
:1059E00020F470621A4321463046FFF7C7F964E19C
:1059F00050B9090141F06D0101F0FD013046FFF79A
:105A000036FAC0F34110DAE7012840F056810C0164
:105A100044F06D04E4B221463046FFF728FA3B68B3
:105A20005B0103F0600320F060021A432146304618
:105A3000FFF7A4F941E158B9090141F06D0101F006
:105A4000FD013046FFF713FA00F00F00386034E133
:105A5000012840F032810C0144F06D04E4B221468B
:105A60003046FFF704FA3B6820F00F0203F00F0303
:105A70001A4321463046FFF781F91EE150B909016A
:105A800041F06D0101F0FD013046FFF7F0F9C0F380
:105A9000006094E7012840F010810C0144F06D048F
:105AA000E4B221463046FFF7E2F93B681B0603F0FB
:105AB000807320F080721A4321463046FFF75EF96A
:105AC000FBE098B9090141F06D0101F0FD0130469C
:105AD000FFF7CDF9001410F0400F00F07F0214BF63
:105AE0006FF07F03002313433B60E3E0012840F0A5
:105AF000E4800C0144F06D04E4B221463046FFF727
:105B0000B6F93B681B0403F4FE0320F4FE021A43BB
:105B100021463046FFF732F9CFE058B9090141F08C
:105B20006C0101F0FC013046FFF7A1F9C0F34040E1
:105B30003860C2E0012840F0C0800C0144F06C04E1
:105B4000E4B221463046FFF792F93B685B0403F468
:105B5000003320F400321A4321463046FFF70EF995
:105B6000ABE000287FF411AB090141F06F01C9B22D
:105B70003046FFF77CF9C0F3044020E700283FF4EB
:105B8000DDAC012840F0998020248C4064B244F0C0
:105B9000110144F014041A683046E4B2C9B2FFF7A8
:105BA000EDF821463046FFF762F93B68002B20F400
:105BB000806214BF4FF4806300231A4321463046AD
:105BC000FFF7DCF879E050B9090141F06C0101F010
:105BD000FC013046FFF74BF9C0F34030EFE60128F7
:105BE0006BD10C0144F06C04E4B221463046FFF75F
:105BF0003EF93B685B0303F4005320F400521A4360
:105C000021463046FFF7BAF857E000287FF4BDAAD6
:105C1000090141F06F01C9B23046FFF728F9C0F31E
:105C20000900CCE6D0B961B1012943D10146304623
:105C3000FFF71DF900F06000A0F120035842584121
:105C4000BDE60846FFF713F900F01800A0F11002B6
:105C50005042504138603046BDE8F88301282CD1CD
:105C600011B1012911D028E00846FFF700F93B687F
:105C700020F0180013B140F0100201E040F00802DB
:105C800000210846FFF77AF817E000213046FFF7B9
:105C9000EEF83B6820F0600013B140F0200201E014
:105CA00040F0400200210120FFF768F805E00420E1
:105CB000BDE8F8832046BDE8F8830020BDE8F883FE
:105CC00007B50129019205D8024601AB0120FFF773
:105CD00036F900E0082003B05DF804FB0129134603
:105CE00003D802460020FFF72AB90820704708B5FC
:105CF00022210020FFF7BBF850B942210120FFF715
:105D0000B6F828B9034B1868BDE808400BF058BE38
:105D1000002008BD4849FF1F70B52D4E2D482E4D5F
:105D20000BF0CCFDF468636803F5827203F1640044
:105D300003F59273AB6023686A60DB68286098475C
:105D4000236868681B6998472368A8681B69984797
:105D5000224B32691A606368214903F5317353603D
:105D6000204B5A690A602049C2F804121F49C2F840
:105D7000081201211170002151701D4A1A621D4A3A
:105D8000DA611D4A9A611D4A5A621D4A9A631D4A88
:105D90005A631D4A9A621D4ADA621D4A9A641D4A74
:105DA0005A641D4A5A651D4A1A651D4ADA641D4A1D
:105DB0001A661D4ADA653222DA6002204FF48C72CC
:105DC0009A601874194A9A65BDE87040FEF764BF7E
:105DD0000C5502005049FF1F3817FF1F4C49FF1F89
:105DE0004849FF1FC82EFF1FEF5C01004D4C01000A
:105DF0000D4E01006D4E0100694E0100654E01001F
:105E0000DD5C0100C15C0100A34D01001D4F0100DC
:105E1000994D01000D4F0100214C0100594C01002A
:105E2000FD4B0100994C0100154C0100D94C0100BB
:105E300001289FBF034B53F820300B60002088BF20
:105E400008207047EC4BFF1F014B00225A6070473F
:105E5000C82EFF1F70B5084E084D336804462A4609
:105E6000014600200BF0FEFD33682A462146012042
:105E7000BDE870400BF0F6BDE84BFF1FEC4BFF1F79
:105E8000014B18680BF051BEE84BFF1F012810B5FD
:105E9000144616D008D302281FD1114B114ADB68D3
:105EA00090681B681B6A12E014680D4A0D4BD2689B
:105EB000126824B15269D8689047002010BD9269D9
:105EC000F9E7074B074ADB6850681B681B6A98476D
:105ED000003018BF01202060EFE7042010BD00BF94
:105EE0000C5502005017FF1F022804BF0B4B93F8FC
:105EF000D00020B90A4BDB681B685B690AE0012807
:105F00000BD1064B93F8D030012B06D1044BDB6844
:105F10001B689B69034A106818477047C82EFF1F0B
:105F20000C5502005017FF1F70B50020FFF7DCFF73
:105F3000104B114CDD6820682B689B6898472B68D4
:105F400060689B6898472B68A0689B6898472B6897
:105F5000A0699B6898472B6820699B6898472B68C5
:105F600060699B6898472B68E0689B68BDE8704053
:105F7000184700BF0C5502005017FF1F2DE9F843CA
:105F8000184C9DF820609DF82450984623680F46D1
:105F90009B68002147F080009146984723680021C4
:105FA0009B6848469847236800219B68404698476D
:105FB000236800219B6830469847236828469B68E1
:105FC00001219847084B1B6848EA092807F07F071A
:105FD00046EA082603EB870745EA06257D60BDE80B
:105FE000F88300BF844EFF1FE84BFF1F07B5D3B2F5
:105FF0000193C2F307230093C2F30743120EFFF786
:10600000BDFF03B05DF804FB0A4601460020FFF720
:10601000EDBF0128F7B505460F4627D8154C0444B7
:1060200094F8943273B1144B202181401B6841F0E5
:10603000070103EB8103C9B25A68FFF7D7FF0023BA
:1060400084F894322026AE4046F00D0100243A46F2
:10605000C9B22846FFF7CAFF284601940094234698
:106060002246F1B2FFF78AFF204600E0082003B085
:10607000F0BD00BFEC4BFF1FE84BFF1F012873B5BD
:1060800005460C4620D82026864084EAE47246F075
:106090000701A2EBE472C9B2FFF7A8FF0C4B2B4437
:1060A000002C4FF0010283F894224FF00004ACBFA3
:1060B0001346022301932846009423462246F1B258
:1060C000FFF75CFF204600E0082002B070BD00BF73
:1060D000EC4BFF1F0021D1E74942CFE7CEE738B5AF
:1060E000234B01F07F04234493F81432DB0705D4DB
:1060F000204B1B6803EB8404606838BD1E4D2B6881
:1061000000219B68204698472B6800219B68084621
:1061100098472B6800219B68084698472B68002108
:106120009B68084698472B6801219B680020984788
:106130002B6800219B68204698472B6800219B68AC
:10614000084698472B68002104029B680846984738
:106150002B680021204304029B68084698472B685F
:10616000204304029B68012100209847204338BD4A
:10617000EC4BFF1FE84BFF1F844EFF1F10B50C4672
:1061800001460020FFF7ABFF206010BD38B50D467B
:106190002021814041F00101C9B20446FFF79FFF71
:1061A0002968014429602046BDE8384031E71C2AAF
:1061B0002DE9F04104460E461F4600F08E835DD85F
:1061C0000C2A00F000822BD8052A00F0588113D841
:1061D000022A00F0EA8007D8002A00F0AD80012AE8
:1061E00000F0C88000F0E3BF032A00F00081042A19
:1061F00000F0158100F0DBBF082A00F0AD8107D860
:10620000062A00F05881072A00F07E8100F0CFBFF7
:106210000A2A00F0B2810B2A00F0C28100F0C7BF49
:10622000122A00F0968213D80F2A00F0398207D87C
:106230000D2A00F0F1810E2A00F0168200F0B7BF9F
:10624000102A00F04982112A00F0678200F0AFBFE7
:10625000152A00F0D28207D8132A00F09682142A59
:1062600000F0AF8200F0A3BF172A00F0FE82C0F05A
:10627000E082182A00F0158300F099BFAC2A00F0E4
:10628000BF852AD8A52A00F02E8413D8A22A00F0B0
:10629000B28307D81D2A00F048838C2A00F04F8370
:1062A00000F085BFA32A00F0CE83A42A00F0F38378
:1062B00000F07DBFA82A00F0048507D8A62A00F0C8
:1062C0007E84A72A00F0D68400F071BFAA2A00F0CD
:1062D000478540F21D8500F06BBDB62A00F0A9820B
:1062E00013D8B32A00F00B8607D8AD2A00F0AF858B
:1062F000AE2A00F0D48500F05ABFB42A00F02786F9
:10630000B52A00F0348600F052BFCE2A00F0BA86DB
:1063100007D8B82A00F06686B92A00F08B8600F00C
:1063200046BFD22A00F0DA86D32A00F0F386D12ABB
:1063300040F03D8700F0B6BE58B92021B14041F091
:106340000D01C9B23046FFF7CAFE38600020BDE833
:10635000F081012802D00020BDE8F0812021B14069
:1063600041F00D0130461A68C9B2FFF73FFE002028
:10637000BDE8F08158B92021B14041F00101C9B216
:106380003046FFF7ACFE38602046BDE8F0810128BA
:10639000E1D12021B14041F0010130461A68C9B273
:1063A000FFF724FE0020BDE8F08158B92021B1405C
:1063B00041F00701C9B23046FFF791FE3860204630
:1063C000BDE8F0810128C6D1CA4B0B44202183F8D7
:1063D00094023A68B140002A41F007013046B8BF44
:1063E0005242C9B2FFF702FE0020BDE8F08188B931
:1063F0002021B14041F00201C9B23046FFF76FFEE3
:1064000010F4000318BF4FF07F4303433B600020AC
:10641000BDE8F081012C9ED10420BDE8F08160B977
:10642000B54B20201B68884040F0070003EB80003C
:1064300043683B602046BDE8F08101288BD1AE4B1C
:106440003A681B682021B14041F0070403EB840344
:10645000002AB8BF52425A60C9B23046FFF73FFE29
:10646000054600287FF477AF3A68002A3046B8BF67
:106470005242E1B2FFF7BAFD2846BDE8F08158B9B3
:106480002021B14041F00601C9B23046FFF727FE96
:1064900038602046BDE8F08101287FF45CAF202100
:1064A000B14041F0060130461A68C9B2FFF79EFDBF
:1064B0000020BDE8F08168B92021B14041F0100111
:1064C000C9B23046FFF70BFEC0F30420386000204D
:1064D000BDE8F08101287FF43EAF20248C4044F0D9
:1064E0001004E4B221463046FFF7F9FD3B681B0279
:1064F00003F4F85320F4F8521A4330462146FFF7CC
:1065000075FD0020BDE8F08168B92021B14041F05F
:106510001001C9B23046FFF7E2FD00F01F003860FD
:106520002046BDE8F08101287FF415AF20248C407F
:1065300044F01004E4B221463046FFF7D0FD3B683A
:1065400020F01F0203F01F0330461A432146FFF7D5
:106550004DFD0020BDE8F08100287FF45BAF2021D5
:10656000B14041F01501C9B23046FFF7B8FDC0F3A4
:10657000402038602046BDE8F08100287FF44AAF13
:106580002021B14041F01501C9B23046FFF7A7FD07
:10659000C0F3400080F0010038600020BDE8F081C9
:1065A00000287FF437AF2021B14041F01501C9B276
:1065B0003046FFF794FD00F0010080F001003860E4
:1065C0002046BDE8F08168B92021B14041F01401B6
:1065D000C9B23046FFF783FDC0F340003860204663
:1065E000BDE8F08101287FF4B6AE20248C4044F051
:1065F0001404E4B221463046FFF771FD3B685B00AE
:1066000003F0020320F002021A4330462146FFF74E
:10661000EDFC0020BDE8F08168B92021B14041F0D7
:106620001401C9B23046FFF75AFD00F0010038608E
:106630000020BDE8F08101287FF48DAE20248C403D
:1066400044F01404E4B221463046FFF748FD3B68AD
:1066500020F0010203F0010330461A432146FFF700
:10666000C5FC0020BDE8F08158B92021B14041F0BF
:106670001401C9B23046FFF732FD38602046BDE84C
:10668000F08101287FF467AE2021B14041F0140170
:1066900030461A68C9B2FFF7A9FC0020BDE8F081B6
:1066A00058B92021B14041F00401C9B23046FFF78A
:1066B00016FD38602046BDE8F08101287FF44BAE1E
:1066C0002021B14041F0040130461A68C9B2FFF7F9
:1066D0008DFC0020BDE8F08180B92021B14041F05F
:1066E0000501C9B23046FFF7FAFC38600020BDE86A
:1066F000F08100BFEC4BFF1FE84BFF1F01287FF428
:106700002AAE2021B14041F0050130461A68C9B2D5
:10671000FFF76CFC0020BDE8F08158B92021B140A2
:1067200041F00801C9B23046FFF7D9FC3860204675
:10673000BDE8F08101287FF40EAE2021B14041F088
:10674000080130461A68C9B2FFF750FC0020BDE8C6
:10675000F08158B92021B14041F00A01C9B2304658
:10676000FFF7BDFC38602046BDE8F08101287FF4CA
:10677000F2AD2021B14041F00A0130461A68C9B299
:10678000FFF734FC0020BDE8F08158B92021B1406A
:1067900041F00301C9B23046FFF7A1FC3860002088
:1067A000BDE8F08101287FF4D6AD2021B14041F051
:1067B000030130461A68C9B2FFF718FC0020BDE893
:1067C000F08158B92021B14041F00B01C9B23046E7
:1067D000FFF785FC38602046BDE8F08101287FF492
:1067E000BAAD2021B14041F00B0130461A68C9B260
:1067F000FFF7FCFB0020BDE8F08158B92021B14033
:1068000041F00C01C9B23046FFF769FC3860204600
:10681000BDE8F08101287FF49EAD2021B14041F018
:106820000C0130461A68C9B2FFF7E0FB0020BDE852
:10683000F0815CB92021B14041F01101C9B230466C
:10684000FFF74DFC38600020BDE8F081012C7FF49B
:1068500082AD2021B14041F0110130463A68C9B201
:10686000FFF7C4FB0020BDE8F08158B92021B140FA
:1068700041F01201C9B23046FFF731FC3860002008
:10688000BDE8F08101287FF466AD2021B14041F0E0
:10689000120130461A68C9B2FFF7A8FB0020BDE814
:1068A000F08158B92021B14041F01301C9B23046FE
:1068B000FFF715FC38602046BDE8F08101287FF421
:1068C0004AAD2021B14041F0130130461A68C9B2E7
:1068D000FFF78CFB0020BDE8F08168B9090141F0A9
:1068E0006C0101F0FC013046FFF7F9FBC0F380407A
:1068F00038602046BDE8F08101287FF42CAD0C0102
:1069000044F06C04E4B221463046FFF7E8FB3B68F4
:106910009B0403F4802320F480221A43304621464E
:10692000FFF764FB0020BDE8F08100287FF472AD22
:10693000CF4B53F821303B600020BDE8F08188B98F
:10694000090141F06C0101F0FC013046FFF7C7FB83
:106950004FF48073C0F3036043FA00F038602046C0
:10696000BDE8F08101287FF4F6AC1B68102B1FD026
:106970000CDC022B18D003DC012B1FD108231FE0F5
:10698000042B13D0082B19D1052319E0402B11D06B
:1069900003DC202B12D1032312E0802B0CD0B3F5A3
:1069A000807F0BD100230BE0072309E0062307E0DB
:1069B000042305E0022303E0386002E04FF0FF33D8
:1069C0003B603B6801333FF4C6AC340144F06C04D7
:1069D000E4B221463046FFF782FB3B681B0603F01A
:1069E000706320F070621A4330462146FFF7FEFACA
:1069F0000020BDE8F08168B9090141F06C0101F0A7
:106A0000FC013046FFF76BFBC0F3C1303860204615
:106A1000BDE8F08101287FF49EAC0C0144F06C04C9
:106A2000E4B221463046FFF75AFB3B68DB0303F430
:106A3000C03320F4C0321A4330462146FFF7D6FA5D
:106A40000020BDE8F08168B9090141F06C0101F056
:106A5000FC013046FFF743FBC0F380303860002074
:106A6000BDE8F08101287FF476AC0C0144F06C04A1
:106A7000E4B221463046FFF732FB3B689B0303F448
:106A8000804320F480421A4330462146FFF7AEFA95
:106A90000020BDE8F08168B9090141F06C0101F006
:106AA000FC013046FFF71BFBC0F300303860204686
:106AB000BDE8F08101287FF44EAC0C0144F06C0479
:106AC000E4B221463046FFF70AFB3B681B0303F4A0
:106AD000805320F480521A4330462146FFF786FA4D
:106AE0000020BDE8F08148BB0D0145F06C05EDB21A
:106AF00029463046FFF7F3FAC0F38038294630467E
:106B0000B8F1000F07D0FFF7EAFAC0F3C3103860FE
:106B10002046BDE8F081FFF7E2FAC0F302103860CA
:106B200029463046FFF7DBFA04057FF514AC3B68D5
:106B300043F008033B604046BDE8F08101287FF444
:106B40000AAC0C0144F06C04E4B221463046FFF775
:106B5000C6FA10F48045214630460FD0FFF7BFFA41
:106B60003B68DB0103F4F06320F4F0621A43304623
:106B70002146FFF73BFA0020BDE8F081FFF7AFFAAE
:106B80003B6813F0080F18BF4FF4006520F4006253
:106B90002A4321463046FFF729FA21463046FFF7BF
:106BA0009EFA3B681B0103F0700320F070021A4349
:106BB00030462146FFF71AFA0020BDE8F08138BBC5
:106BC0000C0144F06C04E4B221463046FFF787FA2A
:106BD00010F480452146304607D0FFF780FAC0F315
:106BE000021038600020BDE8F081FFF778FAC0F3AA
:106BF000C310386021463046FFF771FA00057FF573
:106C0000AAAB3B6843F008033B602846BDE8F0812F
:106C100001287FF4A0AB0C0144F06C04E4B22146DF
:106C20003046FFF75CFA10F48045214630460FD01D
:106C3000FFF755FA3B681B0103F0700320F0700268
:106C40001A4330462146FFF7D1F90020BDE8F08114
:106C5000FFF745FA3B68DB0103F4F06320F4F062D0
:106C60001A4330462146FFF7C1F92846BDE8F081B6
:106C7000EC4BFF1F68B9090141F06C0101F0FC0108
:106C80003046FFF72CFA00F00F0038602046BDE8D0
:106C9000F08101287FF45FAB0C0144F06C04E4B296
:106CA00021463046FFF71BFA3B6820F00F0203F045
:106CB0000F0330461A432146FFF798F90020BDE83C
:106CC000F08168B9090141F06D0101F0FD01304624
:106CD000FFF705FAC0F3C03038602046BDE8F08108
:106CE00001287FF438AB0C0144F06D04E4B2214676
:106CF0003046FFF7F4F93B68DB039BB220F4004217
:106D00001A4330462146FFF771F90020BDE8F081B3
:106D100068B9090141F06D0101F0FD013046FFF74E
:106D2000DEF9C0F3413038602046BDE8F08101282B
:106D30007FF411AB0C0144F06D04E4B221463046FF
:106D4000FFF7CDF93B685B0303F4C04320F4C04276
:106D50001A4330462146FFF749F90020BDE8F0818B
:106D600068B9090141F06D0101F0FD013046FFF7FE
:106D7000B6F9C0F3032038600020BDE8F081012897
:106D80007FF4E9AA0C0144F06D04E4B221463046D8
:106D9000FFF7A5F93B681B0203F4706320F47062EF
:106DA0001A4330462146FFF721F90020BDE8F08163
:106DB00068B9090141F06D0101F0FD013046FFF7AE
:106DC0008EF9C0F3411038602046BDE8F0810128FB
:106DD0007FF4C1AA0C0144F06D04E4B221463046B0
:106DE000FFF77DF93B685B0103F0600320F0600270
:106DF0001A4330462146FFF7F9F80020BDE8F0813C
:106E000068B9090141F06D0101F0FD013046FFF75D
:106E100066F900F00F0038602046BDE8F0810128D7
:106E20007FF499AA0C0144F06D04E4B22146304687
:106E3000FFF755F93B6820F00F0203F00F033046CF
:106E40001A432146FFF7D2F80020BDE8F08168B967
:106E5000090141F06D0101F0FD013046FFF73FF9F6
:106E6000C0F3006038600020BDE8F08101287FF4A5
:106E700072AA0C0144F06D04E4B221463046FFF7DB
:106E80002EF93B681B0603F0807320F080721A43D2
:106E900030462146FFF7AAF80020BDE8F081A8B9E6
:106EA000090141F06D0101F0FD013046FFF717F9CE
:106EB000001410F0400F00F07F0214BF6FF07F034A
:106EC000002313433B602046BDE8F08101287FF496
:106ED00042AA0C0144F06D04E4B221463046FFF7AB
:106EE000FEF83B681B0403F4FE0320F4FE021A4381
:106EF00030462146FFF77AF80020BDE8F08168B9F6
:106F0000090141F06C0101F0FC013046FFF7E7F8A0
:106F1000C0F3404038602046BDE8F08101287FF48E
:106F20001AAA0C0144F06C04E4B221463046FFF783
:106F3000D6F83B685B0403F4003320F400321A43B4
:106F400030462146FFF752F80020BDE8F0810028C6
:106F50007FF460AA090141F06F01C9B23046FFF722
:106F6000BEF8C0F3044038600020BDE8F081A8B945
:106F700020258D406DB245F01401C9B23046FFF7AF
:106F8000AEF841057FF5E7A945F01101C9B23046D9
:106F9000FFF7A5F838602046BDE8F08101287FF4AE
:106FA000DAA920248C4064B244F0110144F01404A6
:106FB0001A683046E4B2C9B2FFF718F821463046E5
:106FC000FFF78DF83B68002B14BF4FF4806300235C
:106FD00020F480621A4330462146FFF707F800206C
:106FE000BDE8F08168B9090141F06C0101F0FC01D4
:106FF0003046FFF774F8C0F3403038600020BDE839
:10700000F08101287FF4A7A90C0144F06C04E4B2DC
:1070100021463046FFF763F83B685B0303F40053F7
:1070200020F400521A4330462146FEF7DFFF0020CD
:10703000BDE8F08168B9090141F06C0101F0FC0183
:107040003046FFF74CF8C0F3035038602046BDE8E7
:10705000F08101287FF47FA90C0144F06C04E4B2B4
:1070600021463046FFF73BF83B681B0503F47003ED
:1070700020F470021A4330462146FEF7B7FF002085
:10708000BDE8F08100287FF4C5A9090141F06F0136
:10709000C9B23046FFF723F8C0F309003860204634
:1070A000BDE8F08158B92021B14041F01901C9B2C1
:1070B0003046FFF714F838602046BDE8F08101281B
:1070C0007FF449A92021B14041F0190130461A68E6
:1070D000C9B2FEF78BFF0020BDE8F08158B920212E
:1070E000B14041F01A01C9B23046FEF7F8FF3860EE
:1070F0000020BDE8F08101287FF42DA92021B140B6
:1071000041F01A0130461A68C9B2FEF76FFF00203D
:10711000BDE8F081E8B979B101294BD1014630468B
:10712000FEF7DDFF00F06000A0F120035842584157
:1071300038602046BDE8F0810846FEF7D0FF00F039
:107140001800A0F110025042504138603046BDE8AE
:10715000F08101287FF4FFA811B1012913D02BE0A1
:107160000846FEF7BCFF3B6820F0180013B140F062
:10717000100201E040F0080200210846FEF736FF49
:107180000020BDE8F08100213046FEF7A8FF3B68F3
:1071900020F0600013B140F0200201E040F0400216
:1071A00000210120FEF722FF0020BDE8F08104202D
:1071B000BDE8F081BDE8F0810020BDE8F08107B5B1
:1071C0000129019205D8024601AB0120FEF7EFFF2D
:1071D00000E0082003B05DF804FB0129134603D842
:1071E00002460020FEF7E3BF0820704708B52221C1
:1071F0000020FEF774FF50B942210120FEF76FFF17
:1072000028B9044B1868BDE808400AF085BC002086
:1072100008BD00BFE84BFF1F70B53D4E3D483E4CDA
:107220000AF0E0FBF5686B6803F58272626003F5B3
:107230009272A26003F57172E26003F5797203F154
:107240006400226103F2044203F22443A3612B6829
:107250006261DB68206098472B68E068DB689847CC
:107260002B68E0689B6998472B6860681B699847A2
:107270002B68A0681B6998472B68A0691B69984711
:107280002B6820691B6998472B6860691B699847C0
:10729000224B32691A606B68214903F531735360E0
:1072A000204B5A690A602049C2F804121F49C2F8EB
:1072B000081201200021107051701D4A1A621D4AE7
:1072C000DA611D4A9A611D4A5A621D4A9A631D4A33
:1072D0005A631D4A9A621D4ADA621D4A9A641D4A1F
:1072E0005A641D4A5A651D4A1A651D4ADA641D4AC8
:1072F0001A661D4ADA6502221A743222DA60DE2228
:107300009A601A4A9A65BDE87040FEF7EDBD00BF6D
:107310000C550200EC4BFF1F5017FF1F844EFF1F40
:10732000E84BFF1FC82EFF1FED710100815E0100B9
:107330007D600100DD600100D9600100D5600100C1
:10734000DB710100BF710100136001008D6101005C
:10735000096001007D610100555E01008D5E010044
:10736000315E0100E95E0100495E0100295F010014
:1073700001289FBF034B53F820300B60002088BFCB
:10738000082070478C4EFF1F014B00225A60704747
:10739000C82EFF1F70B5084E084D336804462A46B4
:1073A000014600200AF00AFC33682A4621460120E3
:1073B000BDE870400AF002BC884EFF1F8C4EFF1FD4
:1073C000014B18680AF045BC884EFF1F012810B514
:1073D000144616D008D302281FD1114B114ADB687E
:1073E00090681B681B6A12E014680D4A0D4BD26846
:1073F000126824B15269D8689047002010BD926984
:10740000F9E7074B074ADB6850681B681B6A984717
:10741000003018BF01202060EFE7042010BD00BF3E
:107420000C5502007817FF1F022804BF0B4B93F87E
:10743000D00020B90A4BDB681B685B690AE00128B1
:107440000BD1064B93F8D030012B06D1044BDB68EF
:107450001B689B69034A106818477047C82EFF1FB6
:107460000C5502007817FF1F70B50020FFF7DCFFF6
:10747000104B114CDD6820682B689B6898472B687F
:1074800060689B6898472B68A0689B6898472B6842
:10749000A0699B6898472B6820699B6898472B6870
:1074A00060699B6898472B68E0689B68BDE87040FE
:1074B000184700BF0C5502007817FF1F2DE9F8434D
:1074C000184C9DF820609DF82450984623680F467C
:1074D0009B68002147F0800091469847236800216F
:1074E0009B6848469847236800219B684046984718
:1074F000236800219B6830469847236828469B688C
:1075000001219847084B1B6848EA092807F07F07C4
:1075100046EA082603EB870745EA06257D60BDE8B5
:10752000F88300BF2451FF1F884EFF1F07B5D3B259
:107530000193C2F307230093C2F30743120EFFF730
:10754000BDFF03B05DF804FB0A4601460020FFF7CB
:10755000EDBF0128F7B505460F4627D8154C044462
:1075600094F8943273B1144B202181401B6841F090
:10757000070103EB8103C9B25A68FFF7D7FF002365
:1075800084F894322026AE4046F00D0100243A469D
:10759000C9B22846FFF7CAFF284601940094234643
:1075A0002246F1B2FFF78AFF204600E0082003B030
:1075B000F0BD00BF8C4EFF1F884EFF1F012873B522
:1075C00005460C4620D82026864084EAE47246F020
:1075D0000701A2EBE472C9B2FFF7A8FF0C4B2B44E2
:1075E000002C4FF0010283F894224FF00004ACBF4E
:1075F0001346022301932846009423462246F1B203
:10760000FFF75CFF204600E0082002B070BD00BF1D
:107610008C4EFF1F0021D1E74942CFE7CEE738B5B6
:10762000234B01F07F04234493F81432DB0705D485
:10763000204B1B6803EB8404606838BD1E4D2B682B
:1076400000219B68204698472B6800219B680846CC
:1076500098472B6800219B68084698472B680021B3
:107660009B68084698472B6801219B680020984733
:107670002B6800219B68204698472B6800219B6857
:10768000084698472B68002104029B6808469847E3
:107690002B680021204304029B68084698472B680A
:1076A000204304029B68012100209847204338BDF5
:1076B0008C4EFF1F884EFF1F2451FF1F10B50C4634
:1076C00001460020FFF7ABFF206010BD38B50D4626
:1076D0002021814041F00101C9B20446FFF79FFF1C
:1076E0002968014429602046BDE8384031E71C2A5A
:1076F0002DE9F34104460E461F4600F03C835DD859
:107700000C2A00F0D6812BD8052A00F0428113D82C
:10771000022A00F0E18007D8002A00F0AE80012A9A
:1077200000F0C58000F0CABE032A00F0F180042AF0
:1077300000F0058100F0C2BE082A00F08C8107D855
:10774000062A00F03B81072A00F05F8100F0B6BEF8
:107750000A2A00F08F810B2A00F09C8100F0AEBE57
:10776000122A00F0718213D80F2A00F0268207D85F
:107770000D2A00F0D5810E2A00F00A8200F09EBE8C
:10778000102A00F02E82112A00F04A8200F096BEE4
:10779000152A00F09A8207D8132A00F06982142A69
:1077A00000F0808200F08ABE172A00F0B982C0F093
:1077B0009F82182A00F0CC8200F080BEAB2A00F035
:1077C000EA842BD8A52A00F0C28313D8A22A00F09D
:1077D000548307D81D2A00F0F1828C2A00F0F6822B
:1077E00000F06CBEA32A00F06B83A42A00F08C8307
:1077F00000F064BEA82A00F0628407D8A62A00F030
:10780000F183A72A00F0398400F058BEA92A00F0BD
:107810007B84AA2A00F09C8400F050BEB52A00F0B8
:10782000808513D8AE2A00F01F8507D8AC2A00F057
:10783000D584AD2A00F0F58400F040BEB32A00F0F4
:107840003F85B42A00F0608500F038BECE2A00F0F3
:107850009C8507D8B62A00F04B82B82A00F0308306
:1078600000F02CBED22A00F0B585D32A00F0C985DD
:10787000D12A40F0238600F095BD50B92021B140B7
:1078800041F00D01C9B23046FFF7C9FE386000F083
:1078900017BE012840F014862021B14041F00D01AF
:1078A0001A68C9B23046FFF741FE00F009BE28B998
:1078B0002021B14041F0010100F079BD012840F0E4
:1078C000FF852021B14041F001011A68C9B230465C
:1078D000FFF72CFE00F0F4BD28B92021B14041F0A3
:1078E000070100F064BD012840F0EA85CA4B0B4453
:1078F000202183F894023A68B140002A41F0070140
:10790000B8BF5242C9B23046FFF710FE00F0D8BDF2
:1079100080B92021B14041F00201C9B23046FFF7E1
:107920007EFE10F4000318BF4FF07F4303433B601B
:1079300000F0C6BD012C00F0C18500F0C1BD50B9FA
:10794000B64B20201B68884040F0070003EB800006
:10795000436800F09CBC012840F0B285AF4B3A6808
:107960001B682021B14041F00704002A03EB840387
:10797000B8BF52425A60C9B23046FFF750FE0028E5
:1079800040F09E853A68002AB8BF5242E1B200F04A
:1079900091BD28B92021B14041F0060100F007BD9A
:1079A000012840F08D852021B14041F006011A6880
:1079B000C9B23046FFF7BAFD00F082BD60B92021A0
:1079C000B14041F01001C9B23046FFF728FEC0F3C4
:1079D0000720386000F074BD012840F07185202434
:1079E0008C4044F01004E4B221463046FFF717FE05
:1079F000C3B201933B7800930022C0F307432146B2
:107A00003046FFF75BFD00F05BBD50B92021B1406F
:107A100041F01001C9B23046FFF701FEC0B200F0DC
:107A2000CABC012840F04C8520248C4044F010044E
:107A3000E4B221463046FFF7F2FD3B780193C0F3F4
:107A4000072300930022C0F3074321463046FFF787
:107A500035FD00F035BD00287FF46CAF2021B1402A
:107A600041F01501C9B23046FFF7D9FDC0F34020FF
:107A700000F0A1BC00287FF45DAF2021B14041F0AF
:107A80001501C9B23046FFF7CAFDC0F340003860A7
:107A900000F016BD00287FF44DAF2021B14041F029
:107AA0001501C9B23046FFF7BAFD00F0010000F041
:107AB00082BC58B92021B14041F01401C9B230460E
:107AC000FFF7ADFDC0F3400000F075BC012840F0A9
:107AD000F78420248C4044F01404E4B2214630465C
:107AE000FFF79DFD3B68002BCCBF0223002320F055
:107AF00002021A4321463046FFF718FD2146304660
:107B0000FFF78DFD3B68022B20F008020CBF082315
:107B100000231A4321463046FFF708FD00F0D0BC91
:107B200060B92021B14041F01401C9B23046FFF7DD
:107B300076FD00F00100386000F0C2BC012840F082
:107B4000BF8420248C4044F01404E4B22146304623
:107B5000FFF765FD3A6820F00100002AD4BF024615
:107B600040F0010221463046FFF7E0FC2146304656
:107B7000FFF755FD3B68022B20F004020CBF0423E5
:107B800000231A4321463046FFF7D0FC00F098BC92
:107B900028B92021B14041F0140100F008BC0128AF
:107BA00040F08E842021B14041F014011A68C9B21E
:107BB0003046FFF7BBFC00F083BC20B92021B14068
:107BC00041F00401F3E3012840F07A842021B14020
:107BD00041F004011A68C9B23046FFF7A7FC00F073
:107BE0006FBC50B92021B14041F00501C9B2304607
:107BF000FFF715FD386000F063BC012840F0608499
:107C00002021B14041F005011A68C9B23046FFF7A2
:107C10008DFC00F055BC00BF8C4EFF1F884EFF1F2F
:107C200020B92021B14041F00801C0E3012840F013
:107C300047842021B14041F008011A68C9B230469A
:107C4000FFF774FC00F03CBC20B92021B14041F0AA
:107C50000A01ACE3012840F033842021B14041F017
:107C60000A011A68C9B23046FFF760FC00F028BC70
:107C700050B92021B14041F00301C9B23046FFF7AD
:107C8000CEFC386000F01CBC012840F01984202193
:107C9000B14041F003011A68C9B23046FFF746FC13
:107CA00000F00EBC20B92021B14041F00B017EE371
:107CB000012840F005842021B14041F00B011A68F1
:107CC000C9B23046FFF732FCFAE320B92021B140B7
:107CD00041F00C016BE3012840F0F2832021B14018
:107CE00041F00C011A68C9B23046FFF71FFCE7E308
:107CF0004CB92021B14041F01101C9B23046FFF723
:107D00008EFC3860DCE3012C40F0DA832021B140A6
:107D100041F011013A68C9B23046FFF707FCCFE3E2
:107D200048B92021B14041F01201C9B23046FFF7F5
:107D300076FC3860C4E3012840F0C2832021B140C2
:107D400041F012011A68C9B23046FFF7EFFBB7E302
:107D500020B92021B14041F0130128E3012840F06F
:107D6000AF832021B14041F013011A68C9B23046F7
:107D7000FFF7DCFBA4E350B9090141F06C0101F00D
:107D8000FC013046FFF74BFCC0F3804013E30128B1
:107D900040F096830C0144F06C04E4B22146304676
:107DA000FFF73DFC3B689B0403F4802320F4802212
:107DB0001A4321463046FFF7B9FB81E300287FF4E0
:107DC000B9ADC54B53F821303B6079E370B9090177
:107DD00041F06C0101F0FC013046FFF720FC4FF44C
:107DE000807300F00F0043FA00F0E4E2012840F055
:107DF00067831B68102B1FD00CDC022B18D003DC10
:107E0000012B1FD108231FE0042B13D0082B19D1FD
:107E1000052319E0402B11D003DC202B12D10323C2
:107E200012E0802B0CD0B3F5807F0BD100230BE048
:107E3000072309E0062307E0042305E0022303E00B
:107E4000386002E04FF0FF333B603B68013300F0E5
:107E50003783340144F06C04E4B221463046FFF726
:107E6000DEFB3B681B0603F0706320F070621A4370
:107E700021463046FFF75AFB22E350B9090141F091
:107E80006C0101F0FC013046FFF7C9FBC0F3C130C3
:107E900091E2012840F014830C0144F06C04E4B238
:107EA00021463046FFF7BBFB3B68DB0303F4C033DE
:107EB00020F4C0321A4321463046FFF737FBFFE279
:107EC0005CB9310141F06C0101F0FC013046FFF773
:107ED000A6FBC0F340303860F2E2012C40F0F082A3
:107EE000340144F06C04E4B221463046FFF797FBBE
:107EF0003B685B0303F4005320F400521A4321460D
:107F00003046FFF713FBDBE250B9090141F06C0189
:107F100001F0FC013046FFF782FBC0F300304AE27B
:107F2000012840F0CD820C0144F06C04E4B22146FB
:107F30003046FFF774FB3B681B0303F4805320F4C7
:107F400080521A4321463046FFF7F0FAB8E20D019D
:107F500045F06C05EDB229463046FFF760FBC0F3F3
:107F6000803874B929463046B8F1000F04D0FFF7C5
:107F700056FBC0F3C3101EE2FFF751FBC0F3021023
:107F800054E0012C40F09C8229463046B8F1000FA5
:107F90000DD0FFF744FB3B68DB0103F4F06320F4F2
:107FA000F0621A4329463046FFF7C0FA88E2FFF72D
:107FB00036FB3B6813F0080F14BF4FF40063002337
:107FC00020F400621A4329463046FFF7AFFA2946EB
:107FD0003046FFF724FB3B681B0103F0700320F0E1
:107FE000700244E00D0145F06C05EDB229463046C3
:107FF000FFF715FBC0F38038DCB929463046B8F1ED
:10800000000F05D0FFF70BFBC0F30210386057E2FA
:10801000FFF705FBC0F3C310386029463046FFF771
:10802000FEFA3B68000A00F008001843386040463A
:1080300047E2012C40F0448229463046B8F1000F57
:108040000DD0FFF7ECFA3B681B0103F0700320F042
:1080500070021A4329463046FFF768FA30E2FFF70C
:10806000DEFA3B68DB0103F4F06320F4F0621A43AC
:1080700029463046FFF75AFAD9E750B9090141F0CD
:108080006C0101F0FC013046FFF7C9FA00F00F0067
:1080900091E1012840F014820C0144F06C04E4B238
:1080A00021463046FFF7BBFA3B6820F00F0203F091
:1080B0000F031A4321463046FFF738FA00E268B949
:1080C000090141F06D0101F0FD013046FFF7A7FA0B
:1080D000C0F3C0306FE100BF8C4EFF1F012840F09D
:1080E000EF810C0144F06D04E4B221463046FFF705
:1080F00096FA3B68DB039BB220F400421A43214608
:108100003046FFF713FADBE158B9090141F06D0180
:1081100001F0FD013046FFF782FAC0F341303860CC
:10812000CEE1012840F0CC810C0144F06D04E4B2B2
:1081300021463046FFF773FA3B685B0303F4C04304
:1081400020F4C0421A4321463046FFF7EFF9B7E169
:1081500050B9090141F06D0101F0FD013046FFF712
:108160005EFAC0F3032026E1012840F0A9810C014A
:1081700044F06D04E4B221463046FFF750FA3B6804
:108180001B0203F4706320F470621A4321463046E8
:10819000FFF7CCF994E150B9090141F06D0101F00C
:1081A000FD013046FFF73BFAC0F3411003E101281F
:1081B00040F086810C0144F06D04E4B22146304663
:1081C000FFF72DFA3B685B0103F0600320F06002CB
:1081D0001A4321463046FFF7A9F971E158B9090160
:1081E00041F06D0101F0FD013046FFF718FA00F093
:1081F0000F00386064E1012840F062810C0144F016
:108200006D04E4B221463046FFF709FA3B6820F0DE
:108210000F0203F00F031A4321463046FFF786F999
:108220004EE150B9090141F06D0101F0FD01304608
:10823000FFF7F5F9C0F30060BDE0012840F0408190
:108240000C0144F06D04E4B221463046FFF7E7F933
:108250003B681B0603F0807320F080721A432146AE
:108260003046FFF763F92BE198B9090141F06D0140
:1082700001F0FD013046FFF7D2F9001410F0400F75
:1082800000F07F0214BF6FF07F03002313433B60B5
:1082900092E0012840F014810C0144F06D04E4B236
:1082A00021463046FFF7BBF93B681B0403F4FE038D
:1082B00020F4FE021A4321463046FFF737F9FFE06B
:1082C00058B9090141F06C0101F0FC013046FFF79B
:1082D000A6F9C0F340403860F2E0012840F0F08099
:1082E0000C0144F06C04E4B221463046FFF797F9E4
:1082F0003B685B0403F4003320F400321A43214648
:108300003046FFF713F9DBE000287FF413AB0901D7
:1083100041F06F01C9B23046FFF781F9C0F3044064
:1083200049E080B920258D406DB245F01401C9B2F5
:108330003046FFF774F9C0F3802010B145F0110109
:1083400035E03860BDE0012840F0BA8020248C4040
:1083500064B244F0110144F014041A683046E4B2E7
:10836000C9B2FFF7E3F821463046FFF758F93B68FA
:10837000002B20F4806214BF4FF4806300231A4363
:1083800021463046FFF7D2F89AE000287FF4D2AABF
:10839000090141F06F01C9B23046FFF740F9C0F35F
:1083A000090008E050B92021B14041F01901C9B2DB
:1083B0003046FFF734F93860204682E001287FD14B
:1083C0002021B14041F019011A68C9B23046FFF7C7
:1083D000ADF875E048B92021B14041F01A01C9B2A9
:1083E0003046FFF71CF938606AE0012868D1202187
:1083F000B14041F01A011A68C9B23046FFF796F849
:108400005EE0C0B961B101295AD101463046FFF79B
:1084100006F900F06000A0F1200358425841CAE775
:108420000846FFF7FCF800F01800A0F110025042D7
:108430005041386044E0012842D1F9B101293FD1CF
:1084400000213046FFF7EBF83B68002B14BF2023D8
:10845000002320F020021A4300213046FFF766F87F
:1084600000213046FFF7DBF83B68002B20F040028C
:108470000CBF402300231A4300211BE00846FFF7EE
:10848000CEF83B68002B0CBF0823002320F0080225
:108490001A4331463046FFF749F831463046FFF778
:1084A000BEF83B68002B20F0100214BF10230023FD
:1084B0001A4331463046FFF739F801E0042000E066
:1084C000002002B0BDE8F08107B50129019205D86E
:1084D000024601AB0120FFF70AF900E0082003B0D3
:1084E0005DF804FB0129134603D802460020FFF77C
:1084F000FEB80820704708B522210020FFF78FF84A
:1085000050B942210120FFF78AF828B9034B1868B7
:10851000BDE8084009F094BB002008BD884EFF1F4D
:1085200070B53D4E3D483E4C09F008FBF5686B6860
:1085300003F58272626003F59272A26003F57172B4
:10854000E26003F5797203F16400226103F20442F0
:1085500003F22443A3612B686261DB6820609847C3
:108560002B68E068DB6898472B68E0689B69984750
:108570002B6860681B6998472B68A0681B6998473F
:108580002B68A0691B6998472B6820691B6998476D
:108590002B6860691B699847224B32691A606B68C7
:1085A000214903F531735360204B5A690A60204911
:1085B000C2F804121F49C2F80812012111700021EB
:1085C00051701D4A1A621D4ADA611D4A9A611D4A9C
:1085D0005A621D4A9A631D4A5A631D4A9A621D4A8D
:1085E000DA621D4A9A641D4A5A641D4A5A651D4A38
:1085F0001A651D4ADA641D4A1A661D4ADA65322276
:10860000DA6002204FF48C729A601874194A9A65E5
:10861000BDE87040FEF708BF0C5502008C4EFF1FEE
:108620007817FF1F2451FF1F884EFF1FC82EFF1F02
:10863000F7840100C1730100BD7501001D760100C2
:108640001976010015760100E5840100C984010056
:1086500053750100CD76010049750100BD7601001A
:1086600095730100CD73010071730100297401003D
:10867000897301006974010018B9034B1B680B6012
:1086800070470820704700BF2C51FF1F014B00228C
:108690005A607047C82EFF1F0428F8B5144677D0DB
:1086A00007D801283BD011D3022856D0032864D024
:1086B0000AE0062800F09780C0F08E80072800F0BE
:1086C0009E80FC2800F0A7800420F8BD136833F0DA
:1086D000030240F0B28013F0010F594D594E03D000
:1086E000F3681B681B6906E0F76868683B68DB682D
:1086F00098473B689B6968689847206810F00204B7
:1087000004D0F36828681B681B6935E0F6682868A0
:108710003368DB689847336828689B6935E01368DD
:1087200044F62062934200F3888042F21072934232
:10873000444A434BD268586A1268CCBF5269926966
:108740009047206842F2117290FBF2F302FB130093
:108750003D4B80B29B6898470FE01468394B74B169
:10876000DC686068236800F5F270DB68984723686E
:1087700060689B6900F5F27098470020F8BDDB68DF
:1087800058681B689B6800F5F27098472046F8BD52
:1087900016682B4D2B4B4EB1012E11D1DF68286985
:1087A0003B68DB6898473B685B6906E0DF682869DF
:1087B0003B68DB6898473B689B692869984709E0F4
:1087C000DE68286933681B699847336828691B6A23
:1087D000984706462660D0E71A4B194ADB68D069ED
:1087E0001B681B6A05E0174B154ADB68106A1B689B
:1087F0001B6A9847003018BF01202060BDE713684E
:10880000104AD268012B12680D4B0CBF5269926955
:1088100098699047B1E71468094D0A4B44B1DC6888
:1088200028692368DB689847236828699B69A3E760
:10883000DB6828691B681B69A7E71020F8BD00BF2B
:10884000A017FF1F0C550200C409FF1F1C4B70B579
:10885000DD681C4C2B68A0689B6998472B68A06A50
:108860009B6898472B68606A9B6898472B68E0680C
:108870009B6898472B6820699B6898472B686069BC
:108880009B6898472B6820689B6898472B686068AE
:108890009B6898472B68E0699B6898472B68206A1B
:1088A0009B6898472B68A0699B6898472B68A068CD
:1088B0009B689847044BBDE870405B68184700BF51
:1088C0000C550200A017FF1FC409FF1F034B044AE9
:1088D0001B680146002007F08EBA00BF2851FF1F19
:1088E0002C51FF1F014B186807F0BDBA2851FF1F1C
:1088F000022804BF0B4B93F8D00020B90A4BDB6869
:108900001B685B690AE001280BD1064B93F8D03055
:10891000012B06D1044BDB681B689B69034A9068F6
:1089200018477047C82EFF1F0C550200A017FF1FE5
:108930002DE9F0471C4D9DF820709DF82460994664
:1089400055F82030044688469B68002148F0800096
:108950009246984755F8243000219B685046984726
:1089600055F8243000219B684846984755F8243034
:1089700000219B683846984755F8243030469B685C
:1089800001219847094B53F8243049EA0A2908F095
:108990007F0847EA092703EB880846EA0726C8F854
:1089A0000460BDE8F08700BFB853FF1F2851FF1FC8
:1089B00007B5D3B20193C2F307230093C2F3074371
:1089C000120EFFF7B5FF03B05DF804FB0A4601463F
:1089D0000020FFF7EDBF38B50D46044690B90246BA
:1089E0002021FFF7E5FF084B1B682046D3F8A020A5
:1089F0002721FFF7DDFF20462A462D21FFF7D8FF6C
:108A0000204638BD082038BD2851FF1F37B50D4618
:108A10000446A0B981EAE172A2EBE1722721FFF7D7
:108A2000C7FF002DACBF0123022301932046009411
:108A3000234622462021FFF77BFF204600E0082046
:108A400003B030BD0021E1E74942DFE7DEE770B562
:108A50002B4A4FF4237301F07F0403FB00232344CC
:108A6000054693F80C32DB0706D4264B53F820302A
:108A700003EB8404606870BD234E56F8203000215B
:108A80009B682046984756F8253000219B68084689
:108A9000984756F8253000219B680846984756F8B5
:108AA000253000219B680846984756F8253001215B
:108AB0009B680020984756F8253000219B68204687
:108AC000984756F8253000219B680846984756F885
:108AD0002530002104029B680846984756F8253047
:108AE0000021204304029B680846984756F8253029
:108AF000204304029B68012100209847204370BD59
:108B00002C51FF1F2851FF1FB853FF1F10B50C46F3
:108B100001460020FFF79BFF206010BD38B50C46D2
:108B2000054648B92121FFF792FF216801442160E1
:108B30002846BDE838404EE7082038BD8C2AF8B5F5
:108B400005460C461E4600F0698359D80E2A00F0EF
:108B5000F98127D8062A00F0418111D8022A00F0B5
:108B6000DD8007D8002A00F0B080012A00F0C38021
:108B700000F056BF042A00F0F88040F2E2801AE1CB
:108B80000A2A00F0768107D8072A00F04781082AD0
:108B900000F0638100F044BF0C2A00F0898140F2AC
:108BA0007881AAE1152A00F0598211D8112A00F023
:108BB000058207D80F2A00F0D981102A00F0EA8137
:108BC00000F02EBF132A00F0218240F20B8231E226
:108BD0001C2A00F0B88209D8182A00F080821B2ACB
:108BE00000F09182172A40F01B874DE2212A00F005
:108BF000D682222A00F0F2821D2A40F01187C2E2BA
:108C0000B32A00F039852CD8A82A00F05D8412D848
:108C1000A42A00F0918307D8A22A00F05183A32A46
:108C200000F06C8300F0FCBEA62A00F0EB8340F25B
:108C3000A18300F02CBCAB2A00F09F8407D8A92A9E
:108C400000F05F84AA2A00F07A8400F0E9BEAD2A21
:108C500000F0CE84C0F0AF84AE2A00F0E78400F0CC
:108C6000DFBEBB2A00F0018615D8B62A00F0708559
:108C700007D8B42A00F01E85B52A00F0278500F039
:108C8000CFBEB92A00F0AA8500F2C685B82A00F046
:108C9000878500F0C5BECC2A00F071860AD8BF2AAD
:108CA00000F02A86C02A00F04986BC2A40F0B88627
:108CB00000F008BED12A00F08C86D22A00F09E86F1
:108CC000CE2A40F0AD8600F078BE38B92D2120467E
:108CD000FFF7BDFE0027306000F0A9BE012802D0DA
:108CE000002700F0A4BE1A682D212046FFF760FE81
:108CF000002700F09CBE38B921212046FFF7A7FECF
:108D00002F46306000F093BE0128E9D11A68212176
:108D10002046FFF74DFE002700F089BE38B9272115
:108D20002046FFF794FE2F46306000F080BE0128F9
:108D3000D6D11A6827212046FFF73AFE002700F017
:108D400076BE68B922212046FFF781FE10F40003A9
:108D500018BF4FF07F43034333602F4600F067BED8
:108D6000012DBDD1042700F062BE40B9C54B53F8B8
:108D70002130D3F8A0303360002700F058BE01281E
:108D8000AED1C04B53F821203368002BB8BF5B42F3
:108D9000C2F8A03020212046FFF759FE07460028E0
:108DA0009ED13268002AB8BF524227212046FFF7E1
:108DB000FFFD00F03CBE38B926212046FFF747FEF4
:108DC0002F46306000F033BE012889D11A68262171
:108DD0002046FFF7EDFD002700F029BE48B910211D
:108DE0002046FFF734FEC0F3042030602F4600F029
:108DF0001EBE01287FF474AF10212046FFF727FE26
:108E000033681B0203F4F85320F4F8521A4310217C
:108E10002046FFF7CDFD002700F009BE48B910211C
:108E20002046FFF714FE00F01F003060002700F01E
:108E3000FEBD01287FF454AF10212046FFF707FE46
:108E4000336820F01F0203F01F031A43102120464D
:108E5000FFF7AEFD002700F0EABD002880D13521E4
:108E60002046FFF7F4FDC0F3402030602F4600F0AD
:108E7000DEBD00287FF474AF35212046FFF7E7FD03
:108E800010F0020F0CBF0123002333602F4600F0C7
:108E9000CEBD00287FF464AF35212046FFF7D7FD13
:108EA00000F0010080F0010030602F4600F0BFBDEF
:108EB00048B934212046FFF7CAFDC0F340003060B6
:108EC000002700F0B4BD01287FF40AAF342120460A
:108ED000FFF7BDFD37683FB940F00202342120465C
:108EE000FFF766FD00F0A3BD20F00202342120460A
:108EF000FFF75EFD002700F09ABD48B934212046F7
:108F0000FFF7A5FD00F0010030602F4600F08FBD97
:108F100001287FF4E5AE34212046FFF798FD37683D
:108F20003FB940F0010234212046FFF741FD00F037
:108F30007EBD20F0010234212046FFF739FD0027D5
:108F400000F075BD38B934212046FFF780FD2F466B
:108F5000306000F06CBD01287FF4C2AE1A68342185
:108F60002046FFF725FD002700F061BD38B9242118
:108F70002046FFF76CFD0027306000F058BD012847
:108F80007FF4AEAE1A6824212046FFF711FD0027BA
:108F900000F04DBD38B925212046FFF758FD2F467A
:108FA000306000F044BD01287FF49AAE1A68252194
:108FB0002046FFF7FDFC002700F039BD38B9282115
:108FC0002046FFF744FD2F46306000F030BD0128F9
:108FD0007FF486AE1A6828212046FFF7E9FC0027B7
:108FE00000F025BD38B92A212046FFF730FD2F4675
:108FF000306000F01CBD01287FF472AE1A682A218F
:109000002046FFF7D5FC002700F011BD38B9232119
:109010002046FFF71CFD0027306000F008BD012846
:109020007FF45EAE1A6823212046FFF7C1FC0027BB
:1090300000F0FDBC38B92B212046FFF708FD2F4674
:10904000306000F0F4BC01287FF44AAE1A682B218E
:109050002046FFF7ADFC002700F0E9BC38B92C2111
:109060002046FFF7F4FC2F46306000F0E0BC0128FA
:109070007FF436AE1A682C212046FFF799FC0027B2
:1090800000F0D5BC2851FF1F90B915212046FFF7ED
:10909000DEFCC64B38B14FF08072B2FBF0F0984264
:1090A00028BF184600E018463060002700F0BFBC1B
:1090B00001287FF415AE1A68BC493AB14FF08073AD
:1090C00093FBF2F28A42A8BF0A4600E00A463260E9
:1090D00015212046FFF76CFC002700F0A8BC38B92A
:1090E00033212046FFF7B3FC0027306000F09FBC1F
:1090F00001287FF4F5AD1A6833212046FFF758FCAC
:10910000002700F094BC48B96C212046FFF79FFC73
:10911000C0F3C04030602F4600F089BC01287FF4C6
:10912000DFAD6C212046FFF792FC3368DB0403F4CB
:10913000002320F400221A436C212046FFF738FC5C
:10914000002700F074BC48B96C212046FFF77FFC73
:10915000C0F3804030602F4600F069BC01287FF4E6
:10916000BFAD6C212046FFF772FC33689B0403F40B
:10917000802320F480221A436C212046FFF718FC3C
:10918000002700F054BC00287FF4EAAD4FF42373AD
:109190005C43874B1B593360074600F048BC48B915
:1091A00000212046FFF753FC00F00100306000274B
:1091B00000F03DBC01287FF493AD00212046FFF76D
:1091C00046FC336820F0010203F001031A4300213A
:1091D0002046FFF7EDFB002700F029BC48B9014607
:1091E0002046FFF734FCC0F3400030602F4600F00B
:1091F0001EBC01287FF474AD00212046FFF727FC38
:1092000033685B0003F0020320F002021A430021DE
:109210002046FFF7CDFB002700F009BC60B96C21A8
:109220002046FFF714FC4FF48073C0F3036043FA49
:1092300000F030602F46FAE301287FF451AD1B683F
:10924000102B1FD00CDC022B18D003DC012B1FD1FC
:1092500008231FE0042B13D0082B19D1052319E094
:10926000402B11D003DC202B12D1032312E0802BE2
:109270000CD0B3F5807F0BD100230BE0072309E06E
:10928000062307E0042305E0022303E0306002E048
:109290004FF0FF3333603368013300F0C3836C2138
:1092A0002046FFF7D4FB33681B0603F0706320F001
:1092B00070621A436C212046FFF77AFB0027B6E361
:1092C00040B96C212046FFF7C2FBC0F3C1303060CB
:1092D0000027ACE301287FF403AD6C212046FFF7A3
:1092E000B6FB3368DB0303F4C03320F4C0321A4307
:1092F0006C212046FFF75CFB002798E340B96C2106
:109300002046FFF7A4FBC0F3803030602F468EE389
:1093100001287FF4E5AC6C212046FFF798FB336809
:109320009B0303F4804320F480421A436C212046BF
:10933000FFF73EFB00277AE340B96C212046FFF798
:1093400086FBC0F3003030602F4670E301287FF4C5
:10935000C7AC6C212046FFF77AFB33681B0303F48C
:10936000805320F480521A436C212046FFF720FBE3
:1093700000275CE36C212046FFF769FBD5B910F4A8
:10938000804708D06C212046FFF761FBC0F3C31073
:1093900030602F464BE3C0F3021300F40060034338
:1093A00014BF08230023336041E300BFFFFF0F0019
:1093B0002C51FF1F012D7FF493AC10F4804710D087
:1093C0006C212046FFF743FB3368DB0103F4F063B5
:1093D00020F4F0621A436C212046FFF7E9FA0027D7
:1093E00025E3326811074CBF40F4006020F40060B0
:1093F000120120F07000D2B202436C212046FFF728
:10940000D7FA14E36C212046FFF721FBADB910F425
:10941000804708D06C212046FFF719FBC0F30210EB
:109420003060002703E3C0F3C31300F4006003437C
:1094300014BF082300233360F9E2012D7FF450AC00
:109440006C212046FFF703FB10F480474FF06C01BE
:1094500020460ED0FFF7FBFA33681B0103F07003C0
:1094600020F070021A436C212046FFF7A1FA002772
:10947000DDE2FFF7ECFA3368DB0103F4F06320F47C
:10948000F0621A436C212046FFF792FACFE240B90E
:109490006C212046FFF7DBFA00F00F0030602F460A
:1094A000C5E201287FF41CAC6C212046FFF7CFFAFF
:1094B000336820F00F0203F00F031A436C2120469B
:1094C000FFF776FA0027B2E240B96D212046FFF798
:1094D000BEFAC0F3C03030602F46A8E201287FF406
:1094E000FFAB6D212046FFF7B2FA3368DB039BB276
:1094F00020F400421A436D212046FFF759FA002755
:1095000095E240B96D212046FFF7A1FAC0F3413042
:10951000306000278BE201287FF4E2AB6D2120460A
:10952000FFF795FA33685B0303F4C04320F4C042AD
:109530001A436D212046FFF73BFA002777E240B936
:109540006D212046FFF783FAC0F3032030602F46D9
:109550006DE201287FF4C4AB6D212046FFF777FA56
:1095600033681B0203F4706320F470621A436D21A8
:109570002046FFF71DFA002759E240B96D21204629
:10958000FFF765FAC0F3411030602F464FE2012823
:109590007FF4A6AB6D212046FFF759FA33685B01D3
:1095A00003F0600320F060021A436D212046FFF7AC
:1095B000FFF900273BE240B96D212046FFF747FA4B
:1095C00000F00F0030602F4631E201287FF488ABB5
:1095D0006D212046FFF73BFA336820F00F0203F0BD
:1095E0000F031A436D212046FFF7E2F900271EE220
:1095F00040B96D212046FFF72AFAC0F300603060C1
:10960000002714E201287FF46BAB6D212046FFF7A1
:109610001EFA33681B0603F0807320F080721A4331
:109620006D212046FFF7C4F9002700E280B96D21C3
:109630002046FFF70CFA001410F0400F00F07F02F4
:1096400014BF6FF07F030023134333602F46EEE116
:1096500001287FF445AB6D212046FFF7F8F9336808
:109660001B0403F4FE0320F4FE021A436D2120467E
:10967000FFF79EF90027DAE140B96C212046FFF799
:10968000E6F9C0F3404030602F46D0E101287FF476
:1096900027AB6C212046FFF7DAF933685B0403F44B
:1096A000003320F400321A436C212046FFF780F982
:1096B0000027BCE100287FF453AB6F212046FFF761
:1096C000C6F9C0F3044030600027B0E1D0B93421BE
:1096D0002046FFF7BCF9430511D514212046FFF7BA
:1096E000B6F9C04B38B14FF08072B2FBF0F098423F
:1096F00028BF184600E018463060002797E1356023
:109700002F4694E101287FF4EBAA34212046FFF78D
:109710009EF93268920220F4806002F48062024373
:1097200034212046FFF744F9326842B14FF080738C
:1097300093FBF2F29A4208BF6FF07F4201E06FF0B4
:109740007F42326014212046FFF732F900276EE194
:1097500088B914212046FFF77AF9A24B38B14FF0AF
:109760008072B2FBF0F0984228BF184600E018461D
:10977000306000275BE101287FF4B2AA1A6842B189
:109780004FF0807393FBF2F2964B9A42C8BF1A4691
:1097900000E0944A14212046FFF70AF9002746E129
:1097A00040B96C212046FFF752F9C0F340303060D9
:1097B0002F463CE101287FF493AA6C212046FFF755
:1097C00046F933685B0303F4005320F400521A4354
:1097D0006C212046FFF7ECF8002728E140B96C2106
:1097E0002046FFF734F9C0F30350306000271EE134
:1097F00001287FF475AA6C212046FFF728F9336809
:109800001B0503F4700320F470021A436C212046F8
:10981000FFF7CEF800270AE188B913212046FFF7A9
:1098200016F9704B38B14FF08072B2FBF0F09842ED
:1098300028BF184600E0184630600027F7E00128EE
:109840007FF44EAA1A6867493AB14FF0807393FBD0
:10985000F2F28A42A8BF0A4600E00A4632601321AB
:109860002046FFF7A5F80027E1E040B97021204627
:10987000FFF7EDF8C0F3072030602F46D7E001284E
:109880007FF42EAA70212046FFF7E1F83268120219
:1098900020F47F4092B2024370212046FFF788F8FF
:1098A00000212046FFF7D3F83368002B20F0040294
:1098B00014BF042300231A4300212046FFF778F841
:1098C0000027B4E038B970212046FFF7C0F8C0B2D5
:1098D00030602F46ABE001287FF402AA70212046B9
:1098E000FFF7B5F8327820F0FF00024370212046E0
:1098F000FFF75EF800279AE040B970212046FFF795
:10990000A6F8C0F301403060002790E001287FF402
:10991000E7A91B68032B00F2878070212046FFF720
:1099200096F833681B0403F4403320F440321A43A2
:1099300070212046FFF73CF8002778E040B97021FD
:109940002046FFF784F8C0F3804030602F466EE079
:1099500001287FF4C5A91B68012B67D87021204618
:10996000FFF775F833689B0403F4802320F480220A
:109970001A4370212046FFF71BF8002757E040B933
:1099800070212046FFF763F8C0F3015030602F4686
:109990004DE001287FF4A4A970212046FFF757F875
:1099A00033681B0503F4401320F440121A4370215E
:1099B0002046FEF7FDFF002739E000287FF4D0A9FC
:1099C0006F212046FFF743F8C0F3090030602F46AF
:1099D0002DE048B939212046FFF739F800273060DB
:1099E00025E000BFFFFF0F0001287FF479A91A6866
:1099F00039212046FEF7DCFF002718E030B93A2174
:109A00002046FFF724F82F46306010E001287FF44D
:109A100067A91A683A212046FEF7CAFF002706E028
:109A2000042704E0102702E0102700E01027384642
:109A3000F8BD07B5019229B9024601AB0120FFF735
:109A40007DF800E0082003B05DF804FB10B4134675
:109A50000446084619B9224610BCFFF76FB8082023
:109A600010BC704738B522210020FEF7F0FF18B96E
:109A70000A4B186806F0EEF9094B0A4CDD68606A7B
:109A80002B689B6998472B6820681B6998472B684F
:109A900060681B699847012038BD00BF2851FF1F2F
:109AA0000C550200A017FF1F70B5534E5348544C7D
:109AB00006F068F9F5686B6803F16402A26003F1CF
:109AC000A402E26003F1C402226103F592722260F3
:109AD00003F5A272626003F5D272626203F5E2726C
:109AE000A26203F5617203F18400A26103F5697259
:109AF00003F57173E3612B6822621B69606198470B
:109B00002B6820691B6998472B68E0681B69984798
:109B10002B68E0691B6998472B68206A1B69984786
:109B20002B68A069DB6898472B6820681B699847F9
:109B30002B6860681B6998472B68A068DB689847AA
:109B40002B68606ADB6898472B68A06ADB689847D7
:109B50002B68A0699B6998472A4B32691A606B6829
:109B6000294903F531735360284B5A690A60284923
:109B7000C2F804122749C2F8081200260121117008
:109B80005670254A1A62254ADA61254A9A61254AA1
:109B90005A62254A9A63254A5A63254A9A62254A97
:109BA000DA62254A9A64254A5A64254A5A65254A42
:109BB0001A65254ADA64254A1A66254ADA65322288
:109BC000DA604FF4F0729A600220224A19749A65A2
:109BD000FEF78EFE2B68A06ADB689847A06A1E4CD1
:109BE000042343752B681B68984723689847A3682C
:109BF0003046BDE8704018470C5502002C51FF1F3D
:109C0000A017FF1FB853FF1F2851FF1FC82EFF1FAB
:109C1000659A0100E58801000D8A01004D8A010066
:109C2000498A0100458A01004D9A0100339A0100DA
:109C3000D78901001D8B0100CD8901000D8B01002A
:109C4000CD8801009986010079860100F188010024
:109C50008D8601004D880100C409FF1F18B9034B10
:109C60001B680B6070470820704700BFC453FF1F7C
:109C7000014B00225A607047C82EFF1F0428F8B518
:109C800014464FD005D8022833D000F28F8038B167
:109C900004E0062871D069D3FC287AD00420F8BDEE
:109CA000136833F0030240F0888013F0010F444D35
:109CB000444E03D0F3681B681B6906E0F7686868C8
:109CC0003B68DB6898473B689B69686898472068F1
:109CD00010F0020404D0F36828681B681B6964E074
:109CE000F66828683368DB689847336828689B699A
:109CF00015E01468334B64B1DC686068236800F5D4
:109D0000F270DB6898476068236800F5F2709B6921
:109D10004BE0DB6858681B689B6800F5F270984759
:109D20002046F8BD1668264D264B4EB1012E11D1A6
:109D3000DF6828693B68DB6898473B685B6906E039
:109D4000DF6828693B68DB6898473B689B6928693E
:109D5000984709E0DE68286933681B6998473368CB
:109D600028691B6A9847064626601FE0154B144A6F
:109D7000DB6890691B681B6A05E0124B104ADB68C0
:109D8000D0691B681B6A9847003018BF012020600B
:109D90000CE014680A4D0B4B54B1DC682869236849
:109DA000DB689847236828699B6998470020F8BDBD
:109DB000DB6828691B681B69B1E71020F8BD00BF8C
:109DC000D817FF1F0C550200144B70B5DD68144CFA
:109DD0002B68A0689B6998472B68E0689B68984748
:109DE0002B6820699B6898472B6860699B68984737
:109DF0002B6820689B6898472B6860689B68984729
:109E00002B68A0699B6898472B68E0699B68984716
:109E10002B68A0689B68BDE8704018470C5502008D
:109E2000D817FF1F034B044A1B680146002006F0A9
:109E30005CB800BFC053FF1FC453FF1F014B18681D
:109E400006F08BB8C053FF1F022804BF0B4B93F8DA
:109E5000D00020B90A4BDB681B685B690AE0012867
